:0200000480007A
:10000000970500009385C547732510FC6B10B5005C
:10001000EF00C046130510006B00050017650100D6
:100020001305C5A417660100130606B63306A640DD
:1000300093050000EF009053171500001305C5C38A
:10004000EF00D03EEF00D048EF0080006F00503F3F
:1000500037450180130101F3130505842322910C18
:100060002326110C2324810C2320210D232E310B58
:10007000232C410B232A510B2328610B93040102EB
:10008000EF00006513870400930700009306400209
:100090002320F7009387170013074700E39AD7FE42
:1000A0001304000013071000B74901801309400230
:1000B00083A70400930504001385C986638687001F
:1000C000EF00006113070000130414009384440040
:1000D000E31024FF63140718374501801305458A90
:1000E000EF00005FEF00401F374501801305458B8F
:1000F000EF00005EEF000025374501801305858C79
:10010000EF00005DEF004030374501801305858D1D
:10011000370400FFEF00C05B93040000374B018001
:10012000B74A0180374A0180B74901801309440169
:1001300023209400930504001305CB8EEF00405953
:100140009385040013858A8FEF00805893850400FF
:100150001305CA90EF00C0571385C99113044400DA
:10016000EF00005793841400E31424FD3745018009
:1001700013054593EF00C055B7570180938787005B
:100180002326F10037690180B7050080B757018049
:1001900013074000938787041306C1009385452801
:1001A000130500011309C9A72328F100232CE1003E
:1001B000232EE100232A2101EF00806F37450180C3
:1001C00013054595EF00C0508327C101930400003B
:1001D000374A0180B749018063860704832781017C
:1001E0001304000063860702B387970213850999F9
:1001F000B387870093972700B307F90083A507000B
:1002000013041400EF00C04C83278101E36EF4FC5B
:1002100013058A86EF00C04F8327C1019384140021
:10022000E3EEF4FA3745018013058599EF00404E5F
:100230008320C10C0324810C8324410C0329010C6D
:100240008329C10B032A810B832A410B032B010B4A
:10025000130500001301010D678000003745018080
:100260001305C587EF00C0466FF01FE79307000036
:100270006388070037150080130545C76F00101B02
:100280006780000083A7450003A70500131525001C
:10029000B386A7003307A70083A7850003270700BD
:1002A00083A606003385A700B307D7002320F500F7
:1002B00067800000F32730CC3767018093962700D2
:1002C0001307C7AC3307D7002320F70093B71700F5
:1002D0006B8007006780000037450180130101FF34
:1002E0001305459A2326110023248100EF00403E88
:1002F000930740006B800700732700CC37540180C0
:100300001304840893172700B307F40023A0E70021
:10031000930710006B80070003250400EF000043E3
:1003200003254400EF00804203258400EF000042D3
:100330000325C400032481008320C10013010101AF
:100340006F00C040130101FF232611002324810008
:10035000930740006B800700F32700CC13B72700FA
:100360006B20070013071000637AF70613B73700F6
:100370006B20070037640180130720001304C4AB0F
:100380006388E70493972700B307F4001307D000AE
:1003900023A0E7006B3000006B30000093071000D3
:1003A0006B80070003250400EF00403A032544005A
:1003B000EF00C03903258400EF0040390325C40055
:1003C000032481008320C100130101016F00003864
:1003D0009307C0002324F4006FF0DFFB13C717005E
:1003E0006B200700376401801304C4AB63980700D7
:1003F0009307A0002320F4006FF0DFF99307B0000B
:100400002322F4006FF01FF9130101FFB7070080EA
:100410002326110023248100130740009387472BD4
:100420006B10F700F32730CC376401801304C4ACA1
:10043000139727003307E4002320F70093B7170032
:100440006B80070003250400EF00403003254400C3
:10045000EF00C02F03258400EF00402F0325C400C8
:10046000032481008320C100130101016F00002ECD
:10047000EF008058130500006B000500732500FC99
:100480006B00050097510100938141381701007FEF
:10049000130141B793050040732610CCB385C50204
:1004A0003301B140F32630CC63860600130500000B
:1004B0006B0005006780000063080520130101F54B
:1004C0002324810A232E31092326110A2322910A8B
:1004D0002320210B232C4109232A510923286109B8
:1004E00023267109930905000345050013841900AB
:1004F0006308051CB7340000B74A0180138A050061
:100500001309500293849480938A4A9B63042505BF
:10051000EF00C06F03450400130B140013040B001D
:10052000E31605FE330534418320C10A0324810A02
:100530008324410A0329010A8329C109032A810965
:10054000832A4109032B0109832BC1081301010BE5
:1005500067800000130504009306D0001306100006
:1005600003470500130B1500930707FE93F7F70FDA
:1005700063E8F600B317F600B3F79700639207102D
:100580009307A002630AF7001306A0009305010475
:10059000EF00502F032B010483470B001307E002E9
:1005A00013051B006382E70E938747FB93F7F70F52
:1005B0001307E0026364F70293972700B38757019C
:1005C00083A707006780070003471B009307800687
:1005D000630AF708130B0500130515002300210516
:1005E00033058540635AA0089307040013071104DC
:1005F0003306A40083C6070093871700130717006C
:10060000A30FD7FEE398C7FE130515009307010853
:10061000B387A70093060A00130601049305001090
:1006200013050100238007FCEF00D02A130401000A
:10063000B30BA100635AA000034504001304140087
:10064000EF00C05CE39A8BFE03451B0013042B00F4
:10065000E31E05EA6FF01FED03471B009307C0067A
:10066000E31AF7F613053B00230021053305854007
:10067000130B2B00E34AA0F6130510006FF01FF9CF
:1006800013050B006FF0DFED03471B009307A0027B
:10069000631AF70083472B0013053B00130B2B0055
:1006A0006FF09FF01306A00093050104EF00901D6A
:1006B000032B010483470B0013051B006FF0DFEED3
:1006C000130510006FF05FE61305F0FF6780000070
:1006D000130101FC130341022322B102930503001D
:1006E000232E11002324C1022326D1022328E10254
:1006F000232AF102232C0103232E11032326610058
:10070000EFF09FDB8320C10113010104678000002B
:10071000130101FF23248100232611001304050087
:1007200003450500630C05001304140013041400B2
:10073000EF00C04D0345F4FFE31A05FE8320C1001E
:10074000032481001301010167800000130101FFF0
:10075000232291002326110023248100232021013C
:100760009307F0009304050063FCA7043749018058
:100770009306000013040002130909A71304C4FF21
:10078000B3D7840093F7F7003307F90063940700A9
:100790006388060003450700EF00404793061000FA
:1007A000E31E04FC032481008320C1008324410054
:1007B000032901001305A000130101016F0000458A
:1007C000B7470180938707A7B384A70003C5040038
:1007D000EF00C043032481008320C1008324410033
:1007E000032901001305A000130101016F0000425D
:1007F000130101FE232E1100232C8100232A9100D6
:100800002328210123263101F32700FC6B800700F8
:10081000F32750CCF32930CC732700CC732600FC8F
:1008200093962700B76701809387C7ADB387D7003A
:1008300083A4070003A4040183A6C40033A989008C
:10084000930704003309D9003384360363D4F900D5
:10085000938709003304F40083A684003304C402A0
:10086000B307E9023304D4003304F40033098900E8
:10087000635E240183A7040083A5440013050400DC
:1008800013041400E7800700E31689FE93B91900EA
:100890006B8009008320C10103248101832441016D
:1008A000032901018329C1001301010267800000AF
:1008B000130101FC232E1102232C8102232A910211
:1008C0002328210323263103F32620FC732810FC60
:1008D000732400FCF32750CC1307F0016344F70C9A
:1008E000B30804031307100063D4A80033471503AB
:1008F00063C8E60C63D8E70A9386F6FF3343E50244
:10090000930803006396F6003365E502B3086500BB
:10091000B3C4880233E9880263CA040B930610004B
:1009200033C70403630607009306070033E7040395
:10093000B76901809389C9AD232EE1001307C10077
:100940002326B1002328C100232CD1003303F30256
:1009500093972700B387F90023A0E700232A6100BB
:10096000634C90066300090433848402232A8100C7
:100970006B000900F32750CC732520CC93972700F8
:10098000B389F90083A7090083A6870003A707009E
:1009900083A547003305D500E70007009307100043
:1009A0006B8007008320C103032481038324410358
:1009B000032901038329C102130101046780000098
:1009C00013870600E3CAE7F26FF0DFFD13070000AC
:1009D000930610006FF0DFF513870400635498004E
:1009E00013070800B70700809387077F6B10F70095
:1009F000EFF01FE06FF01FF7F32750CC3707FF0031
:100A0000B387E70093978700732700B023A0E70020
:100A1000732710B023A2E700732720B023A4E700B8
:100A2000732730B023A6E700732740B023A8E70060
:100A3000732750B023AAE700732760B023ACE70008
:100A4000732770B023AEE700732780B023A0E702BE
:100A5000732790B023A2E7027327A0B023A4E70274
:100A60007327B0B023A6E7027327C0B023A8E7021C
:100A70007327D0B023AAE7027327E0B023ACE702C4
:100A80007327F0B023AEE702732700B123A0E70479
:100A9000732710B123A2E704732720B123A4E7042E
:100AA000732730B123A6E704732740B123A8E704D6
:100AB000732750B123AAE704732760B123ACE7047E
:100AC000732770B123AEE704732780B123A0E70634
:100AD000732790B123A2E7067327A0B123A4E706EA
:100AE0007327B0B123A6E7067327C0B123A8E70692
:100AF0007327D0B123AAE7067327E0B123ACE7063A
:100B00007327F0B123AEE706732700B823A0E708E8
:100B1000732710B823A2E708732720B823A4E70897
:100B2000732730B823A6E708732740B823A8E7083F
:100B3000732750B823AAE708732760B823ACE708E7
:100B4000732770B823AEE708732780B823A0E70A9D
:100B5000732790B823A2E70A7327A0B823A4E70A53
:100B60007327B0B823A6E70A7327C0B823A8E70AFB
:100B70007327D0B823AAE70A7327E0B823ACE70AA3
:100B80007327F0B823AEE70A732700B923A0E70C58
:100B9000732710B923A2E70C732720B923A4E70C0D
:100BA000732730B923A6E70C732740B923A8E70CB5
:100BB000732750B923AAE70C732760B923ACE70C5D
:100BC000732770B923AEE70C732780B923A0E70E13
:100BD000732790B923A2E70E7327A0B923A4E70EC9
:100BE0007327B0B923A6E70E7327C0B923A8E70E71
:100BF0007327D0B923AAE70E7327E0B923ACE70E19
:100C00007327F0B923AEE70E67800000974201001A
:100C10009382C24883A20200732320CC13130301E2
:100C20003363A30023A062006780000093050500E2
:100C30009306000013060000130500006F00006219
:100C4000130101FF930500002324810023261100D6
:100C500013040500EF00406AB767018003A587A56C
:100C60008327C50363840700E7800700130504009A
:100C7000EFF01F80130101FF23248100B75701808B
:100C8000375401801304440093874700B38787409B
:100C9000232291002326110093D42740638004026D
:100CA0009387C7FF33848700832704009384F4FF6E
:100CB0001304C4FFE7800700E39804FE8320C1000B
:100CC0000324810083244100130101016780000097
:100CD000130101FF232481002320210137540180C7
:100CE0003759018093070400130909003309F940BB
:100CF0002326110023229100135929406300090281
:100D00001304040093040000832704009384140058
:100D100013044400E7800700E31899FE375401806C
:100D20003759018093070400130949003309F9403A
:100D300013592940630009021304040093040000BE
:100D4000832704009384140013044400E780070001
:100D5000E31899FE8320C10003248100832441000D
:100D60000329010013010101678000001303F00053
:100D700013070500637EC3029377F7006390070AA9
:100D800063920508937606FF1376F600B386E600B5
:100D90002320B7002322B7002324B7002326B7005F
:100DA00013070701E366D7FE63140600678000009F
:100DB000B306C3409396260097020000B386560000
:100DC0006780C6002307B700A306B7002306B70055
:100DD000A305B7002305B700A304B7002304B70099
:100DE000A303B7002303B700A302B7002302B70091
:100DF000A301B7002301B700A300B7002300B70089
:100E00006780000093F5F50F93968500B3E5D50054
:100E100093960501B3E5D5006FF0DFF693962700B2
:100E200097020000B386560093820000E78006FA1E
:100E300093800200938707FF3307F7403306F600DD
:100E4000E378C3F66FF0DFF3130101FF374301804E
:100E5000232681009302050093870500130353A8FE
:100E600003C70700138E0700938717003308E300BA
:100E70008348080093F88800E39408FE13080700ED
:100E80001307D0026306E8101307B002630CE806EC
:100E9000B70F008093CFFFFF1304000063800608A4
:100EA00013070001138F06006382E610B3F3EF030C
:100EB000930800001305000013039000930E9001A7
:100EC00033DEEF03130708FD6378E3001307F8FB35
:100ED00063E4EE06130798FC6358D70663CA080458
:100EE0009308F0FF636AAE006302AE089308100037
:100EF0003305E5033305A7009387170003C8F7FF01
:100F00006FF05FFCB70F008003C8070093CFFFFFAF
:100F100093072E0013040000E39406F81307000360
:100F20006300E80C130FA0009306A0006FF01FF8F9
:100F30009308F0FF6FF05FFC1307F8F963E6EE002B
:100F4000130798FAE34CD7F863C608026304040059
:100F50003305A04063060600639608042320B6000C
:100F60000324C1001301010167800000E3C6E3F818
:100F70006FF0DFF71307200223A0E20013850F00B4
:100F8000E30006FE9385F7FF13850F006FF01FFD4A
:100F900003C80700B70F008093072E00130410004A
:100FA0006FF0DFEF930F05006FF0DFFD1307000315
:100FB000631AE80003C70700130580051377F70DD0
:100FC0006306A700130F00016FF05FEE03C8170060
:100FD000130F000193872700930600016FF01FEDA8
:100FE00003C70700930680051377F70DE300D7FECC
:100FF000130F8000930680006FF05FEB1307100063
:101000006388E600130740026364D7006FF0DFE3F4
:10101000130101FF23261100EF0040408320C1008F
:10102000930760012320F50013050000130101015F
:1010300067800000130710006304E60213074002F4
:101040006360C70237670180930705000325C7A5C2
:101050009306060013860500938507006FF0DFDE18
:10106000130101FF23261100EF00403B8320C10044
:10107000930760012320F50013050000130101010F
:1010800067800000130710006304E60213074002A4
:101090006360C70237670180930705000325C7A572
:1010A0009306060013860500938507006FF0DFD9CD
:1010B000130101FF23261100EF0040368320C100F9
:1010C000930760012320F5001305000013010101BF
:1010D00067800000130101F8232C8106B7670180A7
:1010E000232E1106232A910603A4C7A563CE050863
:1010F00093078020231AF1002324A100232CA100B0
:10110000638605049387F5FF9304F0FF9305810040
:10111000130504002328F100232EF100231B910066
:10112000EF008030635695009307B0082320F40049
:1011300083278100238007008320C10703248107C0
:101140008324410713010108678000009304F0FF26
:10115000930581001305040023280100232E0100BC
:10116000231B9100EF00402C635695009307B008B5
:101170002320F4008320C10703248107832441072F
:1011800013010108678000009307B0082320F400D2
:101190001305F0FF6FF01FFE130101F8232C8106E9
:1011A000232E1106232A9106930706001304050037
:1011B000634E060813860600930607001307802077
:1011C000231AE1002324B100232CB1006384070417
:1011D0009387F7FF9304F0FF930581002328F10024
:1011E000232EF100231B9100EF000024635695008D
:1011F0009307B0082320F400832781002380070091
:101200008320C107032481078324410713010108B8
:10121000678000009304F0FF9305810023280100FC
:10122000232E0100231B9100EF0000206356950040
:101230009307B0082320F4008320C107032481070B
:101240008324410713010108678000009307B00859
:101250002320F5001305F0FF6FF01FFEB767018034
:1012600003A787A583278714638C070403A7470078
:101270001308F001634EE806131827006306050201
:10128000338307012324C30883A88718130610009B
:101290003316E600B3E8C80023A417192324D3109B
:1012A000930620006304D5021307170023A2E7006A
:1012B000B387070123A4B70013050000678000006F
:1012C0009307C7142324F7146FF05FFA83A6C71897
:1012D0001307170023A2E70033E6C60023A6C718AA
:1012E000B387070123A4B70013050000678000003F
:1012F0001305F0FF67800000130101FDB76701804F
:10130000232C410103AA87A52320210323261102B0
:1013100003298A142324810223229102232E3101DE
:10132000232A5101232861012326710123248101ED
:1013300063000904130B0500938B0500930A10004A
:101340009309F0FF832449001384F4FF63420402ED
:1013500093942400B304990063840B0483A744107E
:10136000638077051304F4FF9384C4FFE31634FF0E
:101370008320C10203248102832441020329010244
:101380008329C101032A8101832A4101032B010121
:10139000832BC100032C810013010103678000002F
:1013A0008327490083A644009387F7FF638E870451
:1013B00023A20400E38806FA8327891833978A005A
:1013C000032C4900B377F70063920702E780060019
:1013D0000327490083278A1463148701E38427F9CC
:1013E000E38807F8138907006FF0DFF58327C91832
:1013F00083A544083377F700631C070013050B002F
:10140000E78006006FF0DFFC232289006FF09FFA6F
:1014100013850500E78006006FF09FFBB76701802A
:1014200003A5C7A567800000130101E12326111E53
:10143000232A511D2328611D2320A11D138B050084
:10144000130D06002326D1002324811E2322911E82
:101450002320211F232E311D232C411D2326711DE6
:101460002324811D2322911D232EB11B930A0500E5
:10147000EF50102883270500138507002320F1046F
:10148000EF70902A8357CB002328010E232A010EE8
:10149000232C010E232E010E93F70708232EA10201
:1014A0006388070083270B01639407006F10C05601
:1014B000B74701809387C7BC232AF10083470D00FB
:1014C000930BC110B74901802322710F2326010E0F
:1014D0002324010E23280100232C010023220104D0
:1014E000232C0102232401042326010423220100CA
:1014F00093880B00938989D4638E072013040D0011
:1015000093065002638AD73C8347140013041400E7
:10151000E39A07FEB304A441630EA41F8326C10E01
:101520008327810E23A0A801B38696009387170016
:1015300023A298002326D10E2324F10E93067000D7
:101540009388880063C2F63A03274100834704006A
:10155000330797002322E100638E071A83441400A7
:10156000A303010C130414001303F0FF130A00007B
:1015700013090000130CA005930C9000930DA0021A
:1015800013041400938704FE6364FC0403274101E1
:1015900093972700B387E70083A7070067800700BA
:1015A000130A0000938704FD8344040093162A0065
:1015B000338A4601131A1A00338A4701938704FDC0
:1015C00013041400E3F2FCFE938704FEE370FCFCBA
:1015D0006382041423069114A303010C130C10005E
:1015E000930C1000130DC114930D000013030000A1
:1015F00023260102232A010223280102937F2900C6
:1016000063840F00130C2C00137F49088327C10E3D
:1016100063160F0033088A41E34E006B8346710C5A
:10162000638A06028326810E1306710C23A0C8006C
:1016300093871700130610009386160023A2C80094
:101640002326F10E2324D10E130670009388880000
:101650006340D65C638A0F028326810E1306810CD9
:1016600023A0C80093872700130620009386160046
:1016700023A2C8002326F10E2324D10E13067000E6
:1016800093888800E346D67493060008E302DF4897
:1016900033089341E34A005593760910E39E0632DE
:1016A0000327810EB387970123A0A8011307170012
:1016B00023A298012326F10E2324E10E9306700045
:1016C00063C2E66A938888001379490063060900BB
:1016D000B3048A416348906A63548A01130A0C0078
:1016E00003274100330747012322E100E39C075A07
:1016F0002324010E63880D0093850D0013850A00D5
:10170000EF20900593880B00130D040083470D0014
:10171000E39607DE8327C10E638407006F109035C0
:101720008357CB0093F70704638407006F20404280
:101730008320C11E0324811E032541008324411EF2
:101740000329011E8329C11D032A811D832A411DEE
:10175000032B011D832BC11C032C811C832C411CDA
:10176000032D011C832DC11B1301011F6780000085
:1017700013850A00232E110123246100EF504077C6
:1017800083274500138507002326F104EF70C079F5
:101790009307050013850A00938407002324F104AE
:1017A000EF50007583278500032381008328C10142
:1017B000232CF102638404006F10800F8344040023
:1017C0006FF01FDC83440400136909026FF05FDBD4
:1017D0001369090193770902638A07688327C100A7
:1017E0009387770093F787FF03A7470083AD070030
:1017F000938787002326F100930C07006342076A52
:101800001307F0FF130C09006308E30033E79D01A1
:10181000137CF9F7E300077663840C006F10804CAB
:10182000130790006374B7016F10C04B938D0D03C5
:10183000A307B11B13090C00930C1000130DF11A30
:101840008347710C130C030063549301138C0C0039
:1018500023260102232A010223280102930D0000FE
:10186000E38E07D8130C1C006FF05FD913690901D0
:10187000937709026384075C8327C100138777008D
:10188000137787FF832D0700832C4700930787007A
:101890002326F100137CF9BF13070000A303010CFA
:1018A0009306F0FF6302D362B3E69D011379FCF760
:1018B000E39E0640E314030CE312076C937C1C00C8
:1018C000130D011BE38E0CF693070003A307F11A17
:1018D000130DF11A6FF0DFF6B304A441E310A4C5B1
:1018E000834704006FF05FC71306410E93050B009A
:1018F00013850A00EF708076E31405E293880B00ED
:101900006FF09FC493778900638407006F10800194
:101910008327C1001305010B232E11019387770044
:1019200093F787FF83A5070003A6470093878700E7
:10193000232461002326F100EF1041788327010B57
:101940008328C101032381002328F10E8327410B43
:10195000232AF10E8327810B232CF10E8327C10B41
:10196000232EF10E1305010F232E110123246100F4
:10197000EF5000502326A10C930720000323810081
:101980008328C1016314F5006F10405B93071000BA
:101990006314F5006F10807A930710066394F400C7
:1019A0006F20000D930710046394F4006F1010452E
:1019B00013F7F4FD9307F0FF2324E1066314F3000B
:1019C0006F10900F930770046314F7006F200019D5
:1019D000032EC10F232A2107832E010F032F410F4E
:1019E000832F810F9367091063540E006F10D07D11
:1019F000232E010613890700930D0000032781069B
:101A0000930760046314F7006F10D01A9307500413
:101A1000232411036314F7006F20400C130C010BF7
:101A20009307010D1307C10C930603001308C10DA2
:101A30001306200093050C0013850A00232261027F
:101A40002328D10B2320D103232AE10B232EE101EC
:101A5000232CF10B2328F101232EC10B2324C101D8
:101A6000EF40000F0327810693077004032E8100C7
:101A7000832F0101032FC101832E010203234102A1
:101A800083288102130D05006304F7006F200035E1
:101A90008327410793F71700638407006F204003F3
:101AA0008327C10D0327C10CB387A7412328F10069
:101AB0002328E10203278106930770046314F700CB
:101AC0006F10500103278106930760046314F70029
:101AD0006F10102F8327010303278106930510043D
:101AE0009387F7FF2326F10C93F6F40F13060000FB
:101AF0006318B7009386F60093F6F60F13061000EE
:101B0000230AD10C9306B00263DA0700032701030E
:101B1000930710009306D002B387E740A30AD10CC5
:101B20009306900063C4F6006F20801F1308310EE7
:101B3000130508001306A000130E3006B3E6C70213
:101B400093050500138307001305F5FF938606032D
:101B5000A38FD5FEB3C7C702E3426EFE9387070388
:101B600013F6F70FA30FC5FE9387E5FF63E40701A4
:101B70006F2040279306610D6F00800003C60700A9
:101B80002380C6009387170093861600E39807FF0B
:101B90009307510EB387B7401307610DB307F700E2
:101BA0009306410DB387D7402322F10483264104D5
:101BB0000327010193071000B38CE60063C4E7001C
:101BC0006F20801A8327C103B38CFC008327410751
:101BD00013CCFCFF135CFC4113F9F7BF1369091028
:101BE00033FC8C0123260102232A0102232801024F
:101BF0008327C107639407006F1000759307D00215
:101C0000A303F10C13030000130C1C006FF01F9FC3
:101C10001306410E93050B0013850A002320610271
:101C2000232EE1012324F101EF704043E316050860
:101C30008327C10E03230102032FC101832F8100DB
:101C400093880B006FF01FA10326810E032701016B
:101C50009306100023A0A801938717009304160091
:101C6000938C8800E3D4E6329306100023A2D800B8
:101C70002326F10E2324910E93067000E3CE963CAA
:101C80000327C1038326010493841400B387E7006C
:101C900023A0DC0023A2EC002326F10E2324910EC6
:101CA00093067000938C8C00E3CA963C8326010F48
:101CB000138814009305010A2328D10A8326410FB3
:101CC0001305010B232EF100232AD10A8326810F4D
:101CD000232401012320010A232CD10A8326C10FCA
:101CE0002322010A2324010A232ED10A2326010AD2
:101CF000EFD01074832701010328810093888C00A2
:101D00009386F7FF130608008327C101E304052A21
:101D100013071D00B387D70023A0EC0023A2DC002B
:101D20002326F10E2324010F13077000E3420777E7
:101D300013870C0113862400938C08009308070076
:101D4000832641041307410D23A0EC00B387D7007D
:101D500023A2DC002326F10E2324C10E13077000FA
:101D6000E354C7961306410E93050B0013850A0032
:101D7000EF70C02E631205748327C10E93880B0089
:101D80006FF09F94930600010327810E63C49600B1
:101D90006F101006B7460180938E86D31309000199
:101DA000930C70006F00C000938404FF635A990481
:101DB000938707011307170023A0D80123A2280146
:101DC0002326F10E2324E10E93888800E3DEECFC49
:101DD0001306410E93050B0013850A002324D1013D
:101DE000EF70C027631A056C938404FF8327C10E2C
:101DF0000327810E832E810093880B00E34A99FA12
:101E0000B38797001307170023A0D80123A29800D7
:101E10002326F10E2324E10E93067000E3DEE68A0A
:101E20001306410E93050B0013850A00EF70002383
:101E3000631405688327C10E6FF01F8A8326C100D3
:101E40009377090113874600E396072C93770904DB
:101E5000639407006F10C02C8327C100930C00000F
:101E60002326E10083DD07006FF0DFA28326C10097
:101E70009377090113874600E394072893770904B1
:101E8000639407006F10C0258327C1002326E1005B
:101E9000839D070093DCFD4113870C00E3520796F6
:101EA0003337B001B3079041B38CE7401307D0023A
:101EB000A303E10C9306F0FFB30DB041130C09002E
:101EC00013071000E312D39E93061000E306D79485
:101ED000930620006300D72C130D011B1396DC0121
:101EE00093F67D0093DD3D0093860603B36DB60146
:101EF00093DC3C00A30FDDFE33E69D0193050D004E
:101F0000130DFDFFE31C06FC93771C00638E072A6C
:101F100093070003638AF62A9385E5FFA30FFDFE6E
:101F20009307011BB38CB74013090C00138D0500F8
:101F30006FF01F918327C100A303010C03AD0700BD
:101F40009386470063140D006F10C0089307F0FFDD
:101F5000E308F32E130603009305000013050D009C
:101F6000232ED1002326110123246100EF50D00C31
:101F7000032381008328C1008326C101930D05003E
:101F8000631405006F10C05AB30CA5418347710C50
:101F900013CCFCFF135CFC412326D1002326010255
:101FA000232A01022328010233FC8C01930D000037
:101FB00013030000E398078A6FF04FE40327C10082
:101FC000A303010C130C100083270700130747001D
:101FD0002326E1002306F114930C1000130DC11405
:101FE0006FF08FE0136C090193770C02E38E070208
:101FF0008327C10013877700137787FF9307870034
:10200000832D0700832C47002326F10013071000BF
:102010006FF0DF8883440400136909086FF04FD61E
:102020008327C1003787FFFF1347078383AD07006E
:102030002314E10C93874700374701802326F100E2
:10204000930787B9930C0000136C2900232CF1002F
:1020500013072000930480076FF05F848326C1007C
:102060009377090203A70600938646002326D10032
:10207000E392070693770901E396077493770904BF
:10208000638407006F10C01713790920E30C0972ED
:1020900083274100130D04002300F7006FF00FE7C2
:1020A000834404009307C006E380F4121369090116
:1020B0006FF00FCD8344040093078006E38EF41283
:1020C000136909046FF0CFCB8344040013698900BE
:1020D0006FF00FCB8327C1008344040003AA0700DD
:1020E000938747002326F100635C0AC8330A404106
:1020F000136949006FF0CFC88344040013691900C5
:102100006FF00FC88347710C83440400639A07C6BD
:1021100093070002A303F10C6FF08FC68344040001
:10212000136949006FF0CFC59307B00283440400E0
:10213000A303F10C6FF0CFC4834404009306140092
:102140006394B4016F105047938704FD1384060015
:102150001303000063E8FCC2834404001318230047
:1021600033086800131818003303F800938704FD40
:1021700013041400E3F2FCFE6FF0CFC093061000CE
:102180006314D7006F10501493062000130C09003D
:10219000E314D7D4130D011B8327810193F6FD00AF
:1021A00093DD4D00B386D70003C606009396CC019D
:1021B000B3EDB60193DC4C00A30FCDFEB3E69D0159
:1021C000130DFDFFE39A06FC9307011BB38CA74197
:1021D00013090C006FF0CFE693065006E3D696A6DF
:1021E0008326010F9305010A1305010B2328D10A49
:1021F0008326410F232EF10023241101232AD10A23
:102200008326810F2320010A2322010A232CD10ACD
:102210008326C10F2324010A2326010A232ED10A73
:10222000EFD01021832881008327C101631A053C68
:102230000327810EB7460180938686BC23A0D80071
:1022400093871700930610001307170023A2D800E6
:102250002326F10E2324E10E930670009388880054
:10226000E3C2E6460327C10C83260101635AD76205
:10227000032701048326C1039388880023ACE8FE6A
:102280000327810EB387D70023AED8FE13071700AC
:102290002326F10E2324E10E9306700063CEE6722E
:1022A000032701019304F7FF635090C293060001D6
:1022B0000327810EE3D89642930C0001130D7000A2
:1022C0006F00C000938404FFE3DE9C409387070106
:1022D0001307170023A0380123A298012326F10E2B
:1022E0002324E10E93888800E35EEDFC1306410E83
:1022F00093050B0013850A00EF605056631E051A04
:102300008327C10E0327810E93880B006FF09FFB7C
:1023100033088A41635E00B7130600018326810EED
:10232000635C0607130E0001930E70006F00C0007F
:10233000130808FF63520E07938707019386160060
:1023400023A0380123A2C8012326F10E2324D10E95
:1023500093888800E3DEDEFC1306410E93050B0034
:1023600013850A00232E010123246100EF60104F22
:10237000631405140328C101130E00018327C10E45
:10238000130808FF8326810E0323810093880B0026
:10239000930E7000E3420EFBB3870701938616008D
:1023A00023A0380123A208012326F10E2324D10EF5
:1023B0001306700093888800635CD6AC1306410E48
:1023C00093050B0013850A0023246100EF60104978
:1023D0006314050E032381008327C10E93880B002D
:1023E00033089341635A00AB130600018326810E24
:1023F0006358060713030001130E70006F00C0003E
:10240000130808FF635E0305938707019386160090
:1024100023A0380123A268002326F10E2324D10E25
:1024200093888800E35EDEFC1306410E93050B00E3
:1024300013850A0023240101EF605042631E050644
:1024400003288100130300018327C10E130808FF2E
:102450008326810E93880B00130E7000E34603FB66
:10246000B38707019386160023A0380123A2080131
:102470002326F10E2324D10E1306700093888800C2
:10248000635CD6A01306410E93050B0013850A006A
:10249000EF60D03C631205028327C10E93880B00C6
:1024A0006FF08F9F1306410E93050B0013850A00F2
:1024B000EF60D03A630E05A263840DA693850D00EC
:1024C00013850A00EF1050296FF08FA5130C090037
:1024D0006FF09F9F37470180130600018326810E0E
:1024E000930E87D3130E0001930270006348060118
:1024F0006F004008130808FF635E0E07938707010B
:102500009386160023A0D80123A2C8012326F10E2A
:102510002324D10E93888800E3DED2FC1306410EFB
:1025200093050B0013850A002324D10323226102A3
:1025300023200103232EE1012324F101EF60103257
:10254000E31C05F603280102130E00018327C10EC8
:10255000130808FF8326810E832E81020323410284
:10256000032FC101832F810093880B009302700019
:10257000E3460EF9B38707019386160023A0D8011E
:1025800023A208012326F10E2324D10E1306700086
:10259000938888006354D6881306410E93050B0078
:1025A00013850A0023206102232EE1012324F10177
:1025B000EF60D02AE31205F08327C10E0323010246
:1025C000032FC101832F810093880B006FF00F85CB
:1025D0001306410E93050B0013850A00232E61009C
:1025E0002324E101EF609027E31805EC8327C10E57
:1025F0000323C101032F810093880B006FF0CF8864
:102600008325C10C635CB07C032701038326010191
:102610009304070063C2E634635690028326810E5A
:10262000B387970023A0A8019386160023A29800E1
:102630002326F10E2324D10E130670009388880000
:10264000E34CD63693C6F4FF0327010393D6F64135
:10265000B3F4D400B30497406348904203270103C6
:1026600093760940B304ED00639406488325C10CBA
:102670000327010163C6E50093761900E38206365D
:10268000832601040327C1031306700023A0D8008A
:102690008326810EB387E70023A2E8009386160005
:1026A0002326F10E2324D10E93888800E342D64ED0
:1026B000832601013307DD003386B6403307974098
:1026C000930C06006354C700930C070063569003F5
:1026D0000327810EB387970123A0980013071700E3
:1026E00023A298012326F10E2324E10E9306700005
:1026F00093888800E3CEE66813C7FCFF1357F741C1
:1027000033F7EC00B304E640634490006FE0DFFB76
:10271000930600010327810E63D6967C930C00017B
:10272000130D70006F00C000938404FF63DC9C7A7B
:10273000938707011307170023A0380123A29801EC
:102740002326F10E2324E10E93888800E35EEDFC3E
:102750001306410E93050B0013850A00EF6010105D
:10276000E31C05D48327C10E0327810E93880B0039
:102770006FF09FFB631C038A13090C001303000016
:10278000930C0000130D011B6FF08F8B93751900D4
:10279000639C05CC23A2D8002326F10E2324910E9E
:1027A000130770006346974E1306260093880801AE
:1027B0006FF00FD96356D0D8130700016344D700D8
:1027C0006F10005F130D70006F000001938606FF0D
:1027D000E350D70C138814009387070123A03C0112
:1027E00023A2EC002326F10E2324010F93040800FA
:1027F000938C8C00E35C0DFD1306410E93050B00DA
:1028000013850A002324D100EF605005E31605CAA2
:102810008327C10E8324810E83268100938C0B00B5
:10282000130700016FF09FFA8326C10093770C0114
:1028300013874600639C070A93770C04E382070C16
:102840008327C100930C00002326E10083DD0700ED
:10285000130710006FF08F841306410E93050B00D1
:1028600013850A00EF60807FE31805C48327C10E3B
:102870008324810E938C0B006FF08FC01306410EE2
:1028800093050B0013850A00EF60407DE31605C237
:102890008327C10E8324810E938C0B006FF00FC130
:1028A00013771900631407006FE01FE26FF05F9C5D
:1028B0008327810383440400639407006FE05FCCA7
:1028C00083C70700639407006FE09FCB136909403B
:1028D0006FE01FCB83264100130D040093D7F64110
:1028E0002320D7002322F7006FE05FE22326E100D8
:1028F00083AD0600930C0000130710006FE01FFA71
:1029000083AD06002326E10093DCFD4113870C0014
:102910006FE0DFEE83AD0600930C00002326E1009C
:102920006FE05FF70327C100832707001307470005
:102930002326E10083A5070003A6470083A687009E
:1029400083A7C7002328B10E232AC10E232CD10E42
:10295000232EF10E6FF00F8193840600E34090CC9C
:102960006FF05FCE130C09006FF00FE8B7470180DE
:10297000938787B9232CF10093770902638A072E86
:102980008327C10013877700137787FF832D070004
:10299000832C4700930787002326F1001377190043
:1029A000630E070033E79D01630A07001307000366
:1029B0002304E10CA304910C13692900137CF9BFD3
:1029C000130720006FE09FED834414001369090290
:1029D000130414006FE0DFBA1306410E93050B00D9
:1029E00013850A00EF608067E31805AC8327C10EEA
:1029F00093880B006FF0DF8A834414001369092069
:102A0000130414006FE0DFB7B74701809387C7BA9C
:102A1000232CF1006FF05FF69305000413850A0084
:102A2000EF40C05E2320AB002328AB0063140500F9
:102A30006F10003C93070004232AFB006FE05FA7A0
:102A400013050D00232411012326D100EF60C04D92
:102A50008347710C134CF5FF135CFC4123260102E4
:102A6000232A01022328010283288100930C0500F8
:102A7000337C8501930D000013030000638407007D
:102A80006FE05FDE6FE09FB7130600018326810EC3
:102A90006356966C930C0001130870006F00C00021
:102AA000938404FF63DC9C6A938707019386160076
:102AB00023A0380123A298012326F10E2324D10E4E
:102AC00093888800E35ED8FC1306410E93050B0043
:102AD00013850A00EF608058E310059E8327C10E1E
:102AE0008326810E93880B00130870006FF05FFB44
:102AF00003270101130E7000130800013307ED00D6
:102B00002324E10003274103630E070A0327C102C0
:102B1000631E070A032781031307F7FF232CE10233
:102B2000032741031307F7FF232AE1028326C10489
:102B3000032781049388880023ACD8FE8326810E66
:102B4000B387E70023AEE8FE938616002326F10E36
:102B50002324D10E6344DE16032781038346070036
:102B600003278100938C0600330697406354D600F8
:102B7000930C0600635890038326810EB387970158
:102B800023A098009386160023A298012326F10E15
:102B90002324D10E634CDE360327810393888800FB
:102BA0008346070013C6FCFF1356F641B3FCCC0066
:102BB000B38C964163449003B384D400032741034C
:102BC000E31607F40327C102630C076E0327C10253
:102BD0001307F7FF2326E1026FF05FF58326810ECE
:102BE000634898016F00C005938C0CFF635A9805E9
:102BF000938707019386160023A0380123A20801BA
:102C00002326F10E2324D10E93888800E35EDEFC98
:102C10001306410E93050B0013850A00EF60004474
:102C2000E31C058813080001938C0CFF8327C10E59
:102C30008326810E93880B00130E7000E34A98FBE5
:102C4000B38797019386160023A0380123A2980129
:102C50002326F10E2324D10E6342DE700327810365
:102C60009388880083460700B384D4006FF01FF573
:102C70008326C100937709011387460063860722E4
:102C800083AD0600930C00002326E1006FF01FD1F6
:102C90001306410E93050B0013850A00EF60003CFC
:102CA000E31C05800326810E8327C10E9308411182
:102CB00013061600938C0B006FF08F881306410EDD
:102CC00093050B0013850A00EF604039631605FE7B
:102CD0008327C10E93880B0013080001130E7000A8
:102CE0006FF09FE713790C4023280100130D011B9F
:102CF0006F0040031306A0009306000013850D002B
:102D000093850C00232E110123246100EFB080680D
:102D1000032381008328C10163840C48930D0500BF
:102D2000938C05001306A0009306000013850D0088
:102D300093850C00232E110123246100EFB0D028CD
:102D40008327010113050503A30FADFE9387170029
:102D50002328F100032381008328C101130DFDFF07
:102D6000E30A09F80327810383460700E394D7F8B1
:102D70001307F00FE380E7F863960C0093079000C9
:102D800063F4B7C5832781048325C104232E110171
:102D9000330DFD401386070013050D002324610049
:102DA000EF604021832781031306A00093060000F3
:102DB00003CE170013850D0093850C00333EC00130
:102DC000B387C701232CF102EFB0C05C032381005D
:102DD0008328C101232801006FF05FF48326810E50
:102DE00037460180130686BC23A0C80093871700CE
:102DF000130610009386160023A2C8002326F10EA6
:102E00002324D10E1306700093888800634CD606E5
:102E10006392051E0327010193761900B3E6E600CD
:102E2000639406006FE05F8A832601040327C103D1
:102E30001306700023A0D8008326810EB307F70085
:102E400023A2E800938616002326F10E2324D10E38
:102E5000634ED642938888000327010193861600AB
:102E600023A0A801B307F70023A2E8002326F10E50
:102E70002324D10E130770006344D7006FE09F84B2
:102E80006FE05FEE1306410E93050B0013850A00F9
:102E9000EF60C01C631205E28325C10C8327C10EBD
:102EA00093880B006FF0DFF693770904638C07209B
:102EB0008327C100930C00002326E10083DD070077
:102EC0006FF0DFAD1306410E93050B0013850A006A
:102ED000EF60C018631205DE8327C10E93880B00D4
:102EE0006FF04FB823A0380123A29800B387970052
:102EF000130717002326F10E2324E10E930670001A
:102F000063C4E6006FE00FFC6FE0DFE51306410EDF
:102F100093050B0013850A00EF604014631E05D86B
:102F20008327810393880B001308000183C60700E1
:102F3000130E70008327C10E6FF0DFC68327010FC9
:102F40009305010A1305010B2328F10A8327410F7A
:102F5000232411012320010A232AF10A8327810F48
:102F60002322010A2324010A232CF10A8327C10FFB
:102F70002326010A232EF10AEFC010738328810053
:102F80006342055A8347710C1307700463509722FC
:102F900037470180130DC7B823260102232A0102F7
:102FA000232801021379F9F7130C3000930D000068
:102FB000930C300013030000638407006FE09F8AC6
:102FC0006FE0CFE383274100130D04002320F700B7
:102FD0006FE0CFF393076000930C030063EE671E6E
:102FE00037470180138C0C002326D100130D07BC3A
:102FF0006FE08FDF832601040327C10313067000EF
:1030000023A0D8008326810EB307F70023A2E8008F
:10301000938616002326F10E2324D10E9388880070
:103020006346D626E3DA05E2130600FFB304B04098
:10303000E3D8C524930C0001130870006F00C00092
:10304000938404FFE3DE9C22938707019386160096
:1030500023A0380123A298012326F10E2324D10EA8
:1030600093888800E35ED8FC1306410E93050B009D
:1030700013850A00EF50907E631005C48327C10EAC
:103080008326810E93880B00130870006FF05FFB9E
:103090001386140013878C00B387D70023A2DC00AB
:1030A00023A03C012326F10E2324C10E93067000B9
:1030B000E3C0C6BE1306160093088700930C0700F2
:1030C0006FE01FC893770920638007168327C1002C
:1030D000930C00002326E10083CD07006FF01F8CC6
:1030E00093770920638607128327C1002326E10016
:1030F000838D070093DCFD4113870C006FE00FF018
:1031000093770C20638607148327C100930C00007B
:103110002326E10083CD0700130710006FE00FF8AE
:1031200093770920638C07108327C100930C00005C
:103130002326E10083CD07006FE0CFF58327C10F81
:1031400063C407128347710C13077004635C9748CC
:1031500037470180130D47B96FF01FE4B38797001D
:103160009386160023A0380123A298002326F10E8F
:103170002324D10E13067000938888006350D6CEA6
:103180001306410E93050B0013850A00EF50106DD6
:10319000631405B28327C10E93880B006FF00FCC28
:1031A00093079000E3ECB7B76FF00F8237470180C9
:1031B000130D87B86FF05FDE1306410E93050B0009
:1031C00013850A00EF509069631805AE8327C10E7E
:1031D00093880B006FF00FC7930C60006FF05FE0F7
:1031E000832601013307DD003386B6403303974061
:1031F000930C06006352C3D0930C03006FF0CFCF43
:1032000083274100130D04002310F7006FE00FD057
:103210008327C1002326E10083AD070093DCFD4135
:1032200013870C006FE08FDD8327C100930C000033
:103230002326E10083AD07006FF04FF68327C1001E
:10324000930C00002326E10083AD07006FE08FE4BC
:103250008327C100930C00002326E10083AD070003
:10326000130710006FE08FE39307D002A303F10C64
:103270006FF09FED1306410E93050B0013850A00B6
:10328000EF50D05D8357CB006FE0CFC91306410EDE
:1032900093050B0013850A00EF50505C631E05A0D8
:1032A0008325C10C8327C10E8326810E93880B00D2
:1032B000E3D405BA6FF05FD7130360006FE04FF1FE
:1032C00003270101B306ED0063F296BA938406006A
:1032D0006FF0CFB9032701039307D0FF6344F700D2
:1032E000635AE3009384E4FF93F7F4FD2324F1068B
:1032F0006FE04FFE83270101032701036340F72698
:1033000083274107930C070093F717006386070094
:103310008327C103B30CF7008327410793F70740C6
:103320006386070083270103E342F00413CCFCFF0C
:10333000135CFC4133FC8C019304700623260102CC
:10334000232A01026FE0DF8A8347710C1303000018
:10335000638407006FE00FD16FE04FAA1306410EA0
:1033600093050B0013850A00EF50504F6316059428
:103370008327810393880B001308000183C607008D
:10338000130E70008327C10EB384D4006FF01F8327
:103390001306410E93050B0013850A00EF50104CE5
:1033A000631C05908325C10C8327C10E93880B00F5
:1033B0006FF00FB0130C010B930603009307010D80
:1033C0001308C10D1307C10C1306300093050C0040
:1033D00013850A0023241103232261022328D10B21
:1033E0002320D103232AE10B232EE101232CF10B0F
:1033F0002328F101232EC10B2324C101EF204075A6
:103400008346050093070003032E8100832F0101EB
:10341000032FC101832E010203234102832881026D
:10342000130D0500930C010A6384F6088327C10C71
:10343000B3876700B306FD0093850C0013050C00ED
:10344000232ED10023281101232461002328D10B2E
:10345000232AE10B232CF10B232EC10B2320010A7D
:103460002322010A2324010A2326010AEFC0407CFB
:103470008326C1010323810083280101938706006D
:10348000631405006FE00FE28327C10D63E4D700EA
:103490006FE04FE19305000313861700232EC10C44
:1034A0002380B7008327C10DE3E8D7FE6FE08FDFED
:1034B000930C010A93850C0013050C0023241103BF
:1034C000232261022328D10B2320D103232AE10BDD
:1034D000232EE101232CF10B2328F101232EC10B14
:1034E0002324C1012320010A2322010A2324010AE3
:1034F0002326010AEFC0C073032E8100832F010130
:10350000032FC101832E010203234102832881027C
:10351000E30E05F093071000B38767402326F10CF4
:103520006FF01FF19307D002A303F10C6FF0DFA53A
:103530008347710C2326D10023260102232A01028E
:1035400023280102130C0300930C03001303000053
:10355000638407006FE00FB16FE04F8A832701019A
:103560000327C10393047006B38CE700832701038C
:103570006350F07E8327410793F70740639A075E05
:1035800013CCFCFF135CFC4133FC8C016FF01FDBA0
:103590001306410E93050B0013850A00EF50102C03
:1035A000630405006FE05FF18324C10C0327010170
:1035B0008327C10E93880B00330697406FF0CF939B
:1035C000832741070327010393F71700B3E7670039
:1035D0006356E07A639C0772832C010393046006B0
:1035E0006FF05FF937470180130D07B96FF0DF9A6D
:1035F000B7460180938E86D36FE09F8093070003C8
:103600002304F10C9307800513672900A304F10C30
:10361000232AE10693073006930D0000130DC11411
:1036200063C2673C032EC10F93F7F4FD2324F10618
:10363000232E0106832E010F032F410F832F810FAD
:103640001369291063460E38930710066388F45AED
:10365000930710046384F4006FE04FBA130C010B5E
:1036600013050C0023261103232461022328D10B08
:10367000232AE10B232CF10B232EC10BEFF0D046B4
:103680001306C10CEF50404E13860500930505004C
:1036900013050C00EFF090229307010993850700B2
:1036A0002324F1008327010B930C010A1306010860
:1036B0002328F1088327410B13850C002326C1061C
:1036C000232AF1088327810B2320010823220108E4
:1036D000232CF1088327C10B23240108232EF10892
:1036E000B707FC3F2326F108EFC0D0100328010ADA
:1036F000032E410A832E810A032FC10A93850C00F1
:1037000013050C002328010B23220103232AC10BDC
:103710002320C103232CD10B232ED101232EE10B17
:103720002328E1012320010A2322010A2324010A7C
:103730002326010AEFC0C04F032F0101832EC101D0
:10374000032E010203284102032381028328C102C0
:1037500063160500930710002326F10CB74701807C
:103760009387C7BA2322F1069306F3FF93070D0050
:103770006F00400993850C0013050C002320C1063F
:10378000232EF105232C5104232A71042328F1044C
:10379000232A1103232861022328710A2326710298
:1037A000232A510A23245102232CF10B2322F10353
:1037B000232EC10A2320C1022320010A2322010A49
:1037C0002324010A2326010AEFC080468326C10173
:1037D000032F0102832E4102032E81020328C1021E
:1037E0000323010383284103832701059386F6FF02
:1037F0009303080093020E00938F0E0013060F0030
:10380000630E05100326810093850C00232AF10224
:1038100013050C00B70703402328D1042328110304
:1038200023266102232EF1082326E10B2320010B1E
:103830002322C10B2324D10B23280108232A0108AA
:10384000232C0108EFC0007B832E010B032E410BBC
:103850000328810B0326C10B13050C002324D1037D
:103860002322C10323200103232EC100EFF00055C2
:10387000930505002328A10013050C00EFF0C06E8E
:103880000326C101832E8102032E4102232EC1088B
:103890000326010B03280102832581002320C10890
:1038A0000326410B13850C002328D1092322C108CC
:1038B0000326810B232AC109232C01092324C108D3
:1038C0000326C10B2326C1080326C106EFD05021D1
:1038D0000327410683270101832601058323010A6B
:1038E0003306F70083450600832741038322410AFC
:1038F000832F810A0326C10A232CF1062380B700F7
:103900002328D1061307F0FF232ED1000323C10281
:103910008328010393871700E39EE6E4B706FE3F82
:1039200093850C0013050C002320F102232E1101B6
:10393000232461002328710A23287102232A510AB3
:1039400023265102232CF10B2324F103232EC10A39
:103950002322C1022320010A2322010A2324010A6F
:103960002326D10AEFC0803F032381008328C101B1
:1039700083270102634EA00893850C0013050C00F9
:10398000EFC0002B032381008328C101832701029C
:10399000631805000327010193761700639A060652
:1039A000032701071306000393061700B386D70009
:1039B000635407006FE00F8F93871700A38FC7FE34
:1039C000E39CD7FE6FE00F8E930D00001389070074
:1039D000B707008033CEC7019307D002232EF1062C
:1039E0006FF09FC69305130013850A002328110169
:1039F00023246100EF3080610323810083280101CB
:103A0000130D050063000540930D05006FF09FC185
:103A10000327810793860700232EE10C0327410625
:103A200003C6F7FF8345F7006310B60213050003D2
:103A3000A38FA6FE8326C10D1386F6FF232EC10C8D
:103A400003C6F6FFE386C5FE930516001305900333
:103A500093F5F50F6306A600A38FB6FE6FE08F8483
:103A6000032741068345A700A38FB6FE6FE08F832F
:103A7000930700032304F10C930780076FF0DFB86E
:103A8000B38797009386160023A0380123A29800DD
:103A90002326F10E2324D10E13067000635CD6BAE0
:103AA0001306410E93050B0013850A00EF50005BCF
:103AB000630405006FE05FA08327C10E8326810E9B
:103AC00093880B006FF04FB9130C09006FD01FD60D
:103AD000B3066D00930C010A6FF01F96930C130050
:103AE000130C010B1308C10D9307010D1307C10C33
:103AF00093860C001306200093050C0013850A0022
:103B0000232261022328D10B2320D103232AE10B96
:103B1000232EE101232CF10B2328F101232EC10BCD
:103B20002324C101EF20C002032E8100832F010155
:103B3000032FC101832E0102032341028328810246
:103B4000130D0500B3069D01930C010A6FF0DF8E83
:103B50009307F0FF2322F1006FD09FBD63040300A1
:103B60006FD01FE7130310006FD09FE69304700619
:103B7000832781039306F00F2326010283C70700E2
:103B8000232A01026388D7040327010363D4E704CF
:103B9000B307F740032781032328F1028347170067
:103BA000638E07000326410313071700232CE1024D
:103BB00013061600232AC1026FF0DFFC0327C1029F
:103BC000832781031307170083C707002326E10219
:103BD0006FF05FFB0327C10283274103B387E70030
:103BE00003278104B387E702B38C970113CCFCFF52
:103BF000135CFC4133FC8C016FD09FFF130C010B55
:103C000013050C0023261103232461022328D10B62
:103C1000232AE10B232CF10B232EC10BEFF0C06CF8
:103C20001306C10CEF405074138605009305050080
:103C300013050C00EFF080489307010993850700F6
:103C40002324F1008327010B930C010A13060108BA
:103C50002328F1088327410B13850C002326C10676
:103C6000232AF1088327810B23200108232201083E
:103C7000232CF1088327C10B23240108232EF108EC
:103C8000B707FC3F2326F108EFC0C0360328010A1E
:103C9000032E410A832E810A032FC10A93850C004B
:103CA00013050C002328010B23220103232AC10B37
:103CB0002320C103232CD10B232ED101232EE10B72
:103CC0002328E1012320010A2322010A2324010AD7
:103CD0002326010AEFB0D075032F0101832EC10105
:103CE000032E010203284102032381028328C1021B
:103CF00063160500930710002326F10CB7470180D7
:103D0000938787B92322F1066FF01FA68327C1038B
:103D100093046006B30CF700B38C6C006FF09F85C2
:103D20009306610D6318060093060003230BD10C64
:103D30009306710D1307011B938707033386E64033
:103D40002380F6009307D60D2322F1046FD01FE6DF
:103D5000B38CFC40938C1C0013CCFCFF135CFC4127
:103D600033FC8C016FF08FDD8327410793F7170039
:103D7000639407006FD09FE56FD0DFE4639A07007C
:103D8000130C100093046006930C10006FF00FDB0F
:103D90008327C10393046006938C1700B38C6C00D7
:103DA00013CCFCFF135CFC4133FC8C016FF00FD98A
:103DB000138708006FF04FAE8327C10003A30700ED
:103DC00093874700635403001303F0FF83441400F8
:103DD0002326F100138406006FD08FFA930C0300A2
:103DE0006FF05FD6930720002322F1046FD01FDC11
:103DF0009307C00023A0FA009307F0FF2322F100ED
:103E00006FD01F938357CB0013E707049307070076
:103E10002316EB006FD01F91130101FE2326310101
:103E2000B7590180232C8100232A910023282101E6
:103E300023244101232E1100138A050013090500D4
:103E400093894963EF30D02B03A78900B71700008F
:103E50001384F7FE832447003304444193F4C4FFE2
:103E6000330494001354C4001304F4FF1314C40067
:103E7000634EF4009305000013050900EF40D0489D
:103E800083A78900B38797006308F502130509002B
:103E9000EF3050278320C101032481018324410195
:103EA000032901018329C100032A810013050000B1
:103EB0001301010267800000B3058040130509006B
:103EC000EF4090449307F0FF630AF504B767018061
:103ED0009387C7B503A7070083A68900B3848440EE
:103EE00093E41400330487401305090023A29600CD
:103EF00023A08700EF3010218320C101032481011A
:103F000083244101032901018329C100032A81007F
:103F100013051000130101026780000093050000E3
:103F200013050900EF40503E03A789009306F000F7
:103F3000B307E540E3DCF6F4B766018083A606A686
:103F400093E717002322F7003305D540B7660180B9
:103F500023AEA6B46FF09FF3638A0512130101FF2D
:103F6000232481002322910013840500930405007B
:103F700023261100EF30D0180328C4FF130784FF55
:103F8000B75501809377E8FF3306F70093854563C3
:103F90008326460003A5850093F6C6FF630AC51A6B
:103FA0002322D600137818003305D6006310080AC0
:103FB000032384FF032845003755018033076740FA
:103FC000832887001305C563B3876700137818003B
:103FD0006380A8140323C70023A6680023241301C9
:103FE0006304081E93E617002322D7002320F6005F
:103FF0009306F01F63E8F60A93F687FF9386860020
:1040000003A54500B386D50003A6060013D85700C4
:1040100093071000B3970701B3E7A700138586FF46
:104020002326A7002324C70023A2F50023A0E6002F
:104030002326E600032481008320C10013850400A9
:1040400083244100130101016F30D00B032545008B
:1040500013751500631E050237550180B387D7001D
:104060001305C5638326860093E817003308F7001D
:104070006388A6160326C60023A6C6002324D600FE
:10408000232217012320F8006FF09FF667800000BD
:1040900093E61700232ED4FE2320F6009306F01F8C
:1040A000E3FCF6F493D6970013064000636CD60E3B
:1040B00093D6670013889603138686031318380077
:1040C0003388050183260800130888FF6308D81287
:1040D00003A646001376C6FF63F6C70083A68600D4
:1040E000E318D8FE03A8C600232607012324D7001F
:1040F000032481008320C1002324E80013850400E9
:104100008324410023A6E600130101016F30807F64
:10411000631608148325C60003268600B387F600BD
:10412000032481002326B60023A4C50093E61700CC
:104130008320C1002322D700138504003307F70032
:10414000832441002320F700130101016F30807B9D
:1041500013781800B387D70063100802032584FF83
:104160003307A7408326C70003268700B387A7002D
:104170002326D60023A4C600B766018013E61700E5
:1041800083A646A62322C70023A4E500E3E4D7EADA
:10419000B767018083A507A713850400EFF0DFC789
:1041A0006FF05FE9130640016374D6021306400501
:1041B0006364D60693D6C7001388F6061386E60610
:1041C000131838006FF0DFEFB387D7006FF09FE967
:1041D0001388C6051386B605131838006FF05FEE16
:1041E00023AAE50023A8E5002326A7002324A7008F
:1041F000232217012320F8006FF0DFE303A5450019
:1042000013562640930710003396C7003366A60066
:1042100023A2C5006FF05FED13064015636CD60056
:1042200093D6F7001388860713867607131838008D
:104230006FF01FE913064055636CD60093D6270133
:104240001388D6071386C607131838006FF05FE788
:104250001308803F1306E0076FF09FE693E6170010
:104260002322D7002320F6006FF0DFDC9306450001
:10427000930700001305A5013788FFFF6F00C001F9
:10428000939717002390E6009397070193862600E3
:1042900093D70701630ED50203D7060013761700E4
:1042A0006304060093E717001357170013F627005F
:1042B000B3650701E30606FC939717002390B60049
:1042C000939707019386260093D70701E316D5FC41
:1042D0006780000093068501130700001305250081
:1042E0006F00C001131717002390F6001317070182
:1042F0009386E6FF135707016304D50483D70600AE
:10430000139607011356064193971700635406004E
:10431000136717009397070193D7070113762700B8
:1043200093E51700E30006FC131717002390B6006F
:10433000131707019386E6FF13570701E310D5FC17
:1043400067800000130101FE370E0100231D0100EC
:10435000231E0100938585019307C1011308810085
:10436000130EFEFF03D705009387E7FF9385E5FF54
:1043700063180702239F07FEE39607FF1306460014
:104380009306E10103D70700938727001306260051
:10439000231FE6FEE398D7FE1301010267800000A9
:1043A0003307A70283D8270003D30700B376C701DA
:1043B000B38616011357070193D806013307670028
:1043C00033071701935807012391D7002390E70083
:1043D000239F17FFE39807F96FF05FFA0357050073
:1043E000835725006306070037870000B3E7E7001F
:1043F0002399F50003572500B78700009387F7FF3F
:104400006304F70293076500938505011305850191
:1044100003D70700938727009385E5FF2391E500E5
:10442000E398A7FE67800000930765001305A501C8
:1044300003D7070093872700631A0702E39AA7FEB2
:10444000138725019387050093872700239F07FE85
:10445000E31CF7FE83D72501378700001307F7FF1A
:10446000B3E7E7002399F500678000001387050193
:104470009387050093872700239F07FEE31CF7FE21
:10448000B7C7FFFF2398F500B787FFFF93C7F7FF74
:104490002399F5006780000083574500130101FF51
:1044A00023229100232611002324810023202101AF
:1044B00093040500639C070C035765001304000078
:1044C0009317070193D7074163C4070A9306A50111
:1044D0001306000A63180702938764006F008000C8
:1044E00003D7070093872700239EE7FEE39AD7FEB2
:1044F000239C040013040401630CC40603D7640066
:10450000E30C07FC937707F063900704138584019D
:1045100093852400930700001307050083560700C6
:104520001307E7FF13968600B3E7C7002311F700D0
:1045300093D78600E394E5FE03D764001304840058
:10454000937707F0E38807FC1309000A6F00400126
:1045500013041400EFF01FD8634C890003D76400E4
:10456000131707011357074113850400E35207FE91
:104570008320C1001305040003248100832441002B
:1045800003290100130101016780000013F707F000
:1045900013040000631007041309F0F66F004001D4
:1045A0001304F4FFEFF09FCCE30424FD83D7440011
:1045B00013850400E39607FE8320C1001305040061
:1045C0000324810083244100032901001301010118
:1045D00067800000930645009305A50113070000BE
:1045E0006F00800083D7060013D687003367C700AB
:1045F000939787002390E600139707019386260080
:1046000013570701E390D5FE83D74400130480FFBE
:104610006FF09FF8130101FE232C8100232A9100E3
:10462000232E110023282101232631019384050024
:104630001304050063C4050A9307F0001386050000
:1046400013054500930684019305F00063D4970297
:104650009307050003D7270093872700239FE7FED2
:10466000E39AF6FE231C0400130606FFE3C2C5FE10
:1046700093F4F4009307700063D897021307840142
:104680009305240093070000835607001307E7FFF4
:1046900013968600B3E7C7002311F70093D786006F
:1046A000E394E5FE938484FF638A04009384F4FF1B
:1046B00013050400EFF01FC2E39A04FE1305000087
:1046C0008320C101032481018324410103290101C5
:1046D0008329C1001301010267800000930710FFC6
:1046E0003309B04063DEF51293058501930900009C
:1046F000930645001306F0000357840193870500D5
:10470000B3E9E90003D7E7FF9387E7FF2391E700C9
:10471000E39AD7FE23120400130909FFE34E26FD96
:10472000130900FF130710FF330999409307000096
:1047300063C6E40A3309F9009307700063CA2705CA
:104740006302090C835784011309F9FF1305040060
:1047500093F71700B3E93701EFF05FB1E31409FEF7
:104760009397090193D707416396070813950901A9
:10477000135505018320C1010324810183244101D4
:10478000032901018329C100130101026780000090
:104790009399090193D90941834784019305A401A1
:1047A000B3E9F9009399090193D90901930700002E
:1047B00003D706009386260013568700B3E7C70089
:1047C00013178700239FF6FE9317070193D707015E
:1047D000E390D5FE130989FF6FF09FF6937709FFE9
:1047E000B307F0403309F90093077000E3DA27F5C7
:1047F0006FF01FFA93091000139509011355050175
:104800006FF05FF713850900639809001315050120
:10481000135505016FF0DFEA130510006FF01FFF5D
:10482000930790FF9309000093064500E3C6F5F651
:104830006FF05FF183572501378600001306F6FFFE
:1048400093D7F700B307F0402390F5008356250176
:104850009307050113874500B376D6002391D50051
:104860006386C60213876500239205001305E5FFE2
:1048700083D607009387E7FF13072700231FD7FE80
:10488000E318F5FE239C0500678000000356250110
:1048900033F6C600631ED6001308250193060500F3
:1048A00003D6060093862600631E0600E39A06FFE1
:1048B0009385A50113072700231F07FEE39CE5FE50
:1048C0006780000013876500239205001305C5FF6C
:1048D00083D607009387E7FF13072700231FD7FE20
:1048E000E398A7FE6780000083572501130101FBB1
:1048F0002324810493C7F7FF23261104139717017C
:1049000013840500631E0700930625019307050025
:1049100003D7070093872700631C0708E39AD7FE95
:104920008357240193C7F7FF139717016300070606
:1049300093058100EFF01FF0930541021305040079
:10494000EFF05FEF8355810003554102630CB5061C
:104950009307A100130761021306010283D6070023
:10496000938727006398060A8356070013072700DA
:104970006392060AE314F6FE130500008320C104C7
:1049800003248104130101056780000093070400DC
:1049900003D707009306240193872700631A0700B3
:1049A000E388D7F803D7070093872700E30A07FEB9
:1049B0008320C104032481041305E0FF13010105D2
:1049C000678000000356A10083566102133515006D
:1049D0001307A10093076102131515001305F5FFD6
:1049E0009305C1039387270013072700631ED60092
:1049F000E384B7F80356070083D6070013072700A0
:104A000093872700E306D6FEE3EAC6F63305A04007
:104A10006FF0DFF613051000E38205F61305F0FFD3
:104A20006FF0DFF5130101FE232C8100232A910092
:104A3000232821012326310123244101232251016E
:104A40001389060093840700232E11001304050028
:104A500093890500130A0600930A0700EFF0DFA30D
:104A6000930700093309A94063DCA718B787000042
:104A70009387E7FF63DA272163840A1E03A54400B6
:104A800083A70400630AF5061387A40193874403F0
:104A900013072700231F07FEE31CF7FE930780037D
:104AA0006300F53663D0A71893070004630EF52E54
:104AB000930710076310F532B78700409387F7FF1D
:104AC0001307A00023AAF400B787FFFF23A4E40084
:104AD000239CF40023A6E4009307A000378700007E
:104AE0009387870093971700B387F4002395E70017
:104AF00023A0A4006358201D83A5840083D744010C
:104B00001308F008139615003306C4000357060077
:104B1000B376F700634AA8021308B0006346B802F0
:104B2000930706009305840103D727006304070059
:104B300093E616002391070093872700E396F5FE7E
:104B40000357060083D7440193C7F7FFB3F7E70085
:104B50002310F60083D7640133F7D70063000706FC
:104B60006392D7026398092083A7C40003D7840106
:104B700093971700B307F40083D70700B3F7E70054
:104B8000638E070213862403930684019384C40171
:104B9000130700008357060083D506009386E6FFBF
:104BA0001306E6FFB387B700B387E70013D7070103
:104BB0002391F60013771700E31E96FC6356201727
:104BC00083574400639E0712B7870000231C04002C
:104BD0009387E7FF63C82709231124018320C101BC
:104BE0000324810183244101032901018329C10098
:104BF000032A8100832A410013010102678000001B
:104C00006354090E930700F7635CF90893072400C7
:104C10001304A40193872700239F07FEE39C87FECC
:104C20006FF0DFFB93078001630AF51493075003CD
:104C30006312F51A37170000B707000493066000E7
:104C40009387F77F1307078023AAF40023A4D400D7
:104C5000239CE40023A6D400930760006FF05FE874
:104C6000231C0400B787FFFF93C7F7FF2311F4004D
:104C700093074400130484012390070093872700BF
:104C8000E31CF4FE6FF09FF5930724001304A401C6
:104C900093872700239F07FEE39C87FE6FF01FF496
:104CA0009305090013050400EFF0DF966304050087
:104CB00093091000638A0A0A03A5440083A704002D
:104CC000E314F5DC930700096302F50883578401B8
:104CD0001305040093F71700B3E9F900EFF00FD9BB
:104CE00003A544006FF05FE1E3800AEE03A54400F2
:104CF00083A70400E31AF5D8E34020E16FF09FFC9E
:104D000013050400EFF08FD6B787000013091900D0
:104D1000231C04009387E7FFE3C627F5E35E09EA57
:104D2000231104006FF09FEB930700096306F50061
:104D300013050400EFF00FDA83574400E39207FCF9
:104D4000231C0400E34E09FC6FF01FE903A6840056
:104D500083D74401131616003306C4000357060018
:104D6000B3F6E7006FF05FDE231C0400231104009C
:104D70006FF0DFE6E3080AE06FF05FE4B70780005A
:104D80009387F70F1307400023AAF400930700103E
:104D900023A4E400239CF40023A6E400930740002E
:104DA000130700106FF0DFD39307700023A4F40003
:104DB000B70701809387F7FF23AAF4009307100039
:104DC000239CF4009307600023A6F400130710004F
:104DD0006FF01FD19307C00023A4F400B707018030
:104DE0009387F7FF23AAF40093071000239CF40095
:104DF0009307B00023A6F400130710006FF05FCEF6
:104E0000B70780009387F70F1307600023AAF40009
:104E10009307001023A4E400239CF40023A6E400DD
:104E200093076000130700106FF09FCB130101FD83
:104E300023202103232E31011389050083592500E6
:104E4000232611022324810223229102232C4101D3
:104E50009304060023267101232A510123286101AE
:104E600023248101232291012320A101930B05001A
:104E7000EFF08FE2035429009307050013050900A2
:104E8000B389F940138A4403EFF00FE13304A440DF
:104E90001387E40493070A0093872700239F07FEE4
:104EA000E39CE7FE63483409138B4B00930A4900E7
:104EB000138CAB01130D290013870A0093070B0015
:104EC00003D60700835607009387270013072700A0
:104ED000631AD60AE39687FF13868B0113078901AD
:104EE0009306000083570700835506001307E7FF6A
:104EF000B387D740B387B74093D607012311F70094
:104F000093F616001306E6FFE31EEDFC930C10006B
:104F100013050A00EFF00FBC83D7C4041304F4FF99
:104F200013050900B3E7FC002396F404EFF08FBAF1
:104F3000E35434F993060400032481028320C10260
:104F40008329C101032A8101832A4101032B010125
:104F5000832BC100032C8100832C4100032D010011
:104F600093870400130509008324410203290102E9
:104F7000130700001306000093050000130101034E
:104F80006FF05FAA930C0000E3E4C6F86FF0DFF463
:104F9000130101F72322910893040500035525010D
:104FA000378700001307F7FF2324810823202109F6
:104FB000232C410723261108232E3107232A5107CA
:104FC00023286107232671072324810723229107C1
:104FD0003375A7001389050013040600138A060021
:104FE000631EE5009389240113870400035607001C
:104FF00013072700631E0622E31A37FF0356290111
:10500000B78700009387F7FFB375F6006394F51236
:105010009306290113070900835707001307270088
:1050200063960722E39AE6FEB78700009387F7FFAF
:105030006304F5109307090003D70700938727003F
:105040006318071CE39AF6FEB7450180938505D8DF
:1050500013850400EFF05F896308052003D5240160
:1050600003562901B78700009387F7FF3378F500CF
:10507000B375F600630AF81AB78700009387F7FF45
:105080006390F514930629019307090003D70700DD
:105090009387270063160712E39AD7FE378700002D
:1050A0001307F7FF9358F50093050800938924012F
:1050B0006304E80E03570900130929006318073237
:1050C000E31AD9FE9357F600B3871741B337F000C0
:1050D0009397F7002319F4001307240193070400A2
:1050E00093872700239F07FEE39CE7FE8357240155
:1050F000378700001307F7FFB3E7E7002319F40031
:105100008320C1080324810883244108032901085E
:105110008329C107032A8107832A4107032B01073B
:10512000832BC106032C8106832C41061301010940
:10513000678000006316F5089389240193870400B3
:1051400003D7070093872700631A072AE39AF9FE1B
:10515000B7450180938505D813050900EFF0CFF816
:105160006304051003562901B78700009387F7FFF2
:10517000B375F6006380F51203D524013377F5008B
:105180006310F7049387040003D707009387270071
:105190006314072AE39AF9FE83D70400938424005A
:1051A000639A0724E39A34FF9358F5003787000089
:1051B0001307F7FFE398E5F0930629016FF09FEFDF
:1051C000138504009305C100EFF0CFE6930581023B
:1051D00013050900EFF00FE68354E1008359A102A3
:1051E000639E040A93070101930641026382D7225A
:1051F00003D7070093872700E30A07FE1305C100C2
:10520000EFF08FA90357A102B304A0406F0040093B
:1052100003D52401B78700009387F7FFB375F50026
:1052200013880500E392F5E6938924016FF09FF55A
:105230001387440183D704009384240013042400BB
:10524000231FF4FEE398E4FE6FF09FEB1307440185
:10525000835709001304240013092900231FF4FEB7
:10526000E318E4FE6FF0DFE913070401930704007D
:1052700093872700239F07FEE39CE7FEB7C7FFFF46
:105280002318F400B787FFFF93C7F7FF2319F40033
:105290006FF01FE7930629016FF0DFD9138709002C
:1052A000138909009307C1029306010463120702E0
:1052B000638AF61603D7070093872700E30A07FEE1
:1052C00013058102EFF04F9D0357A1023389A940D6
:1052D0008357810293098A03231BEA02231AFA02E5
:1052E0001307EA0493870900239007009387270098
:1052F000E31CF7FE130CCA04930B0000930A41024F
:10530000930C0101130B610403D50A00938AEAFF91
:10531000631C05088357CA0413070C00B3EBFB009A
:105320000356E7FF1307E7FF2311C700E39AE9FEDF
:10533000231C0A02E39A9AFD13074A03930781028A
:1053400013062104835607009387270013072700BD
:10535000239FD7FEE318F6FEB7C6FFFFB3842401F0
:105360009386260093850B001305810293070A009C
:1053700013070004B386D40013060000EFF08FEA91
:10538000035781028357C10093050400130581026E
:10539000B387E740B337F000B307F0402314F102BE
:1053A000EFF0CF836FF0DFD5130641049305810240
:1053B000EFE05FF913050C00930500001306C1052B
:1053C00083570500035706001305E5FF1306E6FFA4
:1053D0003307F7003307B700935507012311E500A2
:1053E00093F51500E31E66FD6FF0DFF293070000F2
:1053F0006FF09FCD930800006FF05FDBB787000070
:105400009387F7FFE388F5E803D524016FF09FD772
:105410009307440113042400231F04FEE31CF4FE3D
:105420006FF01FCE9307440113042400231F04FED2
:10543000E31CF4FE6FF0DFCC378800001308F8FFA0
:105440006FF09FC383572501130101F52324810ABF
:1054500093C7F7FF2322910A2320210B232E310922
:105460002326110A232C4109232A510923286109E3
:105470002326710923248109232291092320A109CC
:10548000232EB10713971701930405001389050014
:105490001304060093890600631E07009306250186
:1054A0009307050003D7070093872700631207308F
:1054B000E39AD7FE8357290193C7F7FF1397170184
:1054C000631E0700930629019307090003D707000D
:1054D00093872700631C072EE39AF6FE374A018064
:1054E00093050AD813850400EFF00FC0630E052E54
:1054F00003D6240183552901B78700009387F7FF5E
:105500003375F600B3F6F5006316F50A1388240127
:105510009387040003D707009387270063180708C1
:10552000E39A07FFB78700009387F7FF639AF62C8B
:10553000930629019307090003D7070093872700E3
:10554000631C0748E39AD7FE13070401930704007E
:1055500093872700239F07FEE39CE7FEB7C7FFFF63
:105560002318F400B787FFFF93C7F7FF2319F40050
:105570008320C10A0324810A8324410A0329010AE2
:105580008329C109032A8109832A4109032B0109BF
:10559000832BC108032C8108832C4108032D0108AB
:1055A000832DC1071301010B67800000B78700003E
:1055B0009387F7FF6380F626138504009305C101E6
:1055C000EFF04FA79305810313050900EFF08FA6B5
:1055D000835AA1038354E10163860A2C23265101D7
:1055E00013860400232491009307010293064103CC
:1055F000631206026384F63A03D7070093872700F5
:10560000E30A07FE1305C101EFE01FE9B387A440D9
:105610002324F10003278103938A890393870A00D7
:1056200023AAE9029384E90493872700239F07FEB6
:10563000E39C97FE13058103EFE05FC3035B210248
:1056400037090100130C0105131A0B01330A6A41D3
:10565000930CA1031309F9FF130DE106930D6105E6
:105660008357C1030357E103930B09009397070185
:10567000B387E7006368FA0033D56703931B05011E
:1056800093DB0B01130641059305C10113850B0044
:10569000EFE05FCB1307C1039307810503D6070033
:1056A0008356070093872700130727006314D62229
:1056B000E396A7FF930700009306C10613060C00AC
:1056C0000357060083D506001306E6FF3307F740AD
:1056D0003307B740935707012311E60093F71700EC
:1056E0009386E6FFE31E96FD23907A019307C1039C
:1056F00003D7270093872700239FE7FEE39A87FFBE
:1057000023180104938A2A00E39C54F51307000030
:105710009307C1031306210583D60700938727004B
:105720003367D700E39AC7FE9317070193D7074162
:1057300063840700130710009315070193D5050133
:105740001387490393078103835607009387270034
:1057500013072700239FD7FEE318F6FE8327C10017
:1057600003278100B74600009386F6FFB38AE7401F
:10577000130581039387090013070004B386DA0039
:1057800013060000EFF00FAA035781038357C101EE
:105790009305040013058103B387E740B337F00096
:1057A000B307F040231CF102EFE05FC36FF05FDC52
:1057B0001387440183D70400938424001304240036
:1057C000231FF4FEE398E4FE6FF09FDA130749010C
:1057D000835709001309290013042400231FF4FE32
:1057E000E318E9FE6FF0DFD893050AD81305090026
:1057F000EFF08F8FE31E05CE6FF01FD5E30E08DAB2
:105800009307440113042400231F04FEE31CF4FE49
:105810006FF01FD6130800009306290193070900B3
:1058200003D7070093872700E31A07FCE39AD7FE04
:10583000B78700009387F7FF630AF5041356F60055
:10584000835709001309290063900718E31AD9FE4A
:1058500093D5F5006384C500378700002319E40061
:10586000930704001307240193872700239F07FE53
:10587000E39CE7FE83572401378700001307F7FFF7
:10588000B3E7E7002319F4006FF09FCE13852401DE
:1058900083D7040093842400639C0712E39AA4FE38
:1058A0006FF0DFF99307C103130C0105630EFC0CC5
:1058B00003D7070093872700E30A07FE1305810338
:1058C000EFE09FBDB307A0400356E1012326F1009E
:1058D0006FF05FD1E3F0C6DE9387FBFF939807017B
:1058E00093D8080193060000130641031307C1066D
:1058F00083570700835506001307E7FFB387D74098
:10590000B387B74093D607012311F70093F616002B
:105910001306E6FFE31EB7FD1307C10393078105D6
:1059200003D6070083560700938727001307270035
:105930006318D600E396A7FF938B08006FF09FD7FC
:10594000E3FCC6FE1385EBFF931B050193DB0B0104
:1059500093060000130641031307C106835707008F
:10596000835506001307E7FFB387D740B387B740D7
:1059700093D607012311F70093F616001306E6FFEE
:10598000E31EB7FD6FF01FD39307440113042400F7
:10599000231F04FEE31CF4FE6FF09FBD0357C101FB
:1059A000835781036304F700378600002319C4007E
:1059B000130724019307040093872700239F07FE02
:1059C000E39CE7FE6FF01FEB930500006FF09FE88C
:1059D000130600006FF0DFE6130810006FF01FE4FD
:1059E000130101FD232481022326110213840500E3
:1059F000930741001307E10193872700239F07FEC8
:105A0000E39CE7FE0356E5009317060193D7074191
:105A100063CA0706B78700009387F7FF23120100C8
:105A20003376F600630CF6069307E5002313C100F6
:105A30001307A10083D6E7FF9387E7FF130727002B
:105A4000231FD7FEE318F5FE63120602231401009C
:105A50009305040013054100EFE05F988320C10225
:105A600003248102130101036780000093071000E3
:105A70009305F0FF130541002314F100EFE09FB9F7
:105A80006FF01FFD9307F0FF2312F100B7870000AE
:105A90009387F7FF3376F600E318F6F893070500CF
:105AA0009306E50003D7070093872700631C0706CA
:105AB000E39AF6FE13074401930704009387270037
:105AC000239F07FEE39CE7FE1307240193070400CE
:105AD00093872700239F07FEE31CF7FE83572401CB
:105AE000B78600009386F6FFB3E7D70093970701C8
:105AF00093D707012319F4008316E500E3D006F6D7
:105B00009306040003D6060093862600E31806F4E5
:105B1000E31AD7FE3787FFFFB3C7E7002319F40066
:105B20006FF0DFF313070401930704009387270046
:105B3000239F07FEE39CE7FEB7C7FFFF2318F4008F
:105B4000B787FFFF93C7F7FF2319F4006FF01FF12A
:105B500083A8C500130101E183AE050003AE450033
:105B600003A38500232E1103832505049308F0FF6A
:105B700023201117930800092324811E232C411D83
:105B80002326111E2322911E2320211F232E311D87
:105B9000232A511D2328611D2326711D2324811DC5
:105BA0002322911D2320A11D232EB11B2328D103C5
:105BB000232AC103232C6102232211172322C100AF
:105BC0002326D1002328E100232C0101130A05001C
:105BD0001384070063800502032745049307100020
:105BE000B397E70023A2E50023A4F500EF10505C73
:105BF00023200A0413090106930509001305010374
:105C0000EFF01FDE03562107378700001307F7FF69
:105C1000B375E600639EE5001307090093072107AB
:105C20008356070013072700E3960646E31AF7FE9C
:105C30001356F600032741002320C40093073000C9
:105C4000E300F714930740012324F100E31807440D
:105C500003274116B78700009387F7FF232AE10047
:105C6000639EF500930709009306210703D70700F9
:105C700093872700E3120718E39AD7FE93070009DA
:105C80002322F1161307C1079307090013064107E2
:105C900083D607009387270013072700231FD7FE0B
:105CA000E398C7FE0356E10823200100931706017D
:105CB00093D7074163CA0760374B0180130C0BD899
:105CC000930B4C01930600009307810913870B0087
:105CD000930DC10A6F008000835607009387270049
:105CE000239FD7FE13072700E398B7FF6308061426
:105CF000B78700009387F7FFE30AF6568317C108BA
:105D0000E3D8075E9305C10713850B00EFE0DFBD05
:105D100063020514E34205108357E108E39A07661E
:105D20008317C108930400009309011663C4070296
:105D300013048C111306C10793860900930506000E
:105D400013050400EFF0CFA48317C1089384F4FF78
:105D5000E3D207FE1304010D930A810E130704001A
:105D60009307C1071306010983D60700938727000D
:105D700013072700231FD7FEE398C7FE93060000F2
:105D80009307810913870B006F008000835607007B
:105D900093872700239FD7FE13072700E398B7FFB9
:105DA000930C8C02930DCC1237FDFFFF130C8C115A
:105DB0006F00C000938D4D01938C4C01930504003E
:105DC00013850B00EFE05FB2930705009305040015
:105DD00013850D006356F004EFE01FB19307050033
:105DE00093860900130604009305040013850C0034
:105DF00063C00702EFF0CF9913068109938609006B
:105E00009305060013850C00EFF08F98B384A4016E
:105E10009357FD01338DA701135D1D40E39C8CF961
:105E2000130681099386090093850B00130506006C
:105E3000EFF04FE1930C41126F0000039307C1078D
:105E40009306E10803D7070093872700E31C07EABE
:105E5000E39AF6FE93040000930C41129309011695
:105E60001304010D930A810E9305040013058109A3
:105E7000EFE05F9C130781099307040083D60700B6
:105E80009387270013072700231FD7FEE39857FFA8
:105E9000930504001305C1072318010AEFE09F9939
:105EA0009307C107035704001304240093872700B6
:105EB000239FE7FEE31854FF1305810913860900A9
:105EC0009305C107231A0108EFE05FF60355C11AD5
:105ED0006314051C930B4109130DE1071304610BB7
:105EE00093050BD81305C107EFE01FA06306051A41
:105EF0001307000093860B006F00C00113171700F3
:105F00002390F600131707019386E6FF1357070146
:105F10006384A60583D7060013960701135606412E
:105F200093971700635406001367170093970701B0
:105F300093D707011376270093E51700E30006FCCB
:105F4000131717002390B600131707019386E6FF77
:105F500013570701E390A6FD1307410B9307C107F1
:105F600083D607009387270013072700231FD7FE38
:105F7000E39877FF2316010C130700009306C10C6A
:105F80006F00C001131717002390F60013170701C5
:105F90009386E6FF135707016384860483D70600C0
:105FA0001396070113560641939717006354060092
:105FB000136717009397070193D7070113762700FC
:105FC00093E51700E30006FC131717002390B600B3
:105FD000131707019386E6FF13570701E39086FC2A
:105FE000130700009306C10C6F00C00113171700C0
:105FF0002390F600131707019386E6FF1357070156
:106000006384860483D7060013960701135606415E
:1060100093971700635406001367170093970701BF
:1060200093D707011376270093E51700E30006FCDA
:10603000131717002390B600131707019386E6FF86
:1060400013570701E39086FC1306000093860B00AC
:106050001307C10C83D50600835707009386E6FF1C
:106060001307E7FFB387B700B387C70013D607014D
:106070002391F60013761600E31E87FC13058109B1
:10608000138609009305C107EFE05FDA0355C11AD3
:106090009384F4FFE30605E483270100832641008F
:1060A00013073000B337F000B307F04093F7D70081
:1060B000938707022302F112832781006394E6008D
:1060C000B38797001307A0022320F1006354F70061
:1060D0002320E1001307A0006306E54E1305050326
:1060E0001307E002A302A1122303E11263CC071EEF
:1060F000130C711213040000130D410B930D410991
:10610000930AE107930B610B1306000093850D00C2
:106110006F00C001131616002390F5001316060138
:106120009385E5FF135606016384550583D7050063
:106130001395070113550541939717006354050004
:10614000136616009397070193D70701137526006E
:1061500093E81700E30005FC1316160023901501C1
:10616000131606019385E5FF13560601E39055FDCE
:1061700013060D009307C10783D5070093872700F7
:1061800013062600231FB6FEE398B7FF2316010C63
:10619000130600009305C10C6F00C0011316160012
:1061A0002390F500131606019385E5FF13560601AB
:1061B0006384750583D705001395070113550541C1
:1061C0009397170063540500136616009397070111
:1061D00093D707011375260093E81700E30005FC29
:1061E0001316160023901501131606019385E5FF7B
:1061F00013560601E39075FD130600009305C10CCC
:106200006F00C001131616002390F5001316060147
:106210009385E5FF135606016384750583D7050052
:106220001395070113550541939717006354050013
:10623000136616009397070193D70701137526007D
:1062400093E81700E30005FC1316160023901501D0
:10625000131606019385E5FF13560601E39075FDBD
:106260001305000093850D001306C10C83D80500AB
:10627000835706009385E5FF1306E6FFB3871701F2
:10628000B387A70013D507012391F50013751500F7
:10629000E31E76FD138609009305C10713058109E6
:1062A000EFE0DFB80356C11A0327010093071C0073
:1062B0009305060313041400A38FB7FE634A8702F5
:1062C000138C07006FF05FE413161601B707010087
:1062D000135616019387F7FF2317C1082320F100F7
:1062E0006FF09F9D0356C11A130C61129307711230
:1062F00013074000635AC70413075000E308E6027F
:1063000003C7E7FF032601009386E7FF1377F7072C
:10631000634606029307E002130680039305000319
:10632000630EF776635AE67803C7F6FF2380B6005C
:106330009386F6FF1377F7076FF09FFE130710039E
:10634000238FE7FE93841400B74501801386040071
:10635000938545D713050C00EF2090128357210732
:10636000032741012328911693C7F7FF2322E11643
:10637000139717016306071883260101034741128B
:106380009387140023A0F60093870C00630A07028A
:106390009306E0026302D72003C717009387170014
:1063A000E31A07FE9306500463E6FC006F00400109
:1063B0006388970103C7F7FF9387F7FFE31AD7FEB8
:1063C0002380070093870C00930600021306D00277
:1063D00003C707006304D7006316C700938717003D
:1063E0006FF01FFF13840C006F00C00003C707008D
:1063F000138406002300E40093061400938717001B
:10640000E31607FE83264100930720000347F4FFAD
:10641000638EF610832781009386070063D497006C
:1064200093860400930700036316F702B3079441B1
:1064300063D2F602130600036F00800063DCE600FF
:106440008347E4FFA30F04FE1304F4FF33079441D2
:10645000E386C7FE03274100930730006304F70E6D
:106460008327C10023220A04138697009307700133
:1064700063F4C710130710009307400093971700A9
:10648000938647019305070013071700E378D6FEAC
:106490002322BA0413050A00EF1000472320AA04A0
:1064A00093850C0093040500EF20101D0327810144
:1064B00063080700B3079441B387F4002320F70073
:1064C0008320C11E0324811E0329011E8329C11DAF
:1064D000032A811D832A411D032B011D832BC11C0F
:1064E000032C811C832C411C032D011C832DC11BFB
:1064F000138504008324411E1301011F67800000DF
:10650000930709009306210703D707009387270005
:10651000631A075AE39AD7FE03270101B727000041
:106520009387F7702320F7006FF0DFE993070003EC
:10653000E318F7F2B307944193061000E3CCF6EEAC
:106540006FF01FF283278100B384970063CA044E63
:10655000832701010327C10083A70700B307F700C2
:106560002326F1008327C10023220A041386370063
:1065700093077001E3E0C7F0930500006FF09FF10F
:10658000032CC100232481019307A00263D287ED6D
:106590002324F1006FF0CFEB03C70700E30407E00B
:1065A00003C7170093871700A38FE7FEE30C07DEEE
:1065B00003C7170093871700A38FE7FEE31207FEB8
:1065C0006FF05FDE13071003A302E1121307E0026E
:1065D0002303E112938414006358F02A9307000305
:1065E000A303F11283270100130C81129387F7FF95
:1065F0002320F1006FF01FB0930C4112B7450180CA
:10660000938585D713850C00B7240000EF204067E1
:106610009384F4706FF09FD4130D410B13070D009A
:106620009307C1071306010983D607009387270044
:1066300013072700231FD7FEE398C7FEB7470000C4
:106640009387E7082313F10C93070001232EF10031
:10665000B78700009387F7FF2322F102B7C7FFFF38
:10666000938727009304000013038C0C930C4112B2
:10667000930901161304010D930AA10A2324F102C0
:1066800013050300938609001306810993050D0085
:1066900023206102EFE01FDB032301021307C10483
:1066A0009307810983D607009387270013072700E4
:1066B000231FD7FEE398B7FF832741028355E105E7
:1066C00033F6F500832781023305F6006354A038C2
:1066D000130600093306A640130704009307C104FC
:1066E00083D607009387270013072700231FD7FEB1
:1066F000E39827FF6356C0069307F00013070400D2
:1067000063DEC70293060008B386A64093D6460010
:1067100013871600131717003307E40093070400CC
:1067200093872700239F07FEE31CF7FE130600084C
:106730003306A640939646003306D64093171600BC
:10674000B307FC008356070083D70723B3F7F6008F
:106750002310F7009395050193D5054163C60514F1
:10676000930781091307040003D607008356070027
:1067700093872700130727006316D602E396FAFED5
:1067800013070D009307810983D60700938727001D
:1067900013072700231FD7FEE398B7FF8327C10104
:1067A000B384F4000327C101130343019307CC1200
:1067B00013571700232EE100E314F3EC8357610C09
:1067C0000357E1081306810CB387E70037C7FFFFC3
:1067D000130727F7B387E7002313F10C1307C1074B
:1067E00093070D0083D60700938727001307270020
:1067F000231FD7FEE398C7FE130700009307810904
:106800006F00800003D70B0093872700239FE7FECC
:10681000938B2B00E398B7FF930A8C02B71D0000FF
:10682000130C8C116F00000193DD1D0063848A2717
:10683000938A4A0193050D0013050C00EFE0CF8AFF
:106840001307050093050D0013850A006344E02437
:10685000EFE08F89E34AA0FC9386090013060D0040
:1068600093050D0013850A00EFE0DFBD13068109D3
:10687000938609009305060013850A00EFE04FF1A7
:10688000B384B4016FF05FFA130C7112E39E07AA90
:106890006FF05F86130600006FF0CFB98327C10049
:1068A000138CF7FF6FF01FCE9307C104130704008A
:1068B0006F00C0009306E105E384F6EA03D6070003
:1068C000835607009387270013072700E304D6FEAB
:1068D0008357210E03274102B377F7006386E73C15
:1068E0009305C10E13850B0023206102EFD09FF4A6
:1068F0009305811013050400EFD0DFF30357C10E99
:106900000356A110035EE10E1347F7FF13170701AB
:10691000135707012316E10EB305CE4003230102EE
:1069200093060600635EB00693850C009306811003
:106930009307011203D50600938626009385250050
:10694000239FA5FEE398F6FE231E011293068110F5
:106950009305C10E6F00800003D7050093862600C3
:10696000239FE6FE93852500E398F6FE231001128F
:106970001307C10E93870C001305C11383D60700BC
:106980009387270013072700231FD7FEE398A7FE4E
:106990008356A110B305C6412312011013860600C9
:1069A000638E05322326D1029307F0F663CEF506F7
:1069B0001305C10E23206102EFD0DFC503230102BE
:1069C0008326C102930505009307011213074110A6
:1069D0000355C10E035681106306C534130E000023
:1069E0001305A11003D60700835E07009387E7FF16
:1069F0003306C6413306D641135E06012391C70014
:106A0000137E1E001307E7FFE39EA7FC130610008A
:106A100093870900130700041305811023206102E6
:106A2000EFE04F800323010293050400130581105A
:106A300023206102EFD09F9A032301026FF05FD2FF
:106A4000832701012302011213840C0023A00700F5
:106A50006FF05FB1930704001307410E938727007F
:106A6000239F07FEE39CE7FE6FF0DFCE8327010044
:106A7000930C4112638E0708B7450180938585D535
:106A800013850C00B7240000EF20801F9384F4705E
:106A90006FF0DF8C930A810E6FF00FBD83C7F6FF96
:106AA000130780036370F70E930710039384140099
:106AB000A38FF6FE6FF05F89130717002380E600AF
:106AC0006FF09F88130721076F008000E306E98AB3
:106AD0008357090013092900E38A07FE03270101F0
:106AE000B72700009387F7702320F7006FF09F8D82
:106AF000930C4112B7450180938505D713850C008F
:106B0000B7240000EF20C0179384F4706FF01F8546
:106B1000B7450180938545D613850C00B724000046
:106B2000EF2000169384F4706FF05F839305810962
:106B30001305C107232EF100EFD05F8A93050BD810
:106B400013058109EFD05FDA8327C101631A05FAC3
:106B500003270100634A07FE03C7E7FF930627FDEB
:106B600093B6160093C6F6FFB306DC0083C6060094
:106B700093F61600638A06FC9386E7FF1377F70700
:106B80006FF04FF993871700A38FF6FE6FF0CFFBDE
:106B90001304010D930504001305C107374D0000D0
:106BA000EFD05FC993040000930A810E9309C10CD2
:106BB000930C210D130DEDFF8357810E93F7770092
:106BC000639A070C1307410B9307040083D6070051
:106BD0009387270013072700231FD7FEE39857FF4B
:106BE0001305410B2316010CEFD04FE81305410BA1
:106BF000EFD0CFE7130600009386090013870A0041
:106C000083D50600835707009386E6FF1307E7FF47
:106C1000B387B700B387C70013D607012391F600E7
:106C200013761600E31E97FD8357610B0357810B04
:106C300093873700231BF10A630007021305410BFA
:106C4000EFD0CFE28357610B0357810B9387170077
:106C5000231BF10AE31407FE8357C10C639C070250
:106C60008357610B6368FD02130704009307410B10
:106C700083D607009387270013072700231FD7FE1B
:106C8000E39837FF2314010E9384F4FF930750FD1C
:106C9000E394F4F29305C10713050400EFD00FF459
:106CA000930901166FF08F8B9307040003D7070039
:106CB00093872700E31607AA1307210EE398E7FE40
:106CC0009307040003D7070093872700E31A07C040
:106CD0001307210EE398E7FE6FF09FA81307C1107A
:106CE0009307010F03DE0700035507009387270072
:106CF000130727006314AE0613056110E394A7FE83
:106D00000357C10E835781106302F70693070400EF
:106D10001307410E93872700239F07FEE39CE7FE9E
:106D20006FF01FA413050000130EE10E83DE0700B1
:106D3000035607009387E7FF1307E7FF3306D601E3
:106D40003306A600135506012391C70013751500DD
:106D5000E31EC7FD130600006FF09FCB6360C505FF
:106D600093070112130741106FF09FC69387060027
:106D7000639606000317E110635A07081307A11072
:106D8000930701128355070013072700639C050C26
:106D9000E39AE7FE2315C1106FF01FC913860C009C
:106DA00013078110930701120355070013072700EB
:106DB00013062600231FA6FEE318F7FE231E01126A
:106DC000130581101306C10E13074110035E060060
:106DD0001306260013052500231FC5FFE318E6FE52
:106DE00023100112130EC10E13860C001305C113DC
:106DF000835E060013062600130E2E00231FDEFFFF
:106E0000E318A6FE231201106FF09FBC9306011237
:106E10001305A1106F00C0012390E600939717009F
:106E2000939707019386E6FF93D70701E38EA6BEEB
:106E300003D7060013160701135606411317170050
:106E40006354060093E71700131707011357070150
:106E500013F6270093651700E30006FC2390B600A5
:106E60006FF0DFFB138616002315C1106FF0DFBB38
:106E7000032785008327C5000326050083264500D8
:106E8000130101FC13050100930541012324E100D6
:106E90002326F100232E11022320C1002322D1003A
:106EA000EFE01FB4835761021305000093C7F7FF9B
:106EB00013971701631007029307410193066102BC
:106EC00003D7070093872700631C0700E39AD7FEC8
:106ED000130520008320C103130101046780000013
:106EE000130510006FF01FFF1305050F67800000EA
:106EF000375501801305855B678000003755018099
:106F00001305855B67800000130101FF2326110034
:106F10002324810023229100630C0602B7450180DF
:106F2000938585FD1305060013040600EF10105D20
:106F3000B744018063120502138544FD8320C1001C
:106F400003248100832441001301010167800000B4
:106F5000B74401806FF05FFE938544FD1305040084
:106F6000EF10D059E30A05FCB74501809385059AD7
:106F700013050400EF109058E30005FC1305000012
:106F80006FF0DFFBB757018003C5075F6780000024
:106F9000130101FF232611002324810023229100E5
:106FA000638C050213840500B7450180938585FD38
:106FB00013050400EF109054B744018063120502DA
:106FC000138544FD8320C1000324810083244100F4
:106FD0001301010167800000B74401806FF05FFE7C
:106FE000938544FD13050400EF105051E30A05FC9E
:106FF000B74501809385059A13050400EF101050E2
:10700000E30005FC130500006FF0DFFB130101FD39
:10701000232E3101232611022324810223229102EF
:1070200023202103232C4101232A5101232861011C
:107030002326710123248101232291019387B50026
:1070400013076001930905006366F70693070001C3
:1070500063E6B71EEF00D00A930400019307800196
:10706000130620003759018013094963B307F9005B
:1070700003A44700138787FF630AE42083274400A3
:107080008326C4000326840093F7C7FFB307F400E8
:1070900003A747002326D60023A4C60013671700C2
:1070A0001385090023A2E700EF00D0051305840033
:1070B0006F00801993F487FF63C2071863E0B41868
:1070C000EF0010049307701F63F6974693D7940060
:1070D0006386071A13074000636CF73C93D764007C
:1070E000138697031385870393163600375901805B
:1070F00013094963B306D90003A44600938686FFAB
:10710000638686029305F0006F000001635C07321E
:107110000324C400638C86008327440093F7C7FFD1
:1071200033879740E3D4E5FE1306050003240901E5
:107130009308890063081417032544009306F000A0
:107140001375C5FFB307954063CCF640232A190198
:107150002328190163D6073E9307F01F63EAA72E81
:10716000937785FF9387870083254900B307F9004C
:1071700083A6070013555500130710003317A70007
:107180003367B700938587FF2326B4002324D400F8
:107190002322E90023A0870023A6860093572640D8
:1071A00093051000B395F5006368B710B3F7E500D9
:1071B00063940702939515001376C6FFB3F7E500B5
:1071C00013064600639A070093951500B3F7E50090
:1071D00013064600E38A07FE1308F0001313360077
:1071E00033036900130503008327C500130E06004F
:1071F0006302F52E03A747001384070083A7C70087
:107200001377C7FFB30697406342D82EE3C206FE4A
:107210003307E40083264700032684001385090012
:1072200093E616002322D7002326F60023A4C700E6
:10723000EF00406D130584006F0000019307C0004C
:1072400023A0F900130500008320C102032481025A
:1072500083244102032901028329C101032A8101F8
:10726000832A4101032B0101832BC100032C8100E0
:10727000832C410013010103678000009306002066
:10728000130600041305F0036FF05FE603A4C700C4
:1072900013062600E39487DE03240901930889007E
:1072A000E31C14E903274900935726409305100077
:1072B000B395F500E37CB7EE03248900832A4400EC
:1072C00013FBCAFF63689B00B3079B401307F000E2
:1072D0006346F714B7670180B76C018083AA07A7DC
:1072E00003A70CA69307F0FF330A6401B38A540185
:1072F000630AF734B71700009387F700B38AFA00E0
:10730000B7F7FFFFB3FAFA0093850A001385090067
:10731000EF10807F9307F0FF930B0500630CF528B7
:1073200063684529376C0180130CCCB583250C00AC
:10733000B385BA002320BC00938705006304AA3AF2
:1073400083A60CA61307F0FF638CE63A338A4B4101
:10735000B307FA002320FC0093FC7B0063860C300B
:10736000B7170000B38B9B4193858700938B8B00ED
:10737000B3859541B38A5B019387F7FFB385554188
:1073800033FAF50093050A0013850900EF10C07762
:107390009307F0FF6300F53C33057541B30A4501DF
:1073A00083250C002324790193EA1A00B305BA005F
:1073B0002320BC0023A25B01630824359306F00060
:1073C00063F866350327440093074BFF93F787FF65
:1073D000137717003367F7002322E40013065000E9
:1073E0003307F4002322C7002324C70063EEF636D8
:1073F00083AA4B0013840B00B767018003A7C7A6BD
:107400006374B70023A6B7A6B767018003A787A652
:107410006376B71A23A4B7A66F00401A13E71400C7
:107420002322E400B30494002324990093E7170077
:107430001385090023A2F400EF00C04C130584005B
:107440006FF09FE08326C400032684006FF01FC402
:1074500093579500130740006372F7141307400118
:10746000636AF7229386C7059385B705939636001E
:10747000B306D90083A70600938686FF6388F61CAF
:1074800003A747001377C7FF6376E50083A787004C
:10749000E398F6FE83A6C700032749002326D400FD
:1074A0002324F40023A4860023A687006FF01FCFB7
:1074B000130740016376F71213074005636AF71E4E
:1074C00093D7C4001386F7061385E7069316360094
:1074D0006FF0DFC1130E1E0093773E001305850089
:1074E000638E07108327C5006FF09FD003268400AA
:1074F00093E514002322B4002326F60023A4C7003A
:10750000B3049400232A99002328990093E71600D6
:1075100023A6140123A4140123A2F4003307E400DA
:10752000138509002320D700EF00C03D1305840018
:107530006FF09FD113D63400938784006FF09FB211
:107540003307A400832747001385090093E717003A
:107550002322F700EF00003B130584006FF0DFCE1D
:1075600013E714002322E400B3049400232A9900B3
:107570002328990013E7170023A6140123A414015C
:1075800023A2E4003305A4002320F500138509009D
:10759000EF004037130584006FF01FCB9357650051
:1075A0009386970393858703939636006FF05FEC7D
:1075B000630E241103248900832A440093FACAFF2E
:1075C000B3879A4063E69A001307F000E348F7E4B4
:1075D00013850900EF000033130500006FF0DFC6CC
:1075E0001386C7051385B705931636006FF01FB0D5
:1075F000832783001306F6FF6392671C9377360098
:10760000130383FFE39607FE0327490093C7F5FFA3
:10761000B3F7E7002322F90093951500E3EEB7C80E
:10762000E38C05C833F7F500631A0700939515003E
:1076300033F7F500130E4E00E30A07FE13060E00A3
:107640006FF0DFB9938A0A016FF01FCC0325490060
:1076500093D52540130710003317B7003367A700F1
:107660002322E9006FF09FE3B3855B01B305B040CF
:107670009395450113DA450193050A001385090026
:10768000EF1080489307F0FFE318F5D0130A0000CD
:107690006FF01FD1130740056362F7089357C500C9
:1076A0009386F7069385E706939636006FF05FDCC6
:1076B000130740156362F70893D7F4001386870712
:1076C00013857707931636006FF05FA2376C018041
:1076D000130CCCB583270C00B387FA002320FC00E1
:1076E0006FF01FC613174A01E31C07C40324890067
:1076F000B30A5B0193EA1A00232254016FF0DFCF33
:1077000023A07CA76FF05FC513840B006FF0DFCE62
:107710009307100023A2FB006FF09FEB13074015A7
:107720006362F7069357F50093868707938577077B
:10773000939636006FF0DFD3130740556362F70668
:1077400093D724011386D7071385C70793163600EE
:107750006FF0DF99938C8CFFB38A9A01B38A7A41D8
:10776000130A00006FF0DFC393058400138509003E
:10777000EFC08FFE0324890083250C00832A440078
:107780006FF09FC7130740556364F70293572501B5
:107790009386D7079385C707939636006FF05FCD22
:1077A0009306803F1306F0071305E0076FF01F9460
:1077B0009306803F9305E0076FF09FCB8327490036
:1077C0006FF09FE5B757018083A7C75A678007000E
:1077D000638005026302060463880604834706008B
:1077E00023A0F500034506003335A00067800000A4
:1077F000130101FF9305C10063040602638A0602B8
:107800008347060023A0F500034506003335A0009A
:10781000130101016780000013050000678000006C
:10782000130500006FF0DFFE1305E0FF6780000026
:107830001305E0FF6FF0DFFD9377350093F6F50F4A
:10784000638A07029307F6FF630E06021306F0FF32
:107850006F0080011305150013773500630E0700D4
:107860009387F7FF6380C70203470500E314D7FE41
:107870006780000093070600130730006366F70275
:10788000639607001305000067800000B307F5004A
:107890006F00C00013051500E386A7FE034705002F
:1078A000E31AD7FE6780000093F5F50F93988500E3
:1078B000B3E5B80093980501B3E8B8003708FFFEB8
:1078C000B78580801308F8EF93850508130330000F
:1078D0000327050033C7E800330607011347F7FF06
:1078E0003377E6003377B700E31207FA9387C7FFD1
:1078F00013054500E36EF3FCE39A07F86FF09FF879
:1079000067800000678000008327C504130101FF22
:10791000232481002322910023261100232021010A
:107920001304050093840500638E07021395240059
:10793000B387A70003A50700630605040327050016
:1079400023A0E70023280500232605008320C1008B
:107950000324810083244100032901001301010154
:10796000678000001306100293054000EF201013FB
:107970002326A40493070500E31A05FA1305000063
:107980006FF0DFFC1309100033199900130659003A
:10799000131626009305100013050400EF201010A5
:1079A000E30E05FC23229500232425016FF09FF9A7
:1079B0006380050203A745008327C504131727002A
:1079C000B387E70003A7070023A0E50023A0B700C3
:1079D00067800000130101FE232A910083A40501A2
:1079E00037030100232C81002328210123263101A4
:1079F000232E11002324410113890500930905005A
:107A00001384060013884501930800001303F3FF55
:107A1000832708001308480093881800B3F667000E
:107A2000B386C60293D70701B387C702B386860021
:107A300013DE060133F76600B386C701939706018C
:107A40003387E700232EE8FE13D40601E3C298FC37
:107A5000630204028327890063D0F40493874400FF
:107A600093972700B307F90023A28700938414009B
:107A7000232899008320C10103248101832441012B
:107A80008329C100032A810013050900032901018C
:107A90001301010267800000832549001385090056
:107AA00093851500EFF05FE6130A0500630C0504EB
:107AB000032609019305C9001305C5001306260016
:107AC00013162600EF2010110327490083A7C904CD
:107AD00013172700B387E70003A707002320E90057
:107AE00023A027019387440013090A0093972700D6
:107AF000B307F90023A28700938414002328990078
:107B00006FF05FF7B746018037450180938646FEE8
:107B1000130600009305500B130585FFEF204071FD
:107B2000130101FE232C8100232A91002328210127
:107B300023263101232441019389060093079000F5
:107B400093868600232E110023225101B3C6F6022C
:107B50001309050013840500130A060093040700A7
:107B600063D8370D93071000930500009397170013
:107B700093851500E3CCD7FE13050900EFF0DFD89D
:107B800093050500630A050A930710002328F500F2
:107B9000232A95009307900063D64709930A94001F
:107BA00093840A003304440183C604001306A00032
:107BB00013050900938606FDEFF0DFE193841400BE
:107BC00093050500E39284FE13048AFF33848A0040
:107BD00063563A03B3894941B3093401834604002B
:107BE0001306A00013050900938606FDEFF09FDE43
:107BF0001304140093050500E39289FE8320C1015C
:107C00000324810183244101032901018329C10047
:107C1000032A8100832A4100138505001301010214
:107C2000678000001304A400130A90006FF05FFA4D
:107C3000930500006FF05FF4B7460180374501807F
:107C4000938646FE130600009305E00C130585FF9E
:107C5000EF20005E3707FFFF3377E500930705004D
:107C60001305000063160700939707011305000131
:107C7000370700FF33F7E700631607001305850099
:107C800093978700370700F033F7E7006316070084
:107C90001305450093974700370700C033F7E70007
:107CA00063160700130525009397270063CA070092
:107CB00037070040B3F7E70013051500638407009A
:107CC000678000001305000267800000832705001D
:107CD0001307050093F677006384060293F61700F6
:107CE00013050000639E060493F627006388060AC6
:107CF00093D717002320F7001305100067800000BA
:107D00009396070193D6060113050000638E0606BD
:107D100093F6F70F6380060693F6F7006382060476
:107D200093F637006384060293F61700639C0600FF
:107D300093D717001305150063960700130500027B
:107D4000678000002320F7006780000093D727009A
:107D500093F6170013052500E39606FE6FF05FFD0E
:107D600093D7470093F6370013054500E39E06FAC4
:107D70006FF0DFFD93D7870093F6F70013058500BA
:107D8000E39006FA6FF0DFFD93D7070193F6F70F44
:107D900013050001E39206F86FF0DFFD93D727008B
:107DA0002320F70013052000678000008327C50407
:107DB000130101FF232481002322910023261100B7
:107DC0001304050093840500638C070203A5470094
:107DD000630205060327050023A2E7008320C100F4
:107DE0000324810093071000232A95002326050011
:107DF0002328F5008324410013010101678000005E
:107E00001306100293054000EF2040492326A404E6
:107E100093070500E31C05FAB7460180374501804A
:107E2000938646FE1306000093050014130585FF94
:107E3000EF2000401306C001930510001305040055
:107E4000EF20C045E30A05FC930710002322F5004C
:107E5000930720002324F5006FF05FF8130101FE63
:107E6000232821012326310103A9050183290601C5
:107E7000232A910023244101232E1100232C810069
:107E8000138A050093040600634C39011387090027
:107E90009384050093090900130A060013090700DB
:107EA00083A7840083A5440033842901B3A78700F6
:107EB000B385F500EFF05FA5630E051A13034501C6
:107EC00093182400B3081301930703006378130188
:107ED00023A0070093874700E3EC17FF13084A012C
:107EE000131E2900938E440193952900330EC80177
:107EF000B385BE006376C81393875401130F400007
:107F000063F0F516370601001306F6FF6F008001D7
:107F100093DF0F0163980F08130848001303430011
:107F20006370C811832F0800B3F4CF00E38204FE0E
:107F30009303030093820E001309000003A70200BD
:107F400083AF030093834300B376C700B3869602E2
:107F50009357070133F7CF0093DF0F01938242005D
:107F6000B3879702B386E600B386260113D70601CE
:107F7000B3F6C600B387F701B387E700139707018D
:107F8000B366D70023AED3FE13D90701E3E8B2FAF4
:107F9000B307E30123A02701832F080093DF0F011C
:107FA000E38C0FF6032703009302030093860E0071
:107FB000930407009303000083A7060093D90401EC
:107FC0003377C700B3F7C700B387F70383A4420032
:107FD000938242009386460033F9C400B387370189
:107FE000B38777009393070133E7E30023AEE2FE04
:107FF00003D7E6FF93D707013307F70333072701BA
:108000003307F70093530701E3E8B6FAB307E30138
:1080100023A0E7001308480013034300E364C8F1FA
:10802000634880006F0080011304F4FF63080400BC
:1080300083A7C8FF9388C8FFE38807FE8320C10198
:1080400023288500032481018324410103290101A0
:108050008329C100032A8100130101026780000007
:10806000338F9540130FBFFE137FCFFF130F4F00C9
:108070006FF05FE9B746018037450180938646FE81
:10808000130600009305D015130585FFEF20401A55
:10809000130101FE232C8100232821012326310115
:1080A000232E1100232A9100937736001304060033
:1080B0009309050013890500639E070A13542440A1
:1080C0006306040683A48904638A040C937714006E
:1080D0006390070213541440630A040403A50400C8
:1080E000630605069304050093771400E38407FEF6
:1080F000138604009305090013850900EFF01FD6CD
:10810000630609060327490083A7C90413541440D2
:1081100013172700B387E70003A707002320E90010
:1081200023A0270113090500E31A04FA8320C101E3
:1081300003248101832441018329C100130509001F
:108140000329010113010102678000001386040066
:108150009385040013850900EFF05FD023A0A400ED
:1081600023200500930405006FF01FF81309050094
:108170006FF05FF69387F7FF374701801307070516
:1081800093972700B307F70003A6070093060000A4
:10819000EFF05F84130905006FF05FF293051000A4
:1081A00013850900EFF04FF6930405006300050204
:1081B00093071027232AF500930710002328F500C2
:1081C00023A4A904232005006FF05FF0B7460180C7
:1081D00037450180938646FE130600009305001480
:1081E000130585FFEF20C004130101FE2324410184
:1081F00003AA050183A78500232631019359564020
:10820000338A4901232C8100232A9100232821014C
:1082100023225101232E110013091A009384050013
:108220001304060083A54500930A050063D82701BF
:108230009397170093851500E3CC27FF13850A0059
:10824000EFF08FEC630C0510130845016354300305
:108250009389590093992900330735019307080042
:108260009387470023AE07FEE39CE7FE9389C9FE90
:108270003308380103A60401938744011373F40102
:10828000131626003386C7006304030A9305000211
:10829000B3856540930808009306000003A7070014
:1082A0009388480093874700331767003367D700E8
:1082B00023AEE8FE03A7C7FFB356B700E3E0C7FE4F
:1082C0001387540193074000636AE600B3079640A2
:1082D0009387B7FE93F7C7FF938747003308F800EB
:1082E0002320D80063840600130A090003A7440072
:1082F00083A7CA048320C10113172700B387E700AF
:1083000003A70700232845010324810123A0E400DB
:1083100023A0970003290101832441018329C1007F
:10832000032A8100832A41001301010267800000B3
:1083300003A707009387470013084800232EE8FE91
:10834000E3F6C7FA03A7070093874700130848001E
:10835000232EE8FEE3EEC7FC6FF05FF9B74601801D
:1083600037450180938646FE130600009305901D55
:10837000130585FFEF10D06B0327050183A70501C7
:10838000130805003305F7406312F704939727009D
:1083900013084801938545013307F800B387F500BA
:1083A0006F0080006374E8028326C7FF03A6C7FF3F
:1083B0001307C7FF9387C7FFE386C6FEB3B6C600A1
:1083C0003305D0401365150067800000678000000A
:1083D00083A7050103270601130101FF2324810060
:1083E00023229100232021012326110093840500DC
:1083F000130406003389E7406394E71A93162700B5
:108400009385450113074601B387D5003307D7008D
:108410006F00800063FCF51803A6C7FF8326C7FF23
:108420009387C7FF1307C7FFE306D6FE6360D61620
:1084300083A54400EFF04FCD6302051A03AE04019B
:108440008322040193844401931E2E0013084401E7
:1084500093922200930F4501B708010023262501BE
:10846000B38ED401B3025800138F0F00138304009E
:10847000930700009388F8FF032703008325080073
:10848000130F4F00B3761701B386F600B3F715014B
:10849000B386F64093D5050193570701B387B740DC
:1084A00013D70641B387E70013970701B3F6160108
:1084B000B366D70013084800232EDFFE13034300E2
:1084C00093D70741E36A58FAB38582409385B5FE96
:1084D0001304540193D525001307000063E48200C0
:1084E000139725003387EF001308400063E68200EE
:1084F0009385150013982500B3840401B38F0F01F1
:1085000063FED405B708010013880F0093850400AB
:108510009388F8FF03A705001308480093854500DA
:10852000337617013306F600935606419357070139
:10853000B387D7009396070133761601B3E6C600DA
:10854000232ED8FE93D70741E3E6D5FD1387FEFF20
:10855000330797401377C7FF3387EF00639A06000E
:108560008327C7FF130EFEFF1307C7FFE38A07FE2B
:108570008320C100032481002328C50183244100F6
:1085800003290100130101016780000093870400A3
:108590001309100093040400138407006FF05FE9CF
:1085A000E34609FE130900006FF09FE89305000001
:1085B000EFF08FB5630205048320C100032481001E
:1085C000930710002328F500232A05008324410087
:1085D000032901001301010167800000B7460180F3
:1085E00037450180938646FE13060000930500245C
:1085F000130585FFEF10D043B74601803745018052
:10860000938646FE1306000093052023130585FF7D
:10861000EF101042B707F07FB3F5B700B707C0FC03
:10862000B385F5006358B000930700001385070079
:1086300067800000B305B04093D5454193073001F2
:1086400063C8B700B7070800B3D5B7406FF0DFFDC8
:108650001387C5FE9306E001930500009307100001
:10866000E3C6E6FCB7070080B3D7E7001385070031
:1086700067800000130101FE232A91008324050175
:10868000232C81001304450193942400B304940027
:108690002328210103A9C4FF2326310123244101FA
:1086A0001305090093890500232E1100EFF08FDADE
:1086B00013070002B307A74023A0F9009307A00007
:1086C000138AC4FF63D0A708130555FF63704405E0
:1086D00083A784FF63000504B306A74033D7D70000
:1086E0003319A9003369E900138684FF3707F03F87
:1086F0003367E900B397A7006372C40203A644FF7F
:10870000B356D600B3E7D7006F00400193070000CF
:10871000631405063707F03F3367E9008320C10182
:108720000324810183244101032901018329C1001C
:10873000032A810013850700930507001301010236
:10874000678000009306B000B386A640B707F03FED
:108750003357D9003367F70093070000637644016D
:1087600083A784FFB3D7D700130555013315A9009C
:10877000B367F5006FF09FFA3315A9003707F03F94
:108780003367E500930700006FF05FF9130101FD07
:10879000232A5101938A0500930510002320210309
:1087A000232E3101232C410123261102232481028F
:1087B0002322910213090600138A06009309070079
:1087C000EFF08F9463080510B70710009354490128
:1087D0001386F7FF93F4F47F130405003376260124
:1087E000638404003366F6002326C10063880A0808
:1087F0001305810023245101EFF04FCD0327C10061
:10880000930705006302050C03268100930600020E
:10881000B386A640B316D700B3E6C6003357A70009
:10882000232AD4002326E1003339E000130919007C
:10883000232CE40023282401638404069384D4BCFD
:10884000B384F4001305500323209A00B307F540C6
:1088500023A0F9008320C102130504000324810230
:1088600083244102032901028329C101032A8101D2
:10887000832A410113010103678000001305C10031
:10888000EFF0CFC4930710002328F4008327C10022
:1088900013091000232AF40093070502E39004FA59
:1088A000131729003307E400032507019387E7BC6A
:1088B0002320FA00EFF00FBA131959003309A94029
:1088C00023A029016FF01FF983268100232AD400F9
:1088D0006FF09FF5B746018037450180938646FECD
:1088E000130600009305A030130585FFEF10501408
:1088F000130101FD23202103138905009305810045
:10890000232611022324810223229102232E3101E6
:1089100093090500EFF01FD69304050013840500AA
:10892000130509009305C100EFF0DFD40327090107
:1089300083A709018326C100B387E740032781008D
:10894000939757003307D740B387E7001307050015
:10895000635EF00293974701338487009386050096
:10896000138504009305040013060700EF6000263A
:108970008320C102032481028324410203290102CE
:108980008329C10113010103678000009397470108
:10899000B385F5406FF09FFC130101FF23202101F7
:1089A00023261100232481002322910093077001C4
:1089B0001309050063DAA70437670180832707A43A
:1089C000832547A437670180032487A48324C7A491
:1089D000138507001306040093860400EF60D02A75
:1089E0001309F9FF93070500E31409FE8320C10072
:1089F000032481008324410003290100138507001B
:108A00001301010167800000B74701801319350089
:108A10009387070533892701832709018320C10034
:108A20000324810083254901832441000329010097
:108A300013850700130101016780000083260601EA
:108A40009385F5FF93D5554093851500930746010F
:108A50009396260093952500B386D700B305B500FD
:108A600063F8D7021307050003A8070093874700A0
:108A700013074700232E07FFE3E8D7FEB387C6405E
:108A80009387B7FE93F7C7FF938747003305F50039
:108A90006378B50013054500232E05FEE36CB5FE93
:108AA000678000000327050113D655409306450152
:108AB0006352C70293172700B387F60063F2F604E8
:108AC00003A7C7FF9387C7FFE30A07FE130510003C
:108AD0006780000093172600B387F600E350E6FE98
:108AE00093F5F501E38C05FC03A6070013051000C0
:108AF0003357B600B315B700E302B6FC6780000039
:108B00001305000067800000130101FF232481008A
:108B10002322910013040500B7640180138505002A
:108B20002326110023AA04A6EF50806D9307F0FFBF
:108B3000630CF5008320C1000324810083244100DD
:108B4000130101016780000083A744A7E38407FEA7
:108B50008320C1002320F4000324810083244100EA
:108B60001301010167800000130101FF232291001E
:108B7000B7040080232481002326110093C4F4FF4E
:108B80001304060023200600B3F6B4003706F07F76
:108B9000938705001307050063D0C606B3E8A60057
:108BA000638C080433F6C5001388050093080000A1
:108BB00063120602B767018083A647A503A607A52F
:108BC000EF60900C1307050013880500B3F6B4009E
:108BD0009308A0FC93D64641B70710809387F7FF10
:108BE000938626C03378F800B3861601B707E03FB6
:108BF000B367F8002320D4008320C1000324810040
:108C00008324410013050700938507001301010128
:108C100067800000130101F6930EC108232AF108B2
:108C200037030080B707FFFF138E05001343F3FFE0
:108C30002326D108938787209305810093860E0011
:108C4000232E1106232AF1002328E108232C0109F1
:108C5000232E11092324C101232CC101232E6100DD
:108C6000232861002322D101EF800FFC832781009C
:108C7000238007008320C1071301010A67800000D9
:108C8000130E050037650180130101F60325C5A504
:108C9000930E8108232AF10837030080B707FFFFEE
:108CA0001343F3FF2324C1082326D1089387872089
:108CB0001386050093860E0093058100232E11066E
:108CC000232AF1002328E108232C0109232E11096E
:108CD0002324C101232CC101232E6100232861001C
:108CE0002322D101EF804FF48327810023800700E6
:108CF0008320C1071301010A678000003367B500B4
:108D00009303F0FF1377370063100710B7877F7F57
:108D10009387F7F70326050083A60500B372F600D4
:108D20003363F600B382F200B3E262006392721022
:108D30006316D6080326450083A64500B372F600E5
:108D40003363F600B382F200B3E26200639E720CFA
:108D50006316D6060326850083A68500B372F60047
:108D60003363F600B382F200B3E262006398720CE0
:108D70006316D6040326C50083A6C500B372F600A9
:108D80003363F600B382F200B3E262006392720CC6
:108D90006316D6020326050183A60501B372F60009
:108DA0003363F600B382F200B3E26200639C720A9E
:108DB0001305450193854501E30ED6F4131706010B
:108DC00093970601631EF7001357060193D7060118
:108DD0003305F7409375F50F639005026780000037
:108DE0001357070193D707013305F7409375F50F24
:108DF00063940500678000001377F70F93F7F70F70
:108E00003305F740678000000346050083C6050070
:108E100013051500938515006314D600E31606FEAE
:108E20003305D64067800000130545009385450053
:108E3000E31CD6FC130500006780000013058500C5
:108E400093858500E312D6FC1305000067800000BF
:108E50001305C5009385C500E318D6FA1305000075
:108E6000678000001305050193850501E31ED6F810
:108E70001305000067800000B367B50093F7370063
:108E80006392070803A70500B7867F7F9386F6F7EE
:108E9000B377D700B387D700B3E7E700B3E7D700CE
:108EA0001306F0FF639EC706130605001308F0FFC4
:108EB0002320E60003A745009385450013064600DE
:108EC000B377D700B387D700B3E7E700B3E7D7009E
:108ED000E38007FF83C7050003C7150083C625008D
:108EE0002300F600638A0700A300E600630607007C
:108EF0002301D6006394060067800000A3010600EA
:108F0000678000009307050003C7050093871700DB
:108F100093851500A38FE7FEE31807FE6780000026
:108F2000130605006FF01FFB93773500130705004C
:108F3000639C0704B7867F7F9386F6F79305F0FF5F
:108F40000326070013074700B377D600B387D7007F
:108F5000B3E7C700B3E7D700E384B7FE8346C7FF94
:108F60000346D7FF8347E7FF3307A7406380060424
:108F7000630A06023335F0003305E5001305E5FF0B
:108F800067800000E38806FA83470700130717008D
:108F900093763700E39807FE3307A7401305F7FFE2
:108FA000678000001305D7FF678000001305C7FF27
:108FB00067800000B3E7A50093F7370013070500AB
:108FC000639807069307300063F4C7063703FFFE74
:108FD000B78880801303F3EF93880808130E3000DE
:108FE00083A60500B387660013C8F6FFB3F7070131
:108FF000B3F71701639E07022320D7001306C6FFAD
:109000001307470093854500E36CCEFC938515005C
:10901000930717006304060283C6F5FF1308F6FFE3
:10902000A38FD7FE638E0600138707001306080080
:109030009385150093071700E31006FE6780000074
:109040003306C700630A080093871700A38F07FE43
:10905000E39CC7FE678000006780000083278600CE
:10906000130101FD232A5101232611022324810229
:109070002322910223202103232E3101232C41019D
:10908000232861012326710123248101930A06000C
:1090900063880714130B05008329060003A5050048
:1090A00083A48500138405006F00400D8357C4001E
:1090B00013F70748630A0708832644018325040140
:1090C0001307190093941600B386D40093D4F601C5
:1090D000330AB540B384D40093D414403307470116
:1090E0001386040063F6E4009304070013060700E8
:1090F00093F707406386070A9305060013050B00E4
:10910000EFD0DFF0130C0500630A050A8325040184
:1091100013060A00EF10002C8357C40093F7F7B72B
:1091200093E707082316F40033054C01338A4441C2
:10913000232A940023244401232884012320A4000B
:1091400093040900130A090013060A0093850B0013
:10915000EF10003A032784000325040083A78A0048
:10916000B304974033054501232494002320A40031
:109170003389274123A42A016304090603A949006E
:1091800083AB0900138A040093898900E30809FE70
:10919000E37E99F093040900130A09006FF0DFFAE7
:1091A00013050B00EF10C046130C0500E31E05F677
:1091B0008325040113050B00EFA01FDA9307C000FD
:1091C0002320FB008357C4001305F0FF93E7070437
:1091D0002316F40023A40A0023A20A006F00C00093
:1091E00023A20A00130500008320C1020324810288
:1091F00083244102032901028329C101032A810139
:10920000832A4101032B0101832BC100032C810020
:10921000130101036780000083D7C500130101ED2E
:10922000232C411123286111232EB10F2326111263
:10923000232481122322911223202113232E311162
:10924000232A5111232671112324811123229111E4
:109250002320A11193F707082326D100138A0500C4
:10926000130B0500930D06006386070083A7050115
:10927000E3800756B7470180930AC1049387871795
:10928000374C0180B7440180232051052324010479
:109290002322010413870A0023280100232201024C
:1092A000232401022326010223240100232AF100A2
:1092B000130C4C2E9384442F83C70D00638007202A
:1092C00013840D00930650026386D7388347140039
:1092D00013041400E39A07FE3309B4416300B41F7A
:1092E00083268104832741042320B701B386260106
:1092F00093871700232227012324D1042322F1047A
:10930000930670001307870063CEF634832681002E
:1093100083470400B38626012324D1006380071A03
:1093200083461400930D1400A30D0102930CF0FF6B
:1093300013040000130D00001309A005930B900007
:109340009309A002938D1D00938706FE6364F904C0
:109350000326410193972700B387C70083A707001F
:109360006780070013040000938706FD83C60D0085
:10937000931524003384850013141400338487006C
:10938000938706FD938D1D00E3F2FBFE938706FE97
:10939000E370F9FC638406122306D108A30D0102D1
:1093A00013091000930B10009309C108930C0000DF
:1093B000137F2D0063040F0013092900137E4D084D
:1093C000832781040326410463160E00B30624415B
:1093D000E348D0028346B1031305160093058700C6
:1093E000638006049306B103938717002320D700F8
:1093F000930610002322D7002324F1042322A10482
:1094000093067000E3CCA60C930F26009306070189
:10941000130605001387050013850F0093850600CA
:10942000630C0F029306C1032320D7009387270004
:10943000930620002322D7002324F1042322A10431
:1094400013077000E34AA70C1306050013870500F5
:109450001305150093858500930600086300DE6000
:10946000B38C7C416344906BB387FB0023203701AE
:10947000232277012324F1042322A104130770007F
:109480006340A77493784D0063860800B30B2441B2
:109490006348701F635424011304090003278100EB
:1094A000330787002324E100639C077283C70D0004
:1094B0002322010413870A00E39407E08327810431
:1094C000E39C074A8357CA0093F70704E392074EC9
:1094D0008320C112032481120325810083244112B9
:1094E000032901128329C111032A8111832A411101
:1094F000032B0111832BC110032C8110832C4110ED
:10950000032D0110832DC10F13010113678000008B
:1095100013050B00232CE100EFD09F9D832745000E
:10952000138507002326F102EFF01FA09307050023
:1095300013050B002324F102EFD09F9B0327850026
:10954000832781022322E10203278101E396071684
:1095500083C60D006FF01FDF83C60D00136D0D0273
:109560006FF05FDE136D0D0193770D026382071EAE
:109570008327C1009389770093F989FF83A6490067
:1095800083AB0900938789002326F100138E060020
:1095900063C8061E9306F0FF13090D006388DC0004
:1095A000B3E6CB011379FDF76382067AE31A0E0066
:1095B00093069000E3E6760193870B03A307F10E71
:1095C000130D0900930B10009309F10E6F00C006F4
:1095D000136D0D0193770D02638607148327C10075
:1095E0009389770093F989FF83AB090003AE4900A3
:1095F000938789002326F1001379FDBF93060000AD
:10960000A30D01021306F0FF6380CC1A33E6CB01F1
:10961000137DF9F76312065E63960C3E639C067237
:10962000937B19009309010F63880B0093070003D4
:10963000A307F10E9309F10E13890C0063D47C018A
:1096400013890B008347B103B337F0003309F900E6
:109650006FF01FD63309B441E314B4C98347040043
:109660006FF0DFCB1306010493050A0013050B000E
:10967000EFF0DF9EE31805E413870A006FF01FC9BF
:10968000930600010327410463D07607930C000181
:10969000930970006F00C000938B0BFF63D67C05AD
:1096A000938707011307170023A0850123A29501C3
:1096B0002324F1042322E10493858500E3DEE9FC01
:1096C0001306010493050A0013050B00EFF01F9920
:1096D000E31A05DE938B0BFF8327810403274104E4
:1096E00093850A00E3CE7CFBB3877701130717004D
:1096F00023A0850123A275012324F1042322E10480
:1097000093067000E3D8E6D81306010493050A0017
:1097100013050B00EFF09F94E31605DA832781040D
:109720006FF05FD70326C10093770D0193064600C3
:109730006390077E93770D04E38607188327C100A3
:10974000130E00002326D10083DB07006FF0DFEA51
:109750000326C10093770D019306460063960778B0
:1097600093770D04E38007148327C1002326D100DB
:10977000839B070013DEFB4193060E00E3DC06E04B
:10978000B3367001330EC041330EDE409306D00273
:10979000A30DD1021306F0FFB30B704113090D00A6
:1097A00093061000E394CCE613061000E380C6E0B5
:1097B000130620006382C6269309010F1316DE01EB
:1097C00093F67B0093D73B0093860603B36BF600BA
:1097D000135E3E00A38FD9FE33E6CB0193850900CB
:1097E0009389F9FFE31C06FC937719006380072631
:1097F00093070003638CF6249385E5FFA38FF9FE9E
:109800009307010FB38BB740130D0900938905002F
:109810006FF09FE28327C100A30D010283A9070017
:1098200093864700E38009049307F0FF232CE100AF
:109830002326D1006382FC7813860C009305000078
:1098400013850900EFD05FFF8326C1000327810144
:10985000E30E0512B30B3541930C00006FF0DFDD12
:109860008326C100A30D01021309100083A706007F
:10987000938646002326D1002306F108930B10009F
:109880009309C1086FF09FB28327C10013692D00AF
:10989000B786FFFF83AB0700374D018093874700F2
:1098A00093C606832326F10093078DB9231ED102A8
:1098B000130E00002328F100930620006FF05FD400
:1098C0000326C10093770D02832606001306460087
:1098D0002326C1006390076093770D01639E07768E
:1098E00093770D04E394070893780D206386087638
:1098F000832781002380F6006FF01F9C83C60D0034
:10990000136D0D086FF01FA483C60D0093851D0015
:10991000E386360B938706FD938D0500930C0000BC
:10992000E3E4FBA283C60D0093952C0033839501DD
:1099300013131300B30CF300938706FD938D1D00E2
:10994000E3F2FBFE6FF05FA083C60D00136D4D00C8
:109950006FF05F9F9307B00283C60D00A30DF10265
:109960006FF05F9E8327C10083C60D0003A407002C
:10997000938747002326F100E356049C330480407C
:10998000136D4D006FF01F9C83C60D00136D1D00FD
:109990006FF05F9B8347B10383C60D00E394079A82
:1099A00093070002A30DF1026FF0DF9983C60D004B
:1099B0009307C0066384F666136D0D016FF09F98E0
:1099C00083C60D00930780066382F664136D0D0451
:1099D0006FF05F9713690D0193770902638407386D
:1099E0008327C100930610009389770093F989FFBC
:1099F0009387890083AB090003AE49002326F10059
:109A00006FF01FC013061000638AC678130620008B
:109A100013090D00E392C6DA9309010F83270101B0
:109A200093F6FB009389F9FFB386D70003C60600BF
:109A300093D74B009316CE01B3EBF600135E4E00A6
:109A40002380C900B3E6CB01E39A06FC9307010F1C
:109A5000B38B3741130D09006FF01FBEB3062441CD
:109A6000E350D0A0130E0001635EDE72130F70008E
:109A70006F00C000938606FF635EDE0493870701D4
:109A800013061600232097002322C7012324F10484
:109A90002322C10413078700E35ECFFC13060104F1
:109AA00093050A0013050B00232CD100EFF00FDB08
:109AB000E31A05A083268101130E00018327810488
:109AC000938606FF0326410413870A00130F7000D4
:109AD000E346DEFA13061600130E8700B387D7009D
:109AE000232097002322D7002324F1042322C1043A
:109AF00013077000634CC752B38C7C4113051600EA
:109B000093058E0013070E00E35090971303000196
:109B10006358935F130E70006F00C000938C0CFFAE
:109B2000635A9305938707011306160023209700B5
:109B3000232267002324F1042322C1041307870092
:109B4000E35ECEFC1306010493050A0013050B0027
:109B5000EFF0CFD0E318059613030001938C0CFFB0
:109B6000832781040326410413870A00130E700023
:109B7000E34A93FB1305160013068700B38797018A
:109B800023209700232297012324F1042322A104F8
:109B9000130770006340A720130706001305150084
:109BA000B387FB0023203701232277012324F1040C
:109BB0002322A1041307700093058600E354A78CA9
:109BC0001306010493050A0013050B00EFF00FC9FB
:109BD000E31A058E8327810493850A006FF09F8A1C
:109BE0001306010493050A0013050B00EFF00FC7DD
:109BF000E30E058A6FF01F8D13090D006FF0DFBAB9
:109C00009305000163D0D508930F00019302700003
:109C10006F00C000938606FF63D6DF0693870701B7
:109C200013061600232087012322F7012324F104C1
:109C30002322C10413078700E3DEC2FC13060104DC
:109C400093050A0013050B002320D102232EC10126
:109C5000232CE101EFF08FC0E31605868326010275
:109C6000930F000183278104938606FF0326410496
:109C7000032EC101032F810113870A009302700094
:109C8000E3CEDFF8B387D700130616002322D700F0
:109C9000232087012324F1042322C10493067000AA
:109CA0001307870063D8C6F21306010493050A0060
:109CB00013050B00232EC101232CE101EFF00FBA95
:109CC000E31205808327810403264104032EC1018A
:109CD000032F810113870A006FF0CFEF13060104F1
:109CE00093050A0013050B00232EC101232CE1016B
:109CF000EFF0CFB6631805FC0326410483278104E7
:109D0000032EC101032F81019305410513051600A0
:109D100013870A006FF0CFF01306010493050A00C1
:109D200013050B00232CC101EFF04FB3631C05F8A2
:109D30000326410483278104032E810193054105F5
:109D40001305160013870A006FF00FF1E3960C86D7
:109D5000130D0900930C0000930B00009309010FF1
:109D60006FF09F8D0326C10093770901930646008B
:109D70006396071893770904638407368327C10025
:109D8000130E00002326D10083DB0700930610008A
:109D90006FF01F871306010493050A0013050B00DB
:109DA000EFF0CFAB631005F2032541048327810454
:109DB000930541051305150013870A006FF0CFEADC
:109DC000937709402320F102130D00009309010F3E
:109DD0006F00400393050E001306A00093060000D9
:109DE00013850B00232EE100232CC101EF40805A84
:109DF000032E81010327C10163080E30930B050078
:109E0000138E050093050E001306A00093060000B4
:109E100013850B00232EE100232CC101EF40D01A43
:109E20008327010213050503A38FA9FE032E8101D9
:109E30000327C1019389F9FF130D1D00E38C07F877
:109E40008327410283C60700E396A6F99307F00F24
:109E5000E302FDF863160E0093079000E3F877BF66
:109E6000832781028325C102232EC101B389F940D2
:109E70001386070013850900232CE100EFF08F9370
:109E800003274102032EC1011306A00083451700DA
:109E90009306000013850B00B337B000B307F7003B
:109EA00093050E002322F102EF40C04E03278101EB
:109EB000130D00006FF09FF48327410283C60D004D
:109EC000638207C883C70700638E07C6136D0D4002
:109ED0006FF04FC7032681009357F64123A0C600B9
:109EE00023A2F6006FF04FBD832B06002326D1007E
:109EF00013DEFB4193060E006FF08FE92326D1009D
:109F0000832B0600130E0000930610006FF04FEF36
:109F1000832B0600130E00002326D1006FF0CFED37
:109F200013090D006FF05FABB74701809387C7BA85
:109F30002328F10093770D02638007068327C10071
:109F40009389770093F989FF83AB090003AE490039
:109F5000938789002326F10013761D00630E060007
:109F600033E6CB01630A060013060003230EC10289
:109F7000A30ED102136D2D001379FDBF93062000AF
:109F80006FF00FE8B7470180938787B92328F10066
:109F900093770D02E39407FA8325C10093770D01AF
:109FA000138645006386070483AB0500130E00008B
:109FB0002326C1006FF05FFA13850900EFE0DFF69A
:109FC00003278101930B0500930C00006FF0CFE68F
:109FD00093050004EFD08F832320AA002328AA0032
:109FE0006300052093070004232AFA006FF08FA86E
:109FF00093770D04638A07088327C100130E0000BE
:10A000002326C10083DB07006FF01FF583C61D0008
:10A01000136D0D20938D1D006FF0CFB283C61D0010
:10A02000136D0D02938D1D006FF0CFB11306010467
:10A0300093050A0013050B00EFF04F82631405C867
:10A040000326410483278104930541051305160067
:10A0500013870A006FF0CFC08327810023A0F6008A
:10A060006FF08FA593076000938B0C0063F497014A
:10A07000930B6000B74E018013890B002326D1009B
:10A0800093890EBC6FF08FB293770D206386070C17
:10A090008327C100130E00002326C10083CB0700D5
:10A0A0006FF09FEB93770D20638C07088327C10027
:10A0B0002326D100838B070013DEFB4193060E009D
:10A0C0006FF00FCD93770D20638207068327C100C1
:10A0D000130E00002326D10083CB07006FF0CFD1F1
:10A0E00093770920638807028327C100130E0000BD
:10A0F0002326D10083CB0700930610006FF04FD0CA
:10A10000138605006FF09FA793079000E3E877CFD1
:10A110006FF0DF938327C100130E00002326D100C8
:10A1200083AB0700930610006FF08FCD8327C1002B
:10A13000130E00002326D10083AB07006FF0CFCBB6
:10A140008327C1002326D10083AB070013DEFB4128
:10A1500093060E006FF0CFC38327C100130E0000DB
:10A160002326C10083AB07006FF01FDF8327810028
:10A170002390F6006FF04F941306010493050A0034
:10A1800013050B00EFE09FED6FF0CFB3938B0C0046
:10A190002326D100930C00006FF00FCA13090D00A5
:10A1A0006FF08FC1138E0500130605006FF01F932B
:10A1B0009307F0FF2324F1006FF08FB18327C100D4
:10A1C00083AC07009387470063D40C00930CF0FF27
:10A1D00083C61D002326F100938D05006FF08F9636
:10A1E0009307C0002320FB009307F0FF2324F10016
:10A1F0006FF00FAEB757018083A7875A67800700BB
:10A20000638405029307F00F63E8C7002380C5004D
:10A2100013051000678000009307A0082320F500B5
:10A220001305F0FF67800000130500006780000041
:10A23000B767018003A7C7A5130101FF9387060035
:10A2400013080600232611008328C7009306050083
:10A25000138705001386070063000802B7470180D3
:10A2600093874730B74501809385453113850800B2
:10A27000EF004011EF109067374801809307089A6C
:10A280001308089A6FF01FFE130101FF93060600E2
:10A290001306000023261100EFF09FF9B385C502D5
:10A2A000130101FF2324810023261100EFC01FD6D4
:10A2B00013040500630805020326C5FF13074002C7
:10A2C0001376C6FF1306C6FF6360C7069306300108
:10A2D0009307050063E2C60223A0070023A207003C
:10A2E00023A407008320C100130504000324810078
:10A2F00013010101678000002320050023220500CF
:10A300009307B00163F0C70423240500232605004A
:10A3100093070501E312E6FC232805009307850156
:10A32000232A05006FF05FFB93050000EF601FA478
:10A330008320C100130504000324810013010101DF
:10A3400067800000930785006FF01FF9130101FC7F
:10A350001303C1022326D10293060300232E11000A
:10A360002328E102232AF102232C0103232E1103C7
:10A3700023266100EF0010128320C10113010104A4
:10A3800067800000130E050037650180130101FC92
:10A390000325C5A5130381022324C1022326D1026C
:10A3A000138605009306030093050E00232E11006B
:10A3B0002328E102232AF102232C0103232E110377
:10A3C00023266100EF00100D8320C1011301010459
:10A3D00067800000B3C7A50093F73700B308C50036
:10A3E000639207069307300063FEC7049377350036
:10A3F000130705006398070613F6C8FF930706FEC8
:10A40000636CF708637CC702938605009307070017
:10A4100003A80600938747009386460023AE07FFF4
:10A42000E3E8C7FE9307F6FFB387E74093F7C7FF5C
:10A43000938747003307F700B385F500636817017A
:10A440006780000013070500E37C15FF83C7050044
:10A450001307170093851500A30FF7FEE36817FF96
:10A460006780000083C60500130717009377370045
:10A47000A30FD7FE93851500E38007F883C6050078
:10A480001307170093773700A30FD7FE93851500A6
:10A49000E39A07FC6FF05FF683A6450083A20500F0
:10A4A00083AF850003AFC50083AE050103AE450150
:10A4B00003A3850103A8C5012322D70083A60502B3
:10A4C000232057002324F7012326E7012328D7015F
:10A4D000232AC701232C6700232E07012320D7023C
:10A4E0001307470293854502E368F7FA6FF09FF17F
:10A4F00063F6A502B387C5006372F5023307C50092
:10A50000630A060E83C6F7FF9387F7FF1307F7FF6B
:10A510002300D700E398F5FE678000009307F00062
:10A5200063E8C702930705009306F6FF630C060C69
:10A5300093861600B386D70003C7050093871700DC
:10A5400093851500A38FE7FEE398D7FE6780000090
:10A55000B3E7A50093F737006390070A930806FF57
:10A5600093F808FF93880801330815011387050045
:10A570009307050083260700130707019387070148
:10A5800023A8D7FE832647FF23AAD7FE832687FF6B
:10A5900023ACD7FE8326C7FF23AED7FEE31CF8FC0F
:10A5A0001377C600B38515011378F600630E070410
:10A5B0001387050093880700130E3000032307005C
:10A5C00013074700B306E84023A06800B386D50010
:10A5D00093884800E364DEFE1307C8FF1377C7FFC4
:10A5E0001307470013763600B387E700B385E5000D
:10A5F0006FF09FF3678000009306F6FF9307050056
:10A600006FF01FF367800000130608006FF0DFF1A2
:10A61000130101FD2320210323261102232481029B
:10A6200023229102232E3101232C4101232A51019F
:10A6300023286101232671012324810113090600C7
:10A640006386051C1384050093090500EFD04FAB0A
:10A650009304B9009307600163FE970E93F484FF9F
:10A660001387040063CE040E63EC240F8327C4FF1A
:10A67000930A84FF13FAC7FF338B4A01635EEA1221
:10A68000B7560180938B466303A68B0083264B004D
:10A690006300661F13F6E6FF3306CB000326460071
:10A6A000137616006316061493F6C6FF3306DA0017
:10A6B0006358E60E93F7170063940702032C84FF98
:10A6C000338C8A4183274C0093F7C7FFB386D700AA
:10A6D000B38B460163DAEB34B30BFA0063D4EB2C93
:10A6E0009305090013850900EFC05F921309050067
:10A6F000630C05048327C4FF130785FF93F7E7FF67
:10A70000B387FA006386E7281306CAFF930740025F
:10A7100063E6C7301307300183260400636EC72049
:10A72000930705001307040023A0D70083264700E2
:10A7300023A2D7000327870023A4E7009305040082
:10A7400013850900EF905F8113850900EFD08F9B7F
:10A750006F00C0019304000113070001E3F824F126
:10A760009307C00023A0F900130900008320C10251
:10A7700003248102832441028329C101032A810128
:10A78000832A4101032B0101832BC100032C81008B
:10A79000130509000329010213010103678000006A
:10A7A0008327CB0003278B00130A0600338BCA00D4
:10A7B0002326F70023A4E70083A74A0033079A4023
:10A7C0009306F00093F7170063ECE606B367FA0010
:10A7D00023A2FA0083274B0093E717002322FB00F4
:10A7E00013850900EFD00F92130904006FF01FF8D2
:10A7F00093F71700E39607EE032C84FF338C8A410E
:10A8000083274C0093F7C7FF6FF01FED03248102ED
:10A810008320C10283244102032901028329C1014B
:10A82000032A8101832A4101032B0101832BC100EB
:10A83000032C810093050600130101036FC00FFD77
:10A84000B3E7970023A2FA00B3859A0013671700B5
:10A8500023A2E50083274B0093858500138509001B
:10A8600093E717002322FB00EF900FEF6FF05FF7E5
:10A8700093F6C6FF3306DA00938504016350B60EE3
:10A8800093F71700E39E07E4032C84FF338C8A417F
:10A8900083274C0093F7C7FFB386D700338B46015D
:10A8A000E34CBBE28327CC0003278C001306CAFFCE
:10A8B000930640022326F70023A4E70013098C0027
:10A8C00063ECC626930530010327040093070900B3
:10A8D00063F2C5022324EC00032744009307B00170
:10A8E0002326EC0063E2C7260327840093070C01AC
:10A8F0001304840023A0E7000327440023A2E700F9
:10A900000327840023A4E70033079C00B3079B4080
:10A9100023A4EB0093E717002322F70083274C00C2
:10A920001385090093F71700B3E4970023229C00D6
:10A93000EFC05FFD6FF09FE32320D5008326440026
:10A940001307B0012322D500636EC7168326840047
:10A9500013078400930785006FF01FDDB38A9A0008
:10A96000B307964023A45B0193E7170023A2FA00E4
:10A970008327C4FF138509001309040093F7170008
:10A98000B3E49700232E94FEEFC0DFF76FF01FDED5
:10A990008327C5FF93F7C7FF330AFA00338B4A01B9
:10A9A0006FF09FE18327CC0003278C001306CAFFBA
:10A9B000930640022326F70023A4E70013098C0026
:10A9C000330B7C0163E2C60E9305300103270400BC
:10A9D0009307090063F2C5022324EC000327440017
:10A9E0009307B0012326EC0063E0C710032784001F
:10A9F00093070C011304840023A0E70003274400FD
:10AA0000138A0B00930A0C0023A2E700032784009B
:10AA10001304090023A4E7006FF01FDA9305040074
:10AA2000EFF01FAD6FF09FD18327CB0003278B0082
:10AA30001306CAFF930640022326F70023A4E7006B
:10AA400003278C008327CC0013098C00330B7C0177
:10AA50002326F70023A4E70063E8C6049306300129
:10AA60000327040093070900E3F8C6F82324EC0049
:10AA7000032744009307B0012326EC00032784003A
:10AA8000E3F8C7F62328EC000327C400930740022D
:10AA9000232AEC00032704016304F60693078C01C4
:10AAA000130404016FF05FF593050400130509001A
:10AAB000EFF01FA413040900138A0B00930A0C0083
:10AAC0006FF09FCF032784002324E5000327C400F1
:10AAD0002326E500832604016302F604130704011C
:10AAE000930705016FF05FC4832784002328FC00CF
:10AAF0008327C400232AFC0003270401E310D6FAAD
:10AB0000232CEC000327440193070C021304840157
:10AB1000232EEC00032704006FF01FEE2328D5003E
:10AB2000832644011307840193078501232AD50056
:10AB3000832684016FF05FBF9305040013050900AD
:10AB4000EFF01F9B6FF05FDC832784002328FC005D
:10AB50008327C400232AFC00032704016308D600CE
:10AB600093078C01130404016FF0DFD8232CEC0051
:10AB70000327440193070C0213048401232EEC00E5
:10AB8000032704006FF01FD703A74506130101FD3B
:10AB9000B727000023286101232611022324810204
:10ABA0002322910223202103232E3101232C410152
:10ABB000232A51012326710123248101B3F7E700E1
:10ABC000130B06006388070A83278600832B060081
:10ABD0001389050093090500930AF0FF63880708AD
:10ABE00003AC4B0003A40B00135A2C0063060A06A7
:10ABF000930400006F00C00013044400630C9A0427
:10AC0000832504001306090013850900EF10D050B6
:10AC100093841400E31255FF1305F0FF8320C10253
:10AC20000324810223240B0023220B0083244102EE
:10AC3000032901028329C101032A8101832A4101D9
:10AC4000032B0101832BC100032C8100130101039D
:10AC50006780000083278B00137CCCFFB38787417C
:10AC60002324FB00938B8B00E39C07F61305000065
:10AC70006FF0DFFAEF1010556FF05FFA03278600D0
:10AC8000630407006FF05FF0232206001305000045
:10AC900067800000130101ED232E3111232A511189
:10ACA000232EB10F23261112232481122322911265
:10ACB00023202113232C41112328611123267111F4
:10ACC00023248111232291112320A1112326D100B5
:10ACD000930A050093890500930D0600630605009D
:10ACE000832785036380076E0397C900B72600009A
:10ACF0009317070193D7070133F6D70063180602AD
:10AD000003A64906B367D7009397070137E7FFFF0C
:10AD100093D707411307F7FF3377E6002396F9002F
:10AD20009397070123A2E90693D7070113F787003A
:10AD30006304073E03A709016300073E93F7A701D9
:10AD40001307A000638AE73EB74701809304C1045C
:10AD500093874734374C0180374901802320910481
:10AD60002324010423220104138704002328010063
:10AD700023220102232401022326010223240100AD
:10AD8000232AF100130C0C4B1309094C83C70D0047
:10AD9000638E072413840D0093065002638ED744FC
:10ADA0008347140013041400E39A07FE330AB441E6
:10ADB000630EB42383268104832741042320B70133
:10ADC000B306DA0093871700232247012324D10416
:10ADD0002322F10413067000130787006350F60264
:10ADE000E382063A130601049385090013850A00DD
:10ADF000EFF09FD96310052013870400832681009C
:10AE000083470400B38646012324D1006380071ED4
:10AE100083461400930D1400A30D0102930CF0FF60
:10AE200013040000130D0000130AA005930B9000FB
:10AE3000130BA002938D1D00938706FE6364FA0432
:10AE40000326410193972700B387C70083A7070014
:10AE50006780070013040000938706FD83C60D007A
:10AE60009315240033848500131414003384870061
:10AE7000938706FD938D1D00E3F2FBFE938706FE8C
:10AE8000E370FAFC638406162306D108A30D0102C1
:10AE9000130A1000930B1000130BC108930C000051
:10AEA000937F2D0063840F00130A2A008326410438
:10AEB000137F4D088327810413861600930506002F
:10AEC00063160F0033084441E342001B0345B103FE
:10AED00013068700630C05029306B1032320D700F5
:10AEE00093871700930610002322D7002324F10430
:10AEF0002322B10413077000E348B70E93860500C0
:10AF0000130706009385150013068600638E0F0451
:10AF10009306C1032320D7009387270093062000C0
:10AF20002322D7002324F1042322B1041307700045
:10AF3000E350B712E382072A130601049385090040
:10AF400013850A00232CE101EFF01FC46314050AE6
:10AF50008326410483278104032F810113064105C1
:10AF6000938516001387040013050008630CAF6A6D
:10AF7000B38C7C4163489079B387FB002320670141
:10AF8000232277012324F1042322B1041307700044
:10AF90006352B702638A07261306010493850900EA
:10AFA00013850A00EFF05FBE631605048327810452
:10AFB00013860400937E4D0063860E00B30B44415C
:10AFC000634070276354440113040A00032781007F
:10AFD000330787002324E1006394077E83C70D00B5
:10AFE0002322010413870400E39607DA83278104F0
:10AFF000E39E076283D7C90093F70704E3960766C9
:10B000008320C1120324811203258100832441126D
:10B01000032901128329C111032A8111832A4111B5
:10B02000032B0111832BC110032C8110832C4110A1
:10B03000032D0110832DC10F130101136780000040
:10B0400013850A00232CE100EFB09FEA8327450017
:10B05000138507002326F102EFD01FED93070500AB
:10B0600013850A002324F102EFB09FE8032785002F
:10B07000832781022322E10203278101E390072E27
:10B0800083C60D006FF01FDB83C60D00136D0D022C
:10B090006FF05FDA136D0D0193770D02638207265F
:10B0A0008327C100138B7700137B8BFF83264B0014
:10B0B000832B0B0093078B002326F10013880600D7
:10B0C00063C806269306F0FF130A0D006388DC00B0
:10B0D000B3E60B01137AFDF7E38C060AE3140812BA
:10B0E00093069000E3E0761393870B03A307F10E1A
:10B0F000130D0A00930B1000130BF10E138A0C00B2
:10B1000063D47C01138A0B008347B103B337F0008B
:10B11000330AFA006FF0DFD89385090013850A001F
:10B12000EF001066E312055483D7C9001307A0008F
:10B1300093F7A701E39AE7C08397E900E3C607C046
:10B14000032481128326C1008320C112832441126B
:10B1500003290112032A8111032B0111832BC11032
:10B16000032C8110832C4110032D011013860D0038
:10B1700093850900832DC10F8329C11113850A000E
:10B18000832A4111130101136F009053136D0D01B8
:10B1900093770D02638007148327C100138B770018
:10B1A000137B8BFF832B0B0003284B0093078B0033
:10B1B0002326F100137AFDBF93060000A30D0102C0
:10B1C0001306F0FF638ACC1833E60B01137DFAF700
:10B1D000631A066863940C3E6390067C937B1A00A6
:10B1E000130B010FE38C0BF093070003A307F10E81
:10B1F000130BF10E6FF09FF0330AB441E31CB4BBA4
:10B20000834704006FF09FC023220104937E4D000A
:10B2100063860E72B30B444163527073138604004D
:10B220001307000183264104E3587743930C000180
:10B23000130B70006F0080019385260013068600B3
:10B2400093060700938B0BFF63D87C059387070158
:10B250001387160023208601232296012324F1045C
:10B260002322E104E35AEBFC6386073A1306010448
:10B270009385090013850A00EFF01F91E31C05D6A2
:10B2800083264104938B0BFF8327810413860400DC
:10B2900093851600E3CC7CFBB387770123208601DE
:10B2A000232276012324F1042322B1041307700022
:10B2B000E35AB7D063840768130601049385090035
:10B2C00013850A00EFF05F8CE31605D28327810413
:10B2D0006FF05FCF0326C10093770D019306460000
:10B2E000E390070C93770D04E38E07228327C100B8
:10B2F000130800002326D10083DB07006FF09FEBCB
:10B300000326C10093770D0193064600E3900708DA
:10B3100093770D04E388071E8327C1002326D100FD
:10B32000839B070013D8FB4193060800E3DC06D893
:10B33000B3367001330800413308D8409306D00279
:10B34000A30DD1021306F0FFB30B7041130A0D00D9
:10B3500093061000E39ACCE613061000E380C6D8EB
:10B36000130620006386C626130B010F1316D8019F
:10B3700093F67B0093D73B0093860603B36BF600EE
:10B3800013583800A30FDBFE33E60B0193050B00C7
:10B39000130BFBFFE31C06FC93771A00638407265C
:10B3A000930700036380F6269385E5FFA30FFBFE5A
:10B3B0009307010FB38BB740130D0A00138B0500E1
:10B3C0006FF0DFD3EF10003E6FF01F928327C100B4
:10B3D000A30D010203AB070093864700E3040B10A3
:10B3E0009307F0FF232CE1002326D100E38CFC0619
:10B3F00013860C009305000013050B00EFC0CFC3AC
:10B400008326C10003278101E30C0522B30B6541AC
:10B41000930C00006FF09FCE8326C100A30D0102A4
:10B42000130A100083A70600938646002326D10046
:10B430002306F108930B1000130BC1086FF01FA631
:10B4400083C60D009307C006E380F608136D0D0157
:10B450006FF05F9E83C60D0093078006E38EF604AF
:10B46000136D0D046FF01F9D136A0D0193770A028F
:10B47000638C07528327C10093061000138B77005B
:10B48000137B8BFF93078B00832B0B0003284B0050
:10B490002326F1006FF09FD283C60D00136D0D08B7
:10B4A0006FF05F998327C100136A2D00B786FFFFF5
:10B4B00083AB0700374D01809387470093C606830F
:10B4C0002326F10093078DB9231ED1021308000033
:10B4D0002328F100930620006FF05FCE0326C10001
:10B4E00093770D0283260600130646002326C1002B
:10B4F0006394076893770D016390077E93770D043B
:10B50000E394070C937E0D2063880E7C83278100D3
:10B510002380F6006FF09F878327C10083C60D004C
:10B5200003A40700938747002326F100E354049007
:10B5300033048040136D4D006FF0DF8F83C60D0024
:10B54000136D1D006FF01F8F8347B10383C60D007D
:10B55000E392078E93070002A30DF1026FF09F8D17
:10B5600083C60D00136D4D006FF0DF8C9307B002A2
:10B5700083C60D00A30DF1026FF0DF8B83C60D00B3
:10B5800093851D00E38E660F938706FD938D05005E
:10B59000930C0000E3E2FB8A83C60D0013982C0095
:10B5A0003308980113181800B30CF800938706FDB0
:10B5B000938D1D00E3F2FBFE6FF01F881306100051
:10B5C000E380C60A13062000130A0D00E39EC6D8C6
:10B5D000130B010F8327010193F6FB00130BFBFFF5
:10B5E000B386D70003C6060093D74B009316C80155
:10B5F000B3EBF600135848002300CB00B3E60B0171
:10B60000E39A06FC9307010FB38B6741130D0A0001
:10B610006FF0DFAE93051000930600001386040060
:10B620006FF05FC233084441E354009513050001F5
:10B63000E3520505130F0001930F70006F008001A6
:10B64000138526001307870093060600130808FFDA
:10B6500063500F07938707011386160023202701E5
:10B660002322E7012324F1042322C104E3DACFFCDF
:10B6700063840716130601049385090013850A00E5
:10B68000232C0101EFF04FD0E3160596032881012A
:10B6900083264104130F0001130808FF8327810448
:10B6A0001387040013851600930F7000E3440FFB0B
:10B6B000130F8700B38707012320270123220701E7
:10B6C0002324F1042322A104130770006354A74626
:10B6D0006380076C130601049385090013850A0033
:10B6E000EFF08FCAE318059083264104B38C7C41A8
:10B6F00083278104130641059385160013870400F0
:10B70000E35C908713050001635A956713030001FA
:10B71000130F70006F0080019385260013078700C8
:10B7200093060600938C0CFF635C930593870701D7
:10B730001386160023202701232267002324F10407
:10B740002322C104E35ACFFC6384070613060104D5
:10B750009385090013850A00EFF00FC3E31C0588E9
:10B760008326410413030001938C0CFF832781047B
:10B770001387040093851600130F7000E34893FBB2
:10B7800093068700B387970123202701232297017F
:10B790002324F1042322B10413077000634CB71A69
:10B7A0009385150013868600138706006FF0CFFC83
:10B7B0009305100093060000138704006FF09FF6B6
:10B7C000130601049385090013850A00EFF0CFBB2F
:10B7D000E30605806FF01F8213051000930600003A
:10B7E000138704006FF09FE66382072013060104AD
:10B7F0009385090013850A00232EE101232CF10112
:10B80000EFF08FB8631805FE832641048327810477
:10B81000032FC101832F8101130641059385160073
:10B82000138704006FF08FEE639A072C0347B10370
:10B83000631E0756638E0F1A9307C1032326F10474
:10B84000930720002328F1041306410593051000F7
:10B8500013070600938605009385160013068700DC
:10B860006FF08FF0130A0D006FF01FAF930500010A
:10B8700063D0055F93020001930370006F00C00165
:10B88000138526001307870093060600130808FF98
:10B8900063D80207138616009387070123208701C8
:10B8A000232257002324F1042322C104E3DAC3FC3A
:10B8B000638E0706130601049385090013850A00A9
:10B8C00023200103232EE101232CF101EFF0CFAB64
:10B8D000631205F20328010283264104930200014A
:10B8E000130808FF83278104032FC101832F8101DF
:10B8F000138704001385160093037000E3CC02F94C
:10B90000B387070123208701232207012324F104A1
:10B910002322A10493067000E3C8A6F01307870052
:10B9200093051500930605006FF04FDA93060000AB
:10B9300013051000138704006FF05FF56354440192
:10B9400013040A0083278100B38787002324F100B2
:10B950006FF0CFE863840732130601049385090072
:10B9600013850A00EFF04FA2631605E88325410412
:10B97000832781041306410593851500138704006E
:10B980006FF08FDF23220104138704006FF00FC7CD
:10B99000639C0CF4130D0A00930C0000930B000041
:10B9A000130B010F6FF08FF50326C10093770A0187
:10B9B00093064600639A071893770A046380073A50
:10B9C0008327C100130800002326D10083DB070072
:10B9D000930610006FF08FFE1306410593051000CB
:10B9E00093060000138704006FF00FD863920F1CBA
:10B9F0009306000013064105930510001387040009
:10BA00006FF08FD693770A402320F102130D0000C8
:10BA1000130B010F6F004003930508001306A000ED
:10BA20009306000013850B00232EE100232C010157
:10BA3000EF205016032881010327C1016304083455
:10BA4000930B050013880500930508001306A0005A
:10BA50009306000013850B00232EE100232C010127
:10BA6000EF2090568327010213050503A30FABFEB9
:10BA7000032881010327C101130BFBFF130D1D00D8
:10BA8000E38C07F88327410283C60700E396A6F9F3
:10BA90009307F00FE302FDF8631608009307900088
:10BAA000E3F277B7832781028325C102232E0101A8
:10BAB000330BFB401386070013050B00232CE1001A
:10BAC000EFD04FCF032741020328C1011306A00086
:10BAD000834517009306000013850B00B337B000B1
:10BAE000B307F700930508002322F102EF20900A24
:10BAF00003278101130D00006FF09FF4130601046A
:10BB00009385090013850A00232EE101232CF101FE
:10BB1000EFF08F87631005CE8326410483278104CD
:10BB2000032FC101832F8101138704009385160021
:10BB30006FF0CFB99305150013068F00930605002B
:10BB400013070F006FF0CFC22326D100832B06000E
:10BB500013080000930610006FF04FE683274102A0
:10BB600083C60D00638807AC83C70700638407ACF6
:10BB7000136D0D406FF00FAC032681009357F64113
:10BB800023A0C60023A2F6006FF04FA0832B06006F
:10BB90002326D10013D8FB41930608006FF04FD243
:10BBA000832B0600130800002326D1006FF08FE0DE
:10BBB0009307C1032326F104930720002328F104EF
:10BBC00013074105930610006FF01FC9B7470180A6
:10BBD0009387C7BA2328F10093770D026384070681
:10BBE0008327C100138B7700137B8BFF832B0B0004
:10BBF00003284B0093078B002326F10013761D00CA
:10BC0000630E060033E60B01630A06001306000309
:10BC1000230EC102A30ED102136D2D00137AFDBFB6
:10BC2000930620006FF08FD9130A0D006FF01F8468
:10BC3000B7470180938787B92328F10093770D02D6
:10BC4000E39007FA8325C10093770D011386450021
:10BC50006386070483AB0500130800002326C10098
:10BC60006FF0DFF913050B00EFD00FAC0327810154
:10BC7000930B0500930C00006FF04FC813071000E2
:10BC800093870B0023266105232871052324710562
:10BC90002322E104130641056FF0CFB193770D0421
:10BCA0006380070A8327C100130800002326C10010
:10BCB00083DB07006FF09FF483C61D00136D0D201A
:10BCC000938D1D006FF00F9783C61D00136D0D023D
:10BCD000938D1D006FF00F968327810023A0F6003F
:10BCE0006FF0CF8A93076000938B0C0063EC970B87
:10BCF000B7480180138A0B002326D100138B08BCA0
:10BD00006FF0CF9993770D20638607108327C100CA
:10BD10002326D100838B070013D8FB41930608002C
:10BD20006FF00FBA93770D20638C070C8327C10047
:10BD3000130800002326D10083CB07006FF08FC7C4
:10BD400093770D206384070A8327C100130800003E
:10BD50002326C10083CB07006FF05FEA93770A20A8
:10BD6000638A07068327C100130800002326D10039
:10BD700083CB0700930610006FF04FC493060600B4
:10BD80006FF05FA093079000E3EC77CB6FF09F8795
:10BD90001306410593051000930600001387040065
:10BDA0006FF00F9D930B60006FF09FF49307B1034A
:10BDB0002326F104930710002328F10413064105FC
:10BDC000930510006FF08F93832781002390F60076
:10BDD0006FE0DFFB8327C100130800002326D1009A
:10BDE00083AB0700930610006FF04FBD8327C1009F
:10BDF000130800002326C10083AB07006FF01FE08B
:10BE00008327C100130800002326D10083AB07005D
:10BE10006FF04FBA8327C1002326D10083AB070000
:10BE200013D8FB41930608006FF08FA91306010495
:10BE30009385090013850A00EFE01FD56FF08F9BF3
:10BE4000938B0C002326D100930C00006FF00FABF6
:10BE5000130506006FF0DFAA938516006FF0CFC3BD
:10BE6000130A0D006FF04FA89307F0FF2324F10091
:10BE70006FF00F99130F0600138505006FF09F8375
:10BE80008327C10083AC07009387470063D40C006D
:10BE9000930CF0FF83C61D002326F100938D05004F
:10BEA0006FE05FF937670180930705000325C7A599
:10BEB0009306060013860500938507006FE09FDD5B
:10BEC00083D7C50003AE450603D3E50083A8C501AB
:10BED00003A84502130101B893F7D7FF13070040E9
:10BEE000232C8146231AF1001384050093070107D0
:10BEF00093058100232A914623282147232E1146AA
:10BF0000130905002326C107231B61002322110307
:10BF1000232601032324F100232CF1002328E10030
:10BF2000232EE10023200102EFE0DFD69304050079
:10BF3000635C05028357410193F707046388070098
:10BF40008357C40093E707042316F4008320C147F6
:10BF500003248147032901471385040083244147B3
:10BF60001301014867800000930581001305090053
:10BF7000EF00803FE30005FC9304F0FF6FF09FFBB0
:10BF8000B767018083A7C7A5130101FF23248100A0
:10BF90002322910023261100930405001384050039
:10BFA0006386070003A78703630407080317C40019
:10BFB000931707019376870093D7070163880608D4
:10BFC000832604016388060A13F617006308060235
:10BFD0000326440123240400130500003306C04057
:10BFE000232CC400638A06028320C100032481003D
:10BFF00083244100130101016780000013F627002C
:10C000009305000063140600832544012324B40033
:10C0100013050000E39A06FC93F70708E38607FC84
:10C02000136707042316E4001305F0FF6FF0DFFB2E
:10C0300013850700EF0000770317C400931707016B
:10C040009376870093D70701E39C06F693F60701E2
:10C050006382060893F7470063940704832604016C
:10C0600013678700931707012316E40093D707018E
:10C07000E39C06F413F6072893050020E306B6F4C4
:10C080009305040013850400EF00D0720317C40069
:10C09000832604019317070193D707016FF0DFF29E
:10C0A00083250403638E0500930704046388F50069
:10C0B00013850400EF705FEA0317C400232804020D
:10C0C000832604011377B7FD232204002320D40024
:10C0D0006FF01FF99307900023A0F4001367070483
:10C0E0002316E4001305F0FF6FF01FF0130101FFAA
:10C0F0001305600023261100EF10C03D130510004A
:10C10000EF400FB78397C500130101FE232C810078
:10C1100023263101232E1100232A910023282101F7
:10C1200093F687001384050093090500639C0610AD
:10C13000371700001307078083A64500B3E7E70021
:10C140002396F5006356D01803278402630C070C6E
:10C150009397070193D70701B716000083A409003E
:10C16000B3F6D70023A009008325C40163980616FF
:10C17000930610001306000013850900E70007006E
:10C180009307F0FF630EF5188357C400032784025A
:10C190008325C40193F74700638E0700832644007C
:10C1A000832704033305D540638607008327C40330
:10C1B0003305F540130605009306000013850900BA
:10C1C000E70007009307F0FF631EF51003A70900BF
:10C1D0008317C400630A07169306D0016306D700CD
:10C1E000930660016314D70C8326040137F7FFFF21
:10C1F0001307F77FB3F7E7002316F40023220400A8
:10C200002320D4008325040323A09900638C050018
:10C21000930704046386F50013850900EF70DFD3EC
:10C2200023280402130500008320C1010324810197
:10C2300083244101032901018329C1001301010263
:10C240006780000003A90501E30E09FC83A4050033
:10C2500013970701135707011377370023A0250110
:10C26000B3842441930700006314070083A74501AA
:10C270002324F400634890006FF0DFFA3309A9002B
:10C28000E35290FA832744028325C4019386040075
:10C290001306090013850900E7800700B384A44052
:10C2A000E34EA0FC8357C4001305F0FF93E7070497
:10C2B0008320C1012316F40003248101832441015A
:10C2C000032901018329C1001301010267800000D5
:10C2D00003A7C503E34AE0E66FF0DFF40325040596
:10C2E0006FF05FEB8357C40037F7FFFF1307F77F4B
:10C2F000B3F7E700832604019397070193D707411B
:10C3000013D7C7002316F400232204002320D400EF
:10C3100093771700E38807EE2328A4046FF09FEEBD
:10C3200083A70900E38207E61307D0016388E702C9
:10C33000130760016384E7028357C40093E707048F
:10C340002316F4006FF05FEE37F7FFFF1307F77F58
:10C3500083260401B3F7E7006FF09FFA23A099004A
:10C36000130500006FF05FEC130101FE232C810028
:10C37000232E11001304050063060500832785039F
:10C38000638007028397C500639607028320C1017B
:10C3900003248101130500001301010267800000DE
:10C3A0002326B100EF0000408325C1008397C5001C
:10C3B000E38E07FC13050400032481018320C101DF
:10C3C000130101026FF01FD463080506130101FE7B
:10C3D000B7670180232C81001304050003A5C7A5BE
:10C3E000232E11006306050083278503638A070255
:10C3F0008317C400639C07008320C10103248101CB
:10C40000130500001301010267800000930504007A
:10C41000032481018320C101130101026FF09FCE2B
:10C420002326A100EF0000388317C4000325C100B4
:10C43000E38407FC6FF09FFDB767018003A587A524
:10C44000B7C50080938585366F00902B13050000DB
:10C4500067800000B7E50080938545DA6F00502AB9
:10C460001305000067800000130101FEB7C70080BC
:10C47000232E1100232C8100232A9100232821013F
:10C48000232631012324410123225101232061016C
:10C490000324450093874745232EF5021307C52E35
:10C4A000930730002324E52E2322F52E2320052E8A
:10C4B00093074000130905002326F40013068000AB
:10C4C00093050000232204062320040023220400F5
:10C4D0002324040023280400232A0400232C04001E
:10C4E0001305C405EF409F8837EB00808324890043
:10C4F000B7EA008037EA0080B7E90080130B0B81B0
:10C50000938A4A87130ACA8F93894996B70701000D
:10C5100023206403232254032324440323263403C7
:10C52000232E84009387970023A6F400130680002F
:10C530009305000023A2040623A0040023A2040004
:10C5400023A4040023A8040023AA040023AC0400AD
:10C550001385C405EF409F810324C900B70702007B
:10C5600023A0640323A2540323A4440323A6340377
:10C5700023AE9400938727012326F4002322040688
:10C580002320040023220400232404002328040081
:10C59000232A0400232C04001305C405130680007D
:10C5A00093050000EF408FFC8320C101232064032A
:10C5B000232254032324440323263403232E8400FC
:10C5C0000324810193071000232CF90283244101E5
:10C5D000032901018329C100032A8100832A410024
:10C5E000032B01001301010267800000130101FF0A
:10C5F00023229100130680069384F5FFB384C402BE
:10C600002320210113890500232481002326110002
:10C6100093854407EFA09F9F130405006300050264
:10C620001305C50023200400232224012324A40091
:10C630001386840693050000EF404FF38320C1006A
:10C640001305040003248100832441000329010011
:10C650001301010167800000130101FEB76701802B
:10C660002328210103A987A523263101232E1100A8
:10C6700083278903232C8100232A9100232441014D
:10C6800093090500638A070A1309092E9304F0FF32
:10C69000130A400083274900032489009387F7FF8A
:10C6A00063D807006F00400813048406638E970662
:10C6B0000317C4009387F7FFE31807FEB707FFFFD0
:10C6C000938717002322040623200400232204005A
:10C6D000232404002326F40023280400232A040032
:10C6E000232C040013068000930500001305C405E5
:10C6F000EF40CFE723280402232A04022322040464
:10C70000232404048320C1011305040003248101B0
:10C7100083244101032901018329C100032A8100E7
:10C72000130101026780000003240900630C040068
:10C73000130904006FF01FF613050900EFF0DFD2B4
:10C740006FF09FF49305C01A13850900EFA01F8CAA
:10C7500013040500630605021305C5002320040029
:10C76000232244012324A4001306001A9305000089
:10C77000EF40CFDF23208900130904006FF09FF101
:10C78000232009009307C00023A0F9006FF09FF752
:10C79000B767018003A587A5B7E50080938545DAD3
:10C7A0006F0000768327850363840700678000009D
:10C7B0006FF09FCB678000006780000067800000FB
:10C7C00067800000B767018003A5C7A5B7C50080D3
:10C7D0009385C5446F008068B767018003A5C7A52E
:10C7E000B7C50080938505466F004067130101FDC2
:10C7F00023248102232E31012328610123261102E3
:10C800002322910223202103232C4101232A5101B9
:10C81000130B05009389050013040600EFA08FF6A3
:10C82000930710006310F5029387F9FF1307E00FD9
:10C83000636AF70013F7F90F2306E10013091000EC
:10C840006F00C0029306C405138609009305C1005A
:10C8500013050B00EF10802B9307F0FF1309050061
:10C860006304F50A630E05080347C1009304000042
:10C87000130AF0FF930AA0006F00800283270400D0
:10C88000938617002320D4002380E70093841400AC
:10C890009307C100B387970063F4240703C7070019
:10C8A000832784009387F7FF2324F400E3D807FC51
:10C8B00083268401930507001306040013050B006B
:10C8C00063C4D700E31C57FBEF10400AE31045FD9B
:10C8D0001309F0FF8320C102032481028324410253
:10C8E0008329C101032A8101832A4101032B01010C
:10C8F00013050900032901021301010367800000E9
:10C90000138909006FF01FFD8357C40093E70704E4
:10C910002316F4006FF01FFC8317C600139727013E
:10C920006340070203274606B7260000B3E7D70097
:10C93000B72600003367D7002316F6002322E60649
:10C940006FF0DFEA130101FEB7670180232C81003D
:10C9500003A4C7A5232E1100138605009305050027
:10C960006306040083278403638007048317C600DB
:10C97000139727016340070203274606B7260000E6
:10C98000B3E7D700B72600003367D7002316F600B9
:10C990002322E60613050400032481018320C1013C
:10C9A000130101026FF09FE42324A100130504008A
:10C9B0002326C100EFF01FDF0326C100832581007D
:10C9C0006FF0DFFA832786006388073083D7C500BE
:10C9D000130101FD23248102232C4101232A51014B
:10C9E000232611022322910223202103232E310129
:10C9F000232861012326710123248101232291012F
:10CA00002320A10113F78700130A0600930A0500EB
:10CA1000138405006306070803A7050163020708DE
:10CA200013F7270083240A00630C070883274402B6
:10CA30008325C401370B008093090000130900000F
:10CA4000134B0BC01386090013850A006302090407
:10CA50009306090063742B0193060B00E78007001F
:10CA60006352A02683278A00B389A9003309A9400D
:10CA70003385A7402324AA006300052083274402AE
:10CA80008325C4011386090013850A00E31209FCFB
:10CA900083A9040003A94400938484006FF09FFAE3
:10CAA0009305040013850A00EFF08FCD6314053A57
:10CAB0008357C40083240A0013F72700E31807F6FE
:10CAC00013F7170063160712832C84000325040054
:10CAD000370B0080934BEBFF130C00001309000091
:10CAE000134BFBFF630E090E13F70720630807249F
:10CAF000138D0C00636E992D13F70748630A07081E
:10CB00008329440183250401130719009396190012
:10CB1000B386360193D9F601330DB540B389D900F8
:10CB200093D919403307A7011386090063F6E9007A
:10CB3000930907001306070093F707406386072C45
:10CB40009305060013850A00EFA04FCC930C050057
:10CB5000630A052E8325040113060D00EFD09F877D
:10CB60008357C40093F7F7B793E707082316F40039
:10CB70003385AC01B387A941232894012320A40065
:10CB8000232A3401930C09002324F400130D090017
:10CB900013060D0093050C00EFD09F95032784002A
:10CBA0008327040093090900B30C9741B387A701B9
:10CBB000232494012320F4001309000003268A0093
:10CBC000330C3C01B309364123243A016386090A38
:10CBD000832C8400032504008357C400E31609F066
:10CBE00003AC040003A94400938484006FF09FEF1A
:10CBF000130B000013050000130C00009309000044
:10CC00006380090E6306050E93070B00938B0900E2
:10CC100063F43701938B0700032504008327040185
:10CC20008326440163F8A700032984003389260181
:10CC30006340790F63C4DB1A832744028325C40150
:10CC400013060C0013850A00E7800700130905008E
:10CC5000635AA006330B2B4113051000630C0B0421
:10CC600003268A00330C2C01B3892941330926415C
:10CC700023242A01E31609F8130500008320C102CA
:10CC80000324810283244102032901028329C10173
:10CC9000032A8101832A4101032B0101832BC10057
:10CCA000032C8100832C4100032D0100130101039B
:10CCB000678000009305040013850A00EFF0CFEAB7
:10CCC000E30005FA8317C40093E707042316F40072
:10CCD0001305F0FF6FF09FFA130500006780000056
:10CCE00083A9440003AC040093848400E38A09FE12
:10CCF000138609009305A00013050C00EFA0DFB315
:10CD0000630C051213051500330B85416FF0DFEF3F
:10CD100093050C0013060900EFD08FFD8327040054
:10CD20009305040013850A00B38727012320F4002C
:10CD3000EFF08FE3E30005F26FF0DFF883270401E3
:10CD400063E2A70483274401636EF9029306090096
:10CD500063F42B0193060B00B3C6F60203274402CB
:10CD60008325C40113060C0013850A00B386F6025E
:10CD7000E700070093090500E356A0F433093941A1
:10CD80006FF0DFE393890C00637499019309090044
:10CD90001386090093050C00EFD08FF583278400DC
:10CDA00003270400B3873741330737012324F400F6
:10CDB0002320E400E39407FC9305040013850A0094
:10CDC000EFF08FDAE31005F0330939416FF01FDF20
:10CDD000930C0900130D09006FF09FDB13860B0005
:10CDE00093050C00EFD0CFF00327840083270400C5
:10CDF00013890B0033077741B38777012324E400BD
:10CE00002320F4006FF01FE513850A00EFD05F8048
:10CE1000930C0500E31E05D48325040113850A0045
:10CE2000EF708F938317C4001307C00023A0EA009C
:10CE300093F7F7F76FF05FE993871900138B0700FB
:10CE40006FF0DFDC1307C0008317C40023A0EA00E3
:10CE50006FF09FE71305F0FF6FF05FE2130101FE33
:10CE600023282101232631012324410123225101BA
:10CE700023206101232E1100232C8100232A9100FD
:10CE8000138B0500930A052E130A00009309100066
:10CE90001309F0FF83A44A0003A48A009384F4FFDB
:10CEA00063C604028357C4009384F4FF63FCF90053
:10CEB0008317E4001305040063862701E7000B00D5
:10CEC000336AAA0013048406E39E24FD83AA0A00A1
:10CED000E3920AFC8320C1010324810183244101E0
:10CEE000032901018329C100832A4100032B01008A
:10CEF00013050A00032A8100130101026780000064
:10CF0000130101FD23202103232E3101232C410194
:10CF1000232A5101232861012326710123261102AE
:10CF20002324810223229102930A0500938B05009A
:10CF3000130B052E130A0000930910001309F0FFCC
:10CF400083244B0003248B009384F4FF63C8040202
:10CF50008357C4009384F4FF63FEF9008317E40051
:10CF60009305040013850A0063862701E7800B0000
:10CF7000336AAA0013048406E39C24FD032B0B00F0
:10CF8000E3100BFC8320C1020324810283244102AD
:10CF9000032901028329C101832A4101032B0101D5
:10CFA000832BC10013050A00032A81011301010329
:10CFB0006780000083D7C500130101F8232C810688
:10CFC000232E1106232A9106232821072326310721
:10CFD0002324410713F7270013840500630C07027D
:10CFE0009387350423A0F50023A8F50093071000CC
:10CFF00023AAF5008320C107032481078324410766
:10D00000032901078329C106032A810613010108A8
:10D01000678000008395E5009304050063CC050854
:10D0200013068100EF009066634405088327C10062
:10D0300037F90000130A00403379F900B7E7FFFF22
:10D040003309F900B71700001339190093890780D5
:10D0500093050A0013850400EF905FFB8317C4005B
:10D06000630E050637C700801307474523AEE40269
:10D0700093E707082316F4002320A4002328A40024
:10D08000232A440163180908B3E737018320C10745
:10D090002316F40003248107832441070329010791
:10D0A0008329C106032A8106130101086780000055
:10D0B0008357C40093F70708130900006386070429
:10D0C000130A000493050A0013850400EF901FF46F
:10D0D0008317C40093090000E31605F813F707202F
:10D0E000E31A07F093F7C7FF93E727001307340409
:10D0F0002316F400930710002320E4002328E40003
:10D10000232AF4006FF01FEF130A00409309000078
:10D110006FF01FF48315E40013850400EF00905DA9
:10D12000631605008317C4006FF01FF68357C40011
:10D1300093F7C7FF93E717009397070193D707412A
:10D140006FF09FF4130101F9232481061384050075
:10D150008395E5002322910623202107232611062B
:10D16000930406001389060063CA050413068100B0
:10D17000EF00D051634405040327C100B7F7000056
:10D180008320C106B3F7E70037E7FFFFB387E70067
:10D190000324810693B717002320F900930700406A
:10D1A00023A0F4003715000083244106032901065B
:10D1B0001305058013010107678000008317C40071
:10D1C0002320090093F70708638407028320C10620
:10D1D000032481069307000423A0F4000329010619
:10D1E0008324410613050000130101076780000036
:10D1F0008320C106032481069307004023A0F40086
:10D2000003290106832441061305000013010107C9
:10D21000678000008327C52D638607001305000083
:10D2200067800000130101FF93050008232481009B
:10D230002326110013040500EF905FDD232EA42C9C
:10D240006304050293070508232005001305450024
:10D25000E31CF5FE130500008320C10003248100B8
:10D2600013010101678000001305F0FF6FF0DFFE7E
:10D27000130101FE232A9100232E1100232C81008B
:10D280009307F0019304050063EAB7020327C52D55
:10D290001384050063040704131424003304870077
:10D2A000032504002320C4008320C101032481013D
:10D2B0008324410113010102678000008320C10122
:10D2C00003248101930760012320F5008324410199
:10D2D0001305F0FF130101026780000093050008A9
:10D2E0002326C100EF909FD223AEA42C1307050084
:10D2F000630005020326C100930705009306050895
:10D3000023A0070093874700E39CD7FE6FF0DFF868
:10D310001305F0FF6FF05FF9130101FF2322910065
:10D3200023261100232481009307F00193040500B4
:10D3300063EAB70A8327C52D1384050063840704B5
:10D3400013972500B387E70003A70700630C0702C4
:10D3500093061000630CD7069306F0FF6308D7040A
:10D360001385050023A00700E70007001305000050
:10D370008320C100032481008324410013010101A3
:10D380006780000013850400EF0040481306040086
:10D39000032481008320C100930505001385040048
:10D3A00083244100130101016F00C03F8320C100AD
:10D3B00003248100930760012320F50083244100AA
:10D3C0001305100013010101678000008320C100D4
:10D3D000032481008324410013050000130101018F
:10D3E00067800000930760012320F5001305F0FF1C
:10D3F0006FF01FF89307F00163EAB70C0327C52D00
:10D40000130101FF23248100232291002326110010
:10D410001384050093040500630007061315240018
:10D420003307A70083270700638C07029306F0FFEA
:10D430006386D708930610006386D7061305040099
:10D4400023200700E7800700130500008320C100A8
:10D45000032481008324410013010101678000003F
:10D460008320C100032481008324410013051000A0
:10D47000130101016780000093050008EF901FB9B8
:10D4800023AEA42C13070500630E050293070500C5
:10D490009306050823A0070093874700E39CD7FE67
:10D4A0006FF0DFF78320C100032481008324410053
:10D4B00013053000130101016780000013052000EF
:10D4C0006FF0DFF81305F0FF6FF05FF81305F0FF62
:10D4D00067800000130101FF23229100376701805C
:10D4E00023261100232481009307F0018324C7A57C
:10D4F00063E8A70A83A7C42D130405006382070409
:10D5000013172500B387E70003A70700630A070284
:10D5100093061000630AD7069306F0FF6306D7044C
:10D5200023A00700E7000700130500008320C100C7
:10D53000032481008324410013010101678000005E
:10D5400013850400EF00802C1306040003248100DF
:10D550008320C10093050500138504008324410046
:10D56000130101016F0000248320C1000324810006
:10D570009307600123A0F4001305100083244100E9
:10D5800013010101678000008320C1000324810092
:10D59000832441001305000013010101678000008E
:10D5A0009307600123A0F4001305F0FF6FF01FF84C
:10D5B000130101FF23202101376701802326110079
:10D5C00023248100232291009307F0010329C7A59A
:10D5D00063EEA702130405000325C92D93840500FB
:10D5E0006308050413142400330485000325040094
:10D5F000232094008320C100032481008324410060
:10D600000329010013010101678000008320C1008C
:10D6100003248100930760012320F9008324410043
:10D62000032901001305F0FF1301010167800000C9
:10D630009305000813050900EF905F9D232EA92C88
:10D64000630E0500930705001307050823A00700D4
:10D6500093874700E31CF7FE6FF0DFF81305F0FF38
:10D660006FF05FF9130101FFB76701802324810088
:10D6700003A4C7A5232611008327C42D638C0700AC
:10D68000130500008320C100032481001301010160
:10D69000678000009305000813050400EF901F97B2
:10D6A000232EA42C630C05009307050823200500F6
:10D6B00013054500E31CF5FE6FF09FFC1305F0FF1A
:10D6C0006FF05FFC130101FF232291003767018097
:10D6D00023261100232481009307F0018324C7A58A
:10D6E00063EEA70A03A7C42D130405006300070611
:10D6F000131524003307A70083270700638C070254
:10D700009306F0FF6388D708930610006388D70656
:10D710001305040023200700E7800700130500001D
:10D720008320C100032481008324410013010101EF
:10D73000678000008320C10003248100832441000E
:10D740001305100013010101678000009305000814
:10D7500013850400EF909F8B23AEA42C13070500C4
:10D76000630E0502930705009306050823A0070032
:10D7700093874700E39CD7FE6FF09FF78320C1009B
:10D7800003248100832441001305300013010101AB
:10D7900067800000130520006FF09FF81305F0FF6D
:10D7A0006FF01FF8130101FF138705002324810088
:10D7B0002322910013040500B7640180930506003D
:10D7C000130507002326110023AA04A6EF00101753
:10D7D0009307F0FF630CF5008320C1000324810050
:10D7E00083244100130101016780000083A744A73F
:10D7F000E38407FE8320C1002320F400032481007A
:10D800008324410013010101678000006F00900E26
:10D81000130101FF23248100138405008395E50093
:10D8200023261100EF00C079634005028327040519
:10D830008320C100B387A7002328F40403248100B8
:10D8400013010101678000008357C40037F7FFFF11
:10D850001307F7FFB3F7E7008320C1002316F40096
:10D8600003248100130101016780000013050000FB
:10D87000678000008397C500130101FE232C8100FF
:10D88000232A91002328210123263101232E110070
:10D8900013F7071013840500930405008395E50032
:10D8A0001309060093890600631E070237F7FFFF7E
:10D8B0001307F7FFB3F7E7002316F40003248101F1
:10D8C0008320C10193860900130609008329C10042
:10D8D000032901011385040083244101130101027E
:10D8E0006F0080339306200013060000EF0080666F
:10D8F0008317C4008315E4006FF05FFB130101FF81
:10D9000023248100138405008395E500232611005C
:10D91000EF0040649307F0FF6304F5028357C400EF
:10D92000371700008320C100B3E7E7002328A404D1
:10D930002316F40003248100130101016780000015
:10D940008357C40037F7FFFF1307F7FFB3F7E7006C
:10D950008320C1002316F400032481001301010178
:10D96000678000008395E5006F00C031130101FE60
:10D97000232C8100232A910023282101232E11002A
:10D9800023263101130905009384050013040600C2
:10D990006306050083278503638A07140317C40001
:10D9A00083268401937787002324D40093160701EC
:10D9B00093D6060163840708832704016380070860
:10D9C00037260000B3F6C60093F9F40F93F4F40F72
:10D9D0006380060A0327040083264401B307F74047
:10D9E00063DED70A83268400130617002320C400B1
:10D9F0009386F6FF2324D400230037010327440134
:10DA0000938717006308F70C8357C40093F7170038
:10DA1000638607009307A000638EF40A8320C10188
:10DA200003248101032901018329C1001385040016
:10DA30008324410113010102678000009305040063
:10DA400013050900EFE0CFD3631E05080317C400D8
:10DA50003726000093F9F40F9316070193D60601B9
:10DA6000B3F6C6008327040193F4F40FE39406F69B
:10DA7000832644063367C70037E6FFFF1306F6FF29
:10DA8000B3F6C6002316E400032704002322D406BD
:10DA900083264401B307F740E3C6D7F49305040097
:10DAA00013050900EFE05F8C631E050203270400E5
:10DAB0008326840093071000130617009386F6FF51
:10DAC0002320C4002324D40023003701032744016A
:10DAD000E31CF7F29305040013050900EFE0DF886B
:10DAE000E30E05F29304F0FF6FF05FF3EFE09FCBDE
:10DAF0006FF0DFEA37670180930705000325C7A5AC
:10DB000013860500938507006FF05FE6130101FEA1
:10DB1000232C8100232A9100B7570180232E110066
:10DB200083A7875A130405009384060063820502C5
:10DB3000E78007009307F0FF6306F5028320C10129
:10DB40000324810183244101130101026780000045
:10DB50001306000093054100E78007009307F0FFDC
:10DB6000E31EF5FC23A004009307A0088320C10155
:10DB70002320F400032481018324410113010102C5
:10DB800067800000130101FEB7670180232C81002C
:10DB9000232A9100232E110083A4C7A5B757018023
:10DBA00083A7875A13040600630A0502138605003B
:10DBB000930604009305050013850400E780070021
:10DBC0009307F0FF630AF5028320C101032481015A
:10DBD00083244101130101026780000093060600BF
:10DBE000930541001306000013850400E780070039
:10DBF0009307F0FFE31AF5FC232004008320C10102
:10DC0000032481019307A00823A0F4008324410189
:10DC10001301010267800000130101FF1387050053
:10DC2000232481002322910093050600130405009C
:10DC3000B764018013860600130507002326110030
:10DC400023AA04A6EF00C0659307F0FF630CF5005C
:10DC50008320C100032481008324410013010101BA
:10DC60006780000083A744A7E38407FE8320C100E8
:10DC70002320F400032481008324410013010101C7
:10DC800067800000130101FF2324810023229100FB
:10DC900013040500B76401801385050023261100D5
:10DCA00023AA04A6EF0080389307F0FF630CF50069
:10DCB0008320C1000324810083244100130101015A
:10DCC0006780000083A744A7E38407FE8320C10088
:10DCD0002320F40003248100832441001301010167
:10DCE00067800000130101FF23248100232291009B
:10DCF000232021011384050023261100930405002D
:10DD0000EFE04FC08327C40213090500638A0700B0
:10DD10008325C40113850400E780070063440506DA
:10DD20008357C40093F70708639607068325040307
:10DD3000638C0500930704046386F50013850400D3
:10DD4000EF608FA123280402832544046388050023
:10DD500013850400EF604FA023220404EFE09FA589
:10DD600023160400EFE05FA58320C1000324810097
:10DD70008324410013050900032901001301010157
:10DD8000678000008357C4001309F0FF93F707086A
:10DD9000E38E07F88325040113850400EF60CF9B11
:10DDA0006FF0DFF863840506130101FE232C810068
:10DDB000232E110013040500630605008327850345
:10DDC000638A07028397C500639C07008320C10113
:10DDD0000324810113050000130101026780000084
:10DDE00013050400032481018320C10113010102F2
:10DDF0006FF05FEF2326B100EFE0DF9A8325C100CB
:10DE00008397C500E38407FC6FF09FFD13050000B6
:10DE10006780000063080506130101FEB7670180F3
:10DE2000232C81001304050003A5C7A5232E110090
:10DE30006306050083278503638A07028317C400EE
:10DE4000639C07008320C1010324810113050000A6
:10DE5000130101026780000093050400032481017F
:10DE60008320C101130101026FF0DFE72326A10027
:10DE7000EFE05F938317C4000325C100E38407FC30
:10DE80006FF09FFD1305000067800000130101FF84
:10DE90001387050023248100232291001304050029
:10DEA000B7640180930506001305070023261100BF
:10DEB00023AA04A6EF00001D9307F0FF630CF500F2
:10DEC0008320C10003248100832441001301010148
:10DED0006780000083A744A7E38407FE8320C10076
:10DEE0002320F40003248100832441001301010155
:10DEF00067800000130101FF232481002322910089
:10DF000013040500B7640180138505002326110062
:10DF100023AA04A6EF00801E9307F0FF630CF50010
:10DF20008320C100032481008324410013010101E7
:10DF30006780000083A744A7E38407FE8320C10015
:10DF40002320F400032481008324410013010101F4
:10DF500067800000130101FF13870500232481005F
:10DF6000232291009305060013040500B764018085
:10DF700013860600130507002326110023AA04A612
:10DF8000EF00001E9307F0FF630CF5008320C10033
:10DF900003248100832441001301010167800000F4
:10DFA00083A744A7E38407FE8320C1002320F40055
:10DFB00003248100832441001301010167800000D4
:10DFC000130101FF13870500232481002322910000
:10DFD0009305060013040500B7640180138606004C
:10DFE000130507002326110023AA04A6EF00401CF6
:10DFF0009307F0FF630CF5008320C1000324810028
:10E0000083244100130101016780000083A744A716
:10E01000E38407FE8320C1002320F4000324810051
:10E02000832441001301010167800000130101FFF7
:10E03000232611002324810093050000130600000D
:10E040009306000013070000930700009308900355
:10E050007300000013040500634C05008320C10019
:10E0600013050400032481001301010167800000EF
:10E0700033048040EF308FBA232085001304F0FF73
:10E080006FF0DFFD130101F7232291082326110809
:10E0900093840500232481089305010013060000E2
:10E0A0009306000013070000930700009308000583
:10E0B0007300000013040500634405021385040087
:10E0C00093050100EF00C0228320C108130504005E
:10E0D000032481088324410813010109678000009B
:10E0E00033048040EF308FB3232085001304F0FF0A
:10E0F0006FF0DFFC1305100067800000130101F9C9
:10E100009305810023261106EFF0DFF79307F0FF58
:10E11000630EF5000325C1008320C1061355D50009
:10E120001375150013010107678000008320C106E5
:10E13000130500001301010767800000130101FFB0
:10E1400023261100EF308FAD8320C10093076001BB
:10E150002320F5001305F0FF130101016780000083
:10E16000130101FF232611002324810093060000E0
:10E1700013070000930700009308E00373000000FA
:10E1800013040500634C05008320C100130504003F
:10E1900003248100130101016780000033048040E3
:10E1A000EF30CFA7232085001304F0FF6FF0DFFDD1
:10E1B000130101FF23261100232481009306000090
:10E1C00013070000930700009308F003730000009A
:10E1D00013040500634C05008320C10013050400EF
:10E1E0000324810013010101678000003304804093
:10E1F000EF30CFA2232085001304F0FF6FF0DFFD86
:10E2000037630180832783A7130101FF23261100B1
:10E21000130805006398070213050000930500002A
:10E220001306000093060000130700009308600D1A
:10E23000730000001307F0FF930705006304E50473
:10E24000232CA3A63305F800930500001306000055
:10E250009306000013070000930700009308600D69
:10E2600073000000832783A73308F800631C0501AF
:10E270008320C100232CA3A61385070013010101ED
:10E2800067800000EF308F998320C1009307C000A2
:10E290002320F5001305F0FF130101016780000042
:10E2A000130101FF2326110023248100930600009F
:10E2B0001307000093070000930800047300000098
:10E2C00013040500634C05008320C10013050400FE
:10E2D00003248100130101016780000033048040A2
:10E2E000EF30CF93232085001304F0FF6FF0DFFDA4
:10E2F000130101FF83A3450183A2850183AFC501FB
:10E3000003AF050283AE050303AE050403A3850333
:10E3100003A8850483A8C50403A6850523268100D8
:10E320002324910003A4050183A485002322210155
:10E3300003A9050083A6C50503A7850683A7C5060F
:10E340002310250123119500232285002314750035
:10E35000231555002316F5012317E5012328D501C0
:10E360002326C50523246504232C0501232E15012E
:10E370002324C5022326D5020324C100232CE50251
:10E38000232EF5028324810003294100130101019A
:10E3900067800000930805009387050013080600B6
:10E3A000138506001383080063940628B74601808E
:10E3B0009386465863F6C50E370701006378E60C6E
:10E3C0001307F00F3337C700131737003355E60034
:10E3D000B386A60083C60600130500023387E60055
:10E3E000B306E540630CE500B395D70033D7E800EA
:10E3F0003318D600B365B7003393D800935808019B
:10E40000B3D61503131608011356060193570301DB
:10E4100033F7150313850600B305D602131707015A
:10E42000B367F70063FEB700B38707011385F6FFF4
:10E4300063E8070163F6B7001385E6FFB3870701BA
:10E44000B387B74033F717031313030113530301C3
:10E45000B3D717031317070133636700B306F60238
:10E4600013860700637CD300330368001386F7FF2D
:10E47000636603016374D3001386E7FF1315050178
:10E480003365C500930500006F00400E370500019D
:10E4900013070001E36CA6F2130780016FF01FF36E
:10E4A00063160600130710003358C7023707010030
:10E4B0006370E80C1307F00F637407011305800005
:10E4C0003357A800B386E60003C706001306000210
:10E4D0003307A700B306E6406316E60AB387074191
:10E4E00093051000935808011316080113560601EE
:10E4F00013570301B3F61703B3D717039396060117
:10E5000033E7E600330EF60213850700637EC7018A
:10E51000330707011385F7FF636807016376C701B7
:10E520001385E7FF330707013307C741B3771703A5
:10E530001313030113530301335717039397070171
:10E5400033E36700B306E60213060700637CD300DB
:10E55000330368001306F7FF636603016374D30097
:10E560001306E7FF131505013365C500678000003A
:10E570003707000113050001E364E8F41305800187
:10E580006FF01FF43318D80033D5E7003393D80069
:10E59000B397D70033D7E800935808013366F700E4
:10E5A000337715039317080193D707019355060195
:10E5B00033551503131707013367B700B386A70256
:10E5C00093050500637ED700330707019305F5FF28
:10E5D000636807016376D7009305E5FF33070701FA
:10E5E000B306D74033F71603131606011356060178
:10E5F000B3D61603131707013385D702B367C700D5
:10E600001387060063FEA700B38707011387F6FF91
:10E6100063E8070163F6A7001387E6FFB3870701E6
:10E6200093950501B387A740B3E5E5006FF09FEB35
:10E6300063E6D5183707010063F4E6041307F00F0B
:10E64000B335D700939535003747018033D5B600F1
:10E65000130747583307A7000347070013050002B5
:10E660003307B700B305E5406316E5021305100054
:10E67000E3EEF6EE33B5C800134515006FF01FEF5B
:10E680003707000193050001E3E0E6FC93058001F4
:10E690006FF09FFB3358E600B396B6003368D8009E
:10E6A00033DEE700935E0801B376DE03B397B7006D
:10E6B00033D7E8003313B6003366F7009317080129
:10E6C00093D7070113570601335EDE0393960601C5
:10E6D00033E7E600338FC70313050E00637EE701BF
:10E6E000330707011305FEFF636807016376E7013F
:10E6F0001305EEFF330707013307E741B376D7036E
:10E700003357D70393960601338EE702931706011A
:10E7100093D70701B3E7F6001306070063FEC701AE
:10E72000B38707011306F7FF63E8070163F6C70124
:10E730001306E7FFB387070113150501B70E0100A4
:10E740003365C5009386FEFF3378D5001356050167
:10E75000B376D30013530301B387C741330ED802F6
:10E76000B306D60213570E01330868023308D800E7
:10E7700033070701330666026374D7003306D601F8
:10E78000935607013386C60063E6C702E39CC7CEF3
:10E79000B70701009387F7FF3377F70013170701D7
:10E7A000337EFE00B398B8003307C701930500001D
:10E7B000E3FEE8DA1305F5FF6FF0DFCC9305000008
:10E7C000130500006FF09FDA930E05001383050018
:10E7D0001308060093870600639A062237470180D4
:10E7E0001307475863FCC50CB7060100637ED60AC1
:10E7F0009306F00F63F4C60093078000B356F6004B
:10E800003307D70003470700B307F70013070002D9
:10E81000B308F740630CF700B3151301B3D7FE003C
:10E8200033181601B3E5B70033951E01935608015E
:10E83000B3F7D50213160801135606011357050145
:10E84000B3D5D5029397070133E7E700B305B602C6
:10E85000637AB70033070701636607016374B70083
:10E86000330707013307B740B377D7021315050104
:10E87000135505013357D7029397070133E5A700D6
:10E880003307E602637AE500330505016366050197
:10E890006374E500330505013305E5403355150183
:10E8A0009305000067800000B70600019307000190
:10E8B000E366D6F4930780016FF05FF463160600F9
:10E8C0009306100033D8C602B70601006376D8124B
:10E8D0009306F00F63F4060193078000B356F80027
:10E8E0003307D70003460700B30503413306F6009C
:10E8F00093070002B388C7406386C708331818011E
:10E90000B357C300B31513011353080133D6CE0018
:10E910003366B6009315080193D5050133951E01A2
:10E92000B3D6670233F7670293570601B386D50261
:10E93000131707013367F700637AD700330707011E
:10E94000636607016374D70033070701B306D74036
:10E9500033F766021316060113560601B3D6660294
:10E9600013170701B386D502B365C70063FAD50054
:10E97000B385050163E6050163F4D500B3850501A0
:10E98000B385D5409356080133F7D5029317080194
:10E9900093D7070113560501B3D5D5021317070105
:10E9A0003367C700B385B702637AB700330707013F
:10E9B000636607016374B70033070701B305B74007
:10E9C00033F7D5021315050113550501B3D5D5024B
:10E9D000B385B7029317070133E5A700637AB50043
:10E9E00033050501636605016374B5003305050150
:10E9F0003305B5406FF09FEAB706000193070001A9
:10EA0000E36ED8EC930780016FF05FEDE3ECD5E89F
:10EA1000B707010063F8F6049308F00FB3B7D80006
:10EA2000939737003747018033D8F60013074758CC
:10EA30003307070183480700B388F80093070002F3
:10EA400033881741639A170363E46600E3ECCEE46E
:10EA50003385CE40B305D340B3BEAE00B385D541B8
:10EA60006FF05FE43707000193070001E3ECE6FA7B
:10EA7000930780016FF01FFBB3571601B396060191
:10EA800033EED700335F1301B3D71E0133950E0168
:10EA9000935E0E01B31503013353DF03B3E7B700F1
:10EAA00093150E0193D5050113D7070133160601FF
:10EAB000B376DF03338F65029396060133E7E600F2
:10EAC00093060300637EE7013307C7019306F3FF54
:10EAD0006368C7016376E7019306E3FF3307C70165
:10EAE0003307E7413373D7039397070193D70701A0
:10EAF0003357D703131303013363F300B385E502E0
:10EB000093070700637EB3003303C3019307F7FF46
:10EB10006368C3016376B3009307E7FF3303C30160
:10EB200093960601370F0100B3E6F600B305B34034
:10EB30001303FFFFB3FE66001357060193D60601C9
:10EB400033736600B3876E0233836602B38EEE02C0
:10EB5000B386E602B38E6E0013D707013307D701E1
:10EB600063746700B386E60113530701B306D3004D
:10EB7000370301001303F3FF33776700131707010F
:10EB8000B3F76700B307F70063E6D500639ED500CF
:10EB9000637CF5003386C740B3B7C700B387C701AE
:10EBA000B386F64093070600B307F5403335F5000A
:10EBB000B385D540B385A540B398150133D507017A
:10EBC00033E5A800B3D505016FF0DFCD130101FDDA
:10EBD00023248102232A5101232291012326110299
:10EBE0002322910223202103232E3101232C4101D2
:10EBF00023286101232671012324810113040500C8
:10EC0000930C0600938A06007329200013DB45014C
:10EC1000939BC500137BFB7F93DBCB0013DAF501DD
:10EC2000630A0B029307F07F6308FB081357D501B3
:10EC3000939B3B00B36B7701B7078000B3EBFB00FE
:10EC400093193500130B1BC0130C00009304000034
:10EC50006F00C008B3E7AB00638E070E63800B0440
:10EC600013850B00EF401039130755FF9307C001C0
:10EC700063CCE7029306D001930985FFB386E64093
:10EC8000B39B3B01B356D400B3EB7601B319340107
:10EC90009305D0C0338BA5406FF01FFBEF4090353C
:10ECA000130505026FF05FFC930B85FDB31B740128
:10ECB000930900006FF0DFFD33E4AB006306040A44
:10ECC000B7070800B3F7FB0093090500130BF07FAB
:10ECD000130C300093040001E39A07F61395CA0061
:10ECE0001354C50013D54A019375F57F93870C0023
:10ECF00093DAFA01638405081307F07F6386E50E53
:10ED000093D7DC011315340033E5A70037048000E6
:10ED10003364850093973C00138515C013070000EA
:10ED200093162C00B3E6E600B305AB409386F6FFDE
:10ED30001305E00033465A016362D5103745018060
:10ED4000939626001305054DB386A60083A60600FC
:10ED500067800600930B000093090000130B00006E
:10ED6000130C10006FF09FEE930B0000930900004E
:10ED7000130BF07F130C20006FF05FEDB36794016D
:10ED8000638607086302040413050400EF4090261D
:10ED900093050500938655FF9307C00163CED70204
:10EDA0001307D001938785FF3307D7403315F4004D
:10EDB00033D7EC003364A700B397FC001307D0C02F
:10EDC0003305B7406FF09FF513850C00EF4090229C
:10EDD000930505026FF01FFC138585FD3394AC008D
:10EDE000930700006FF09FFD33669401630A0602EB
:10EDF000370708003377E4001305F07F631C070230
:10EE000013073000930400016FF09FF1130400001A
:10EE10009307000013050000130710006FF05FF068
:10EE200013040000930700001305F07F1307200070
:10EE30006FF01FEF130730006FF09FEE63667401F1
:10EE400063968B2E63E4F92E1395FB0113D71900FB
:10EE50009396F90193DB1B00B369E5001315840059
:10EE600013D887013368A8001355050133DEAB02C0
:10EE7000131F0801135F0F019398870093D70901AF
:10EE8000B3FBAB0213030E003307CF03939B0B01BD
:10EE9000B3E7770163FEE700B38707011303FEFFC3
:10EEA00063E8070163F6E7001303EEFFB38707018A
:10EEB000B387E740B3DEA702139709011357070191
:10EEC000B3F7A70293890E00330EDF039397070170
:10EED0003367F700637EC701330707019389FEFF9D
:10EEE000636807016376C7019389EEFF3307070163
:10EEF00013130301B369330137030100930EF3FFCA
:10EF000093D2090193DF08013307C74133FED901CA
:10EF1000B3FED801B307DE033384D203338ECF03AD
:10EF2000B3038E0013DE0701330E7E00B382F203BB
:10EF300063748E00B3826200B703010013530E01A5
:10EF40009383F3FFB302530033737E001313030163
:10EF5000B3F777003303F3006368570013840900A5
:10EF60006314570463F26604B3861601B3B716013F
:10EF7000B38707013307F7001384F9FF6366E800DE
:10EF80006314E80263E2160363665700639EE200BF
:10EF900063FC6600B3861601B3B71601B387070199
:10EFA0001384E9FF3307F700338366403307574084
:10EFB000B3B666003307D7409307F0FF6304E81247
:10EFC000B352A702935703013377A7029386020037
:10EFD000330E5F021317070133E7E700637EC701B3
:10EFE000330707019386F2FF636807016376C70161
:10EFF0009386E2FF330707013307C741335EA70259
:10F000009317030193D707013377A702330FCF0379
:10F010001317070133E7E70093070E00637EE7014C
:10F02000330707019307FEFF636807016376E70173
:10F030009307EEFF3307070193960601B3E6F60048
:10F040009397060193D7070113D30601338E6F02FE
:10F050003307E741B38FFF02338FFE02B30ED303B2
:10F0600093570F01B38FDF01B387F70163F6D70121
:10F0700037050100330EAE0013D307013303C3017C
:10F08000370E0100130EFEFF33F5C70113150501FE
:10F09000337FCF013305E501636867006312673E84
:10F0A00093870600630005043307E8009387F6FFA3
:10F0B00063640703636667006312673C63F0A8023A
:10F0C0009387E6FF93961800B3B8160133880801BA
:10F0D0003307070193880600631467006384A80060
:10F0E00093E717001388F53F635C001913F7770067
:10F0F000630A070A1307200093E414006302E90A75
:10F10000130730006308E908631E090813F7F700C6
:10F11000930640006308D70813874700B337F7000A
:10F120003304F400930707006F00C0079385F5FFD1
:10F13000930600006FF09FD213060A0013840B00A1
:10F140009387090013070C0093063000630ED73035
:10F15000930610006304D73093062000E314D7F819
:10F160006F00000113860A006FF01FFE93E4840015
:10F1700013050000930700001307F07F6F000006DF
:10F18000370408009307000013060000130730003F
:10F190006FF09FFB63180600138787006FF01FF85E
:10F1A000E31C06FE370700013377E400630A07001B
:10F1B000370700FF1307F7FF3374E4001388054097
:10F1C0001307E07F634E070713D737009317D40167
:10F1D000B3E7E7001355340013070800131747017E
:10F1E000B706F07F1315C5003377D7001355C50058
:10F1F0003365A7001316F6013367C50093050700B2
:10F20000138507006384040073A014008320C102E7
:10F210000324810283244102032901028329C101BD
:10F22000032A8101832A4101032B0101832BC100A1
:10F23000032C8100832C410013010103678000002F
:10F2400093072000630AF90293073000630AF9006C
:10F25000631A0900930700001307F07F6F00000195
:10F26000E30A06FE9307F0FF1307E07F93E45400E0
:10F27000138507006FF09FF6E31E06FC6FF09FFEFC
:10F28000130710006310080693F6770013070400B5
:10F29000638406049306200093E41400630CD902EF
:10F2A000930630006302D9026318090293F6F7004F
:10F2B000130540006382A60213B7C7FF1347170068
:10F2C000330787006F0040016318060013B787FFFC
:10F2D0006FF0DFFEE31C06FE13578701134717008C
:10F2E00013771700130510003305054193068003BB
:10F2F00063CEA60E9306F00163C2A6069385E54190
:10F3000033D8A700B316B400B397B700B3E606012D
:10F31000B337F000B3E7F6003355A40093F6770057
:10F32000638006089306200093E414006308D9065E
:10F3300093063000630ED9046314090693F6F700B0
:10F3400093054000638EB60493864700B3B7F6007A
:10F350003305F500938706006F008004930610FEC6
:10F36000B386064193080002B356D4001308000088
:10F37000630615019385E5433318B400B367F800BD
:10F38000B337F000B3E7F600130500006FF01FF984
:10F3900063180600938687006FF05FFBE31C06FE90
:10F3A000B7068000B376D500638E060093E41400A0
:10F3B00013050000930700006316070213071000EF
:10F3C0006FF0DFE193D637009317D501B3E7D7008D
:10F3D00013553500E30407E013F71400E30007E0DA
:10F3E0001307000093E424006FF05FDFB3E78700AA
:10F3F000638407029307200093E41400630EF9026C
:10F40000930730006302F9029307100063140900A8
:10F410009307500093D7370093E4240013050000AE
:10F42000130700006FF09FDB93079000E30406FED4
:10F43000930710006FF01FFE93079000E31C06FC7B
:10F440006FF01FFF37050800930700001307F07FD8
:10F4500013060000930400016FF05FD8130500004D
:10F46000930700006FF0DFFB3705080093070000EB
:10F470001307F07F130600006FF05FD69386070036
:10F48000938706006FF0DFC5130101FD232481027D
:10F49000232A5101232291012326110223229102C2
:10F4A00023202103232E3101232C41012328610134
:10F4B000232671012324810113040500930C060007
:10F4C000938A06007329200093DB45019399C500B8
:10F4D00093FBFB7F93D9C90013DBF501638A0B0211
:10F4E0009307F07F6388FB089357D5019399390000
:10F4F000B3E93701B7078000B3E9F900131A350003
:10F50000938B1BC0130C0000930400006F00C00815
:10F51000B3E7A9006380071063800904138509001D
:10F52000EF40402D130755FF9307C00163CCE7025E
:10F530009307D001130A85FFB387E740B3994901C8
:10F54000B357F400B3E93701331A4401930BD0C029
:10F55000B38BAB406FF01FFBEF40C02913050502D2
:10F560006FF05FFC930985FDB3193401130A0000A5
:10F570006FF0DFFD33E4A9006308040AB707080051
:10F58000B3F7F900130A0500930BF07F130C30005A
:10F5900093040001E39A07F613D54A011394CA00B5
:10F5A0001375F57F93870C001354C40093DAFA01A6
:10F5B000630605081307F07F6306E50E93D7DC01A9
:10F5C0001314340033E48700B70780003364F40079
:10F5D000130515C093973C001307000093162C00E9
:10F5E000B3E6E600B38BAB009386F6FF1306E000AC
:10F5F000B3455B0113851B00636CD616374601804B
:10F60000939626001306C650B386C60083A606004E
:10F610006780060093090000130A0000930B0000A6
:10F62000130C10006FF05FEE93090000130A000046
:10F63000930BF07F130C20006FF01FEDB367940164
:10F64000638407086300040413050400EF40801A74
:10F65000930655FF9307C00163CED7021307D0016D
:10F66000930785FF3307D7403314F40033D7EC00FA
:10F6700033648700B397FC001307D0C03305A7405D
:10F680006FF09FF513850C00EF40C01613050502BF
:10F690006FF01FFC130485FD33948C00930700006A
:10F6A0006FF09FFD33669401630A06023707080076
:10F6B0003377E4001305F07F631C07021307300063
:10F6C000930400016FF09FF1130400009307000002
:10F6D00013050000130710006FF05FF01304000023
:10F6E000930700001305F07F130720006FF01FEF52
:10F6F000130730006FF09FEE3704080093070000F7
:10F700001307F07F930500009304000113174701CE
:10F71000B706F07F1314C4003377D7001354C40026
:10F720009395F501336487003367B40013850700B0
:10F73000930507006384040073A014008320C102B2
:10F740000324810283244102032901028329C10188
:10F75000032A8101832A4101032B0101832BC1006C
:10F76000032C8100832C41001301010367800000FA
:10F77000B70E0100138EFEFF13570A0193D807013D
:10F78000337ACA01B3F7C70133884803B386470306
:10F79000330FF7023303E80113D80601330868007A
:10F7A000330617036374E8013306D601935F08013B
:10F7B0003378C801B3F6C601935E0401337EC401F9
:10F7C000131808013308D800330FC703B306CA0360
:10F7D000338A4E033303EA0113DA0601330A6A005F
:10F7E0003307D7036376EA01370301003307670065
:10F7F00013530A013303E30037070100130FF7FF28
:10F80000337AEA01B3F6E60113D40901131A0A01A7
:10F81000B3F9E901338F3703330ADA00B38F4F01AD
:10F82000B3863803B307F402B3828802B388F600C4
:10F8300093560F01B386160163F4F600B382E2001B
:10F84000370701009307F7FF337FFF0093D80601C6
:10F85000B3F6F600B387C90393960601B386E601B3
:10F86000B3885800330EC403B3893E03338F8E022E
:10F87000B389C90113D40701B309340163F4C90181
:10F88000330FEF00370E0100130EFEFF33F7C901EF
:10F89000B3F7C701131707013306F6013307F70063
:10F8A000333A460133076700330447013306D60075
:10F8B000B336D600330E1401B30EDE0033376700C3
:10F8C0003334440133648700B3B6DE0093D90901B1
:10F8D000B3381E0133043401B3E6D8003304D40036
:10F8E0003304E40193D77E01131494003364F400CD
:10F8F00093179600B3E70701B337F000135676016C
:10F9000037070001B3E7C700939E9E003377E400FA
:10F91000B3E7D7016300070A13D7170093F717005F
:10F92000B367F7001317F401B3E7E70013541400AB
:10F930001308F53F635A001113F7770063080708AF
:10F940001307200093E414006300E9081307300054
:10F950006306E906631C090613F7F70093064000E7
:10F960006306D70613874700B337F7003304F40064
:10F97000930707006F00800593050B0013840900AF
:10F9800093070A0013070C00930620006300D72892
:10F99000930630006304D72893061000E31AD7F8C3
:10F9A00013040000930700006F00002493850A00F1
:10F9B0006FF09FFD13850B006FF09FF763980500B4
:10F9C000138787006FF05FFAE39C05FE370700019D
:10F9D0003377E400630A0700370700FF1307F7FFD8
:10F9E0003374E400130805401307E07F634E0701FA
:10F9F00013D737009317D401B3E7E700135434004B
:10FA0000130708006FF09FD093072000630AF902E4
:10FA100093073000630AF900631A09009307000096
:10FA20001307F07F6F000001E38A05FE9307F0FFE4
:10FA30001307E07F93E45400138407006FF01FCD99
:10FA4000E39E05FC6FF09FFE13071000631008068D
:10FA500093F67700130704006384060493062000DE
:10FA600093E41400630CD902930630006302D902B8
:10FA70006318090293F6F700130640006382C6027A
:10FA800013B7C7FF13471700330787006F00400104
:10FA90006398050013B787FF6FF0DFFEE39C05FE58
:10FAA00013578701134717001377170093061000A9
:10FAB000B386064113068003634ED60E1306F0018B
:10FAC0006342D6061305E5413316A40033D8D700A8
:10FAD000B397A70033660601B337F000B367F600AB
:10FAE0003354D40093F67700638006089306200011
:10FAF00093E414006308D90693063000630ED9041A
:10FB00006314090693F6F70013064000638EC604DB
:10FB100093864700B3B7F6003304F40093870600DA
:10FB20006F008004130610FE33060641930800029E
:10FB30003356C40013080000638616011305E5431D
:10FB40003318A400B367F800B337F000B367F600CA
:10FB5000130400006FF01FF9639805009386870077
:10FB60006FF05FFBE39C05FEB7068000B376D40020
:10FB7000638E060093E41400130400009307000052
:10FB800063160702130710006FF05FB893D63700B3
:10FB90009317D401B3E7D70013543400E30807B632
:10FBA00013F71400E30407B61307000093E42400DE
:10FBB0006FF0DFB5B3E78700638407029307200087
:10FBC00093E41400630EF902930730006302F90214
:10FBD00093071000631409009307500093D7370070
:10FBE00093E4240013040000130700006FF01FB219
:10FBF00093079000E38405FE930710006FF01FFE4B
:10FC000093079000E39C05FC6FF01FFF13040000B6
:10FC1000930700001307F07F6FF05FAF3704080011
:10FC2000930700001307F07F930500006FF01FAEED
:10FC300083270500832E4500032F85008326C500FA
:10FC400003A7050083A2450083AF850003A3C50079
:10FC5000130101FF732620003788000013D6060128
:10FC60001308F8FF139E06019315030193D8F601BC
:10FC70003376060193560301135E0E0193D50501F9
:10FC8000B3F606011353F301631E060133E8D701EF
:10FC90003368E8013368C80163120808639CC60A28
:10FCA0006F008000639A0601336857003368F801DB
:10FCB0003368B80063160804130510006396C60283
:10FCC0006394E70263925E026310FF03631EBE004B
:10FCD00063846802639A060033E5D7013365E50162
:10FCE0003365C5013335A0001301010167800000B1
:10FCF000736018006F000006130500006FF0DFFE50
:10FD0000378500001305F5FF6310A604B3E7D7019C
:10FD1000B3E7E701B3E7C7016388070213150E01D4
:10FD200013550541E35605FCB78700009387F7FF9D
:10FD300013051000E39AF6FA336757003367F701AB
:10FD40003367B700E30207FA9395050193D50541A0
:10FD5000E3D005FA130510006FF01FF9832F05009B
:10FD600003284500032E850083A205000325C50056
:10FD700083A8450083AE850083A6C500130101FF5B
:10FD8000F3272000B7870000135605019387F7FF7C
:10FD9000931505011393060113D706013376F60078
:10FDA00093D505011355F501135303013377F7007C
:10FDB00093D6F6016310F602B367F801B3E7C70103
:10FDC000B3E7B700638A070C736018001305E0FF00
:10FDD0006F004006631AF700B3E71201B3E7D701DB
:10FDE000B3E76700E39207FE631A060AB367F801F8
:10FDF000B3E7C701B3E7B70093B71700631A07006B
:10FE000033EF1201336FDF01336F6F00630A0F06A8
:10FE1000639C07006394A6006352C702630E050447
:10FE20001305F0FF6F0000011305F0FF6384060067
:10FE30001385060013010101678000006356E60088
:10FE4000E31A05FE6FF0DFFDE36AB3FC639E650213
:10FE5000E3E6CEFD631EDE03E3E208FD6314180152
:10FE6000E3EEF2FBE36E18FD63141801E3EA5FFCB6
:10FE7000130500006FF01FFC130510006FF09FFBCF
:10FE8000E39807FE6FF09FF9E3EC65FA6FF05FFE11
:10FE9000E368DEFB6FF0DFFDE300C7F4E31C07F669
:10FEA000930700006FF0DFF5832F0500032845005E
:10FEB000032E850083A205000325C50083A8450005
:10FEC00083AE850083A6C500130101FFF327200040
:10FED000B7870000135605019387F7FF93150501B7
:10FEE0001393060113D706013376F60093D5050167
:10FEF0001355F501135303013377F70093D6F60139
:10FF00006310F602B367F801B3E7C701B3E7B700C0
:10FF1000638A070C73601800130520006F00400609
:10FF2000631AF700B3E71201B3E7D701B3E767003D
:10FF3000E39207FE631A060AB367F801B3E7C70145
:10FF4000B3E7B70093B71700631A070033EF120146
:10FF5000336FDF01336F6F00630A0F06639C070086
:10FF60006394A6006352C702630E05041305F0FFF5
:10FF70006F0000011305F0FF63840600138506007F
:10FF800013010101678000006356E600E31A05FED5
:10FF90006FF0DFFDE36AB3FC639E6502E3E6CEFD2E
:10FFA000631EDE03E3E208FD63141801E3EEF2FBD7
:10FFB000E36E18FD63141801E3EA5FFC130500000B
:10FFC0006FF01FFC130510006FF09FFBE39807FE16
:10FFD0006FF09FF9E3EC65FA6FF05FFEE368DEFB1C
:10FFE0006FF0DFFDE300C7F4E31C07F693070000A2
:10FFF0006FF0DFF5130101F4232A910A2326310B58
:02000004800179
:100000002322510B2320610B232E7109232A9109EE
:100010009309050083A6050083A7450003A5850075
:1000200083ABC500832C060083244600032B860087
:10003000832AC600232E110A232C810A2328210B90
:100040002324410B232C81092328A1092326B1094C
:10005000732920003786000013970B0113DA0B0178
:10006000135707011306F6FF232671072320D10635
:100070002322F1062324A1062328D102232AF102F8
:10008000232CA102232EE102337ACA0093DBFB0169
:1000900063000A06630ACA16370501003367A70022
:1000A000232EE102130601039307C10303A70700F0
:1000B00083A6C7FF9387C7FF1317370093D6D601D0
:1000C0003367D70023A2E700E312F6FE832701037C
:1000D00037C5FFFF13051500939737002328F1025A
:1000E000330AAA00130C0000130400006F00001470
:1000F00033E6D7003366A6003366E60063020620C7
:100100006300070813050700EF30C06E13040500F5
:10011000130744FF135657401377F701630C070882
:100120009307C0FFB307F60213050002930801030B
:100130003305E540931526009387C700B387F80081
:100140006392F80A93070108B385B7008327010378
:100150001306F6FF3397E70023A8E5FA1306160007
:1001600037CAFFFF1316260093050000130501038D
:10017000130A1A01EF009FBF330A8A406FF09FF6FF
:1001800063080500EF300067130405026FF05FF8A5
:10019000638A070013850700EF30C0651304050468
:1001A0006FF01FF713850600EF30C06413040506D7
:1001B0006FF01FF69306C0FFB306D6029307C10384
:1001C00013073000B385D70083A505001307F7FF99
:1001D0009387C7FF23A2B700E356C7FE1306F6FFB7
:1001E0006FF0DFF783A6070003A8C7FF3383B700CC
:1001F000B396E6003358A800B3E606012320D300E7
:100200009387C7FF6FF0DFF3B3E7D700B3E7A7002B
:10021000B3E7E700638C070E131707011357074175
:10022000130C300013040001E34007EC13950A019E
:100230003787000093D70A01135505011307F7FF0D
:1002400023265107232091072322910623246107A7
:100250002320910523229104232461052326A10450
:10026000B3F7E70093DAFA016386070A6380E71CB5
:10027000370701003365E5002326A1049305010437
:100280001307C104832607000326C7FF1307C7FF10
:10029000939636001356D601B3E6C6002322D70044
:1002A000E392E5FE0327010437C5FFFF13051500A0
:1002B000131737002320E104B387A70013070000BA
:1002C000B38747012324F100938717002322F1000D
:1002D00093172C00B3E7E7009387F7FF9306E0003E
:1002E000B3C45B0163E2F61AB74601809397270017
:1002F00093868654B387D70083A7070067800700DB
:10030000130A0000130C10006FF01FDE130C200006
:100310006FF09FDDB3E79401B3E76701B3E7A70090
:10032000638C0712630E0506EF30C04C9304050082
:10033000938744FF13D6574093F7F701638E07085E
:100340001307C0FF3307E6021305000293080104F8
:100350003305F540931526001307C7003387E800DF
:100360006394E80A13070108B305B70003270104E3
:100370001306F6FFB317F70023A0F5FC13061600CB
:10038000131626009305000013050104EF001F9EBD
:10039000B7C7FFFF93871701B38797406FF01FF22E
:1003A000630A0B0013050B00EF30C04493040502F1
:1003B0006FF01FF8638A040013850400EF30804358
:1003C000930405046FF0DFF613850C00EF308042D4
:1003D000930405066FF0DFF59306C0FFB306D6025F
:1003E0009307C10413073000B385D70083A5050028
:1003F0001307F7FF9387C7FF23A2B700E356C7FE93
:100400001306F6FF6FF09FF7832607000328C7FF48
:100410003303B700B396F6003358A800B3E60601DD
:100420002320D3001307C7FF6FF09FF3B3E49401B9
:10043000B3E46401B3E4A40013072000E38204E8FA
:10044000131505011355054113073000E34A05E66E
:10045000130400016FF0DFE693070000130710009C
:100460006FF01FE613040001378A0000232E4105B8
:10047000232C0104232A010423280104130AFAFF70
:10048000930400006F0010100326010303250104EC
:10049000B70801009386F8FF9352060193570501B0
:1004A0003376D6003375D5003387C702B305C5024E
:1004B0003383A2023308670013D70501330707010E
:1004C000B383F20263746700B3831301032341040F
:1004D000135807013377D700B3F5D5001317070179
:1004E0003307B700135F03013373D300B308C302AC
:1004F0002326E1002320E106B38662023307CF0200
:10050000B305D70013D708013307B700B38BE20355
:100510006376D700B7060100B38BDB009356070163
:10052000370E01002320D1009306FEFFB375D700DC
:10053000B3F8D80093950501B38515013307B800CA
:100540002320E10203274103935F0701B376D7001D
:10055000B388A602338AAF0213D808013387D702C3
:10056000330747013307E800B38EF703637447018D
:10057000B38ECE0113580701370A01003308D801A2
:10058000130EFAFF130B08003378C701B3F8C80144
:1005900013180801338E6602330818013307DF028F
:1005A000935A0E01B3886F02330717013387EA00AD
:1005B000B30EFF0363741701B38E4E019358070106
:1005C000B388D801B70A0100232811019388FAFFE4
:1005D00033771701337E1E0113170701B30DC701CF
:1005E00003278104B3781701135E0701338AC80219
:1005F000338C1203935C0A01B30ECE02B38E8E01CC
:10060000B38EDC013387C20363F48E0133075701D5
:1006100093DA0E013387EA00370D0100232AE10047
:100620001307FDFFB3FEEE00337AEA00939E0E013E
:10063000B38E4E01032A8103232CD1013377EA00C4
:10064000935E0A01338AAE02B30AA702B38CE702B3
:10065000B38C4C0113DA0A01330A9A01B38CAE024F
:10066000338CD70363749A01330CAC01935C0A0199
:10067000338C8C01232E8101370C0100130DFCFFFC
:10068000337AAA01B3FAAA01131A0A01B30C5A0168
:10069000032A0102B3834301032A0100B3B5B30067
:1006A000B3830301330ABA00B30B7A01338C6B01B5
:1006B00033B80301B30A0C0133B80A01333C6C01AF
:1006C00033680C01B3BBBB00B30B78010328810175
:1006D000338ABA01B33DBA0183250101330A0A0105
:1006E00033380A01232C010103284101B38BBB00DD
:1006F000232071002322710683238101B385BB016E
:1007000033880501B30A78008323C101330A9A01B3
:10071000B33C9A01338C7A00B3039C01138B030022
:1007200083230101B3B5B501B33C9B01B3BB7B008F
:10073000B3EBBB0083254101232441073338B800C4
:1007400083258101B3BABA008325C101B36A580178
:10075000B38B5B01333CBC00B36C9C01B3859B0144
:10076000232AB1008325C10413D8050133FDA50157
:10077000B305CD02B38AA20393DB05013306C80299
:10078000330656013386CB00B382020363765601EB
:10079000370C0100B3828201935A0601B3825A00DA
:1007A000370C0100832AC103232E51009302FCFF62
:1007B00033765600B3F5550013160601B3F25A000E
:1007C0003306B60093D50A01B38BB702B38AA202EF
:1007D000B387570293DD0A013385A502B387A700CB
:1007E000B387FD0063F4A700B38B8B01370C0100C6
:1007F000930DFCFF13D50701B3F7B701330575015E
:1008000093970701B3FDBA012320A102B38A1F0306
:10081000B38DB7013385D802B307DE02935C0501BF
:10082000B3875701B387FC00B38BCF0363F4570141
:10083000B38B8B0193DA0701B3837A01B70B010005
:10084000938AFBFFB3F7570133755501939707015F
:10085000B387A700B38A6E022328F1002322710216
:10086000B3076702B30CEF0213D50701B38C5C0129
:1008700033059501330CDF0363745501330C7C01A0
:10088000935A0501338C8A01B70A0100938AFAFF53
:100890003375550113150501B3F75701B307F5007B
:1008A0008323C10103254101B30ACB0033B6CA003B
:1008B000B30C7500832301023385CC00B38ABA01DF
:1008C000B3BDBA01B30B7500B383BB01232671021C
:1008D00083230101032B41023336C500B38A7A001A
:1008E000B3B37A0023247102B383BB01B3836301E2
:1008F000032B81020325010223287100B38AFA0029
:10090000B3836301138B0300B3B7FA00B38383018E
:10091000232A7100B383F300B3BBAB00232C710017
:100920000325C1028323C10123265107B33DB5012D
:10093000B3BC7C000325010183234102B3EDBB015D
:1009400033E6CC00B33B75000325410183238102CC
:100950003306B601333C850103258101B33D7B009D
:10096000B3EDBB01B337F5003306B601330517030A
:10097000B36DFC00B30DB601338C1E031356050195
:10098000B307EE02B3878701B307F600B30BDE03AC
:1009900063F6870137060100B38BCB0013D607013E
:1009A000370C0100B30B76011306FCFFB3F7C70049
:1009B0003376C500B38CAF03939707013386C70026
:1009C0003305DD02B306D80293570501B3869601BD
:1009D000B387D700B38F0F0363F49701B38F8F01F1
:1009E00093D60701B70C0100B38FF6019386FCFF85
:1009F000B3F7D70093970701B376D500330CBF0246
:100A0000B386D700330F5F02B38762023383650278
:100A100013D50701330F6F00330FE50163746F00C7
:100A2000330C9C0113530F0133038301370C010076
:100A30001305FCFF337FAF00131F0F0133F5A70031
:100A4000B38CAE033305AF00330FA7033307E802BF
:100A500093570F0133079701B387E700B38E0E0357
:100A600063F49701B38E8E0113D70701370C010091
:100A7000B30ED7011307FCFFB3F7E7009397070105
:100A80003377EF003387E700330FBE02B3871203DB
:100A9000330E5E0293DC0701B3881503330E1E018B
:100AA000338ECC0163741E01330F8F0193580E01F6
:100AB000338FE801B7080100832381019388F8FF91
:100AC000337E1E01B3F71701131E0E01330EFE0015
:100AD000B387C30033B6C700B38D7D01B383CD00A8
:100AE000B387D700B3B6D700338CF301B387A70021
:100AF000138B0300B303DC002328F106B3B7A70070
:100B000033856300B30CF50023287100B383EC0038
:100B100033B7E300232A710083230101B3BD7D01B4
:100B20003336CB00B33FFC01B3B6D30033E6CD0080
:100B3000B3E6DF00B3B7FC00B33D65003306D60073
:100B4000B3EDFD00B30DB60103264101B38DDD0108
:100B5000B386ED00B307C6013386A203B3BEDD0141
:100B600033B7E60033E7EE00232AF106B38EE60141
:100B7000B3B7C701B386FE00B3B7F600B3BEEE014C
:100B8000338DA503B3EEFE0093570601B30258025E
:100B9000B382A201B305B802338857006376A80177
:100BA000B7070100B385F500B377180193970701E4
:100BB000B378160113580801B38817013308E80009
:100BC0008327C10003270100B38616013308D8012B
:100BD000B3B81601B3E3E70033081801B305B80052
:100BE000336A7A00939ADA00232EB106232CD106B9
:100BF00033EA4A01930701061306010703A7C7005A
:100C000083A6070193874700135737019396D600B1
:100C10003367D70023AEE7FEE312F6FE0327810613
:100C2000832A01068327C106232CE10403274106FA
:100C3000333A4001336A5A01232AE104370710008E
:100C4000232EF10423284105B3F7E700638C072224
:100C5000131AFA01930701051306C10503A707003C
:100C600083A6470093874700135717009396F60112
:100C70003367D70023AEE7FEE312F6FE8327C105F4
:100C8000333A400193D71700232EF104832701053F
:100C900033EA4701232841058327410037470000F5
:100CA0001307F7FF3387E7006356E02A8327010520
:100CB00093F677006380060613062000832641051D
:100CC0008325C10513641400630EC91E130630008A
:100CD0006300C91C6310090413F6F70013054000F4
:100CE000630AA602938747002328F10493B74700BD
:100CF000B386D700B3B7F600232AD1048326810533
:100D0000B386D700232CD104B3B6F600B386B60061
:100D1000232ED1048327C105B7061000B3F6D700F0
:100D2000638006023707F0FF1307F7FFB3F7E7000A
:100D3000232EF10483274100374700003387E70063
:100D4000930701059305C10583A6070003A6470085
:100D50009387470093D636001316D601B3E6C60034
:100D600023AED7FEE392F5FEB78700009387E7FF37
:100D700063C2E7188327C105130A070093D737001A
:100D8000232EF1048327C105131A1A019394F4004A
:100D9000135A1A0133EA44012316F10623174107B7
:100DA0000326010583264105032781058327C10604
:100DB00063040400732014008320C10B0324810BFF
:100DC00023A0C90023A2D90023A4E90023A6F90087
:100DD0008324410B0329010B032A810A832A410A38
:100DE000032B010A832BC109032C8109832C4109A0
:100DF000032D0109832DC108138509008329C10A28
:100E00001301010C6780000093840B00832701030A
:100E10002328F10483274103232AF1048327810334
:100E2000232CF1048327C103232EF1049307200010
:100E3000630AFC48930730006308FCE29307100044
:100E4000E31CFCE4232E0104232C0104232A0104C7
:100E5000232801046F00004593840A0083270104BE
:100E6000130C07002328F10483274104232AF104EB
:100E700083278104232CF1048327C104232EF1044A
:100E80006FF0DFFA832781002322F1006FF0DFE0AB
:100E9000E39204E893878700032681052328F10461
:100EA00093B78700B386D700B3B7F6003386C70081
:100EB000232AD104232CC104B337F600B386B7002C
:100EC0006FF01FE5E38804E4938787002328F1048B
:100ED00093B78700B386D700B3B7F600232AD104AF
:100EE00083268105B386D700232CD104B3B7F6003F
:100EF0006FF0DFFC93072000630AF90493073000CA
:100F00006304F90263140902378A0000232E0104E6
:100F1000232C0104232A010423280104130AFAFFC5
:100F2000136454006FF01FE6E38004FE9307F0FFA4
:100F3000378A0000232EF104232CF104232AF10424
:100F40002328F104130AEAFF6FF09FFDE38004FEFB
:100F50006FF09FFB130A1000631007088327010539
:100F6000832641050326810593F57700032AC105F1
:100F7000638E050493052000136414006306B9040E
:100F800093053000630AB9026312090493F5F70070
:100F900013054000638CA5029387470093B7470071
:100FA000B386F600B3B7F6003306F600B337F600A3
:100FB000330AFA006F008001639A04009387870068
:100FC00093B787006FF0DFFDE39A04FE135A4A01DE
:100FD000134A1A00137A1A00930610003387E6406A
:100FE0009307400763C2E726130B010513555740CB
:100FF00093060B00930A0000930700006392A70476
:101000001377F701931725006316070413063000C2
:1010100013070B00930600003306A640B305F70044
:1010200083A505009386160013074700232EB7FEFD
:10103000E356D6FE930740003385A7406F000007B4
:1010400003A606009387170093864600B3EACA00FA
:101050006FF0DFFA9308C0FFB30815039306010889
:10106000B386F60083A606FD93050002B385E5402E
:10107000B396B600B3EADA0093063000B307FB007C
:1010800013080000B386A6406340D80E93074000C3
:101090003385A7409396260093070108B386D700AF
:1010A0008327C10533D7E70023A8E6FC930B400054
:1010B0003386AB4013152500131626009305000058
:1010C0003305AB00EFF09ECA03270105B33750018B
:1010D000B3E7E7002328F10413F77700630E070452
:1010E000130720008325C10513641400630EE90C67
:1010F00013073000630EE9086310090413F7F700C3
:10110000630C770303264105938747002328F104E6
:1011100093B747003386C700B337F600232AC104CC
:10112000032681053386C700232CC1043336F6001D
:101130003307B600232EE1040327C105B7070800D3
:10114000B3F7E700638E070A232E0104232C010462
:10115000232A0104232801041364140063120A0ED5
:10116000130A10006FF01FC203A6070003A3470075
:10117000338E17013356E6003313B300336666002F
:101180002320CE0013081800938747006FF0DFEF8D
:10119000E39404FA83264105938787002328F1040A
:1011A00093B78700B386D700B3B7F600232AD104DC
:1011B00083268105B386D700232CD104B3B6F6006D
:1011C0003387B6006FF01FF7E38804F60327410565
:1011D00093878700832681052328F10493B787002E
:1011E0003387E700B337F700232AE1043387D700BA
:1011F000232CE1043337F7003307B7006FF09FF378
:101200009306CB0083270B0003274B00130B4B00E7
:1012100093D737001317D701B3E7E700232EFBFE60
:10122000E39266FF8327C10593D73700232EF1048D
:10123000E30A0AB4137A1400E3060AB4130A00009E
:10124000136424006FF01FB40327410583270105B1
:10125000B3E7E70003278105B3E7E7000327C105EC
:10126000B3E7E700638E0702232E0104232C010459
:10127000232A01042328D1049307200013641400B7
:10128000630EF902930730006302F90293075000DE
:10129000630209028327010593D737002328F1044D
:1012A00013642400130A00006FF0DFADE39404FE22
:1012B000930790002328F1046FF0DFFDE39A04FE0A
:1012C0006FF05FFD378A0000232E0104232C0104F8
:1012D000232A010423280104130AFAFF6FF09FAAAE
:1012E000130101F983A6050003A7450083A7850024
:1012F000232E3105232A510583A9C50023229105F8
:10130000930A050023261106232481062322910631
:1013100023202107232C410523286105232671055D
:10132000232481052320A1058328060003254600E8
:1013300083258600832CC600732A2000232CF1020B
:101340002324F100939709011399190093D70701FA
:101350002328D102232E31032320D100232AE102A6
:101360002322E1002326F1001359190193D9F90131
:10137000130801009306C10083A7060003A7C6FF58
:101380009386C6FF939737001357D701B3E7E7005B
:1013900023A2F600E312D8FE832B010093970C01E1
:1013A000139C1C00939B3B0093D70701232AA102A7
:1013B000232E9103232AA100232071012328110346
:1013C000232CB10223281101232CB100232EF1007C
:1013D000135C1C0193DCFC01130501011307C1011F
:1013E000832707000326C7FF1307C7FF939737001C
:1013F0001356D601B3E7C7002322F700E312E5FE38
:10140000032B0101B78700009387F7FF131B3B00F5
:10141000232861016310FC02032681018327410117
:10142000B3E7C7000326C101B3E7C700B3E767010D
:101430006394070093CC1C00B3078941E39C3C3DB7
:10144000635EF03883244100832C81000324C100B3
:1014500063140C1083254101832681010328C101F7
:1014600033E6D5003366060133666601631406046D
:10147000378700001307F7FF6392E70233E7940111
:101480003367870033677701630A07003707040073
:101490003377E40063140700130C00012320710369
:1014A00023229102232491032326810213090C0095
:1014B0006F00000A1386F7FF631A0604338B6B0173
:1014C000B3859500B33B7B0123206103338B75010A
:1014D000B33B7B01B3B59500B3E47501B3869601C8
:1014E000B3879600B3B49700B3B69601B3E69600FF
:1014F0003304880033848600232261032324F1020D
:1015000023268102930710006F00C01FB7860000DA
:101510009386F6FF6384D7006F10500033E7940181
:10152000336787003367770113090000630A0700F8
:1015300037090400337924011339190013194900BC
:101540002320710323229102232491032326810265
:10155000930500006F000074B78600009386F6FFC5
:101560006312D904B3E79401B3E78700B3E77701C7
:1015700013070000638A0700370704003377E4008D
:1015800013371700131747002320710323229102FA
:1015900023249103232681029307090013090700DE
:1015A0006FF01FFB8326C10137060800B3E6C600B3
:1015B000232ED1009306400763D4F6006F10C07647
:1015C000138607009357564093050700130B00003E
:1015D00093060000639EF6021376F60193962700A9
:1015E0006312060493053000B385F5403308D70035
:1015F000032808001306160013074700232E07FFD1
:10160000E3D6C5FE13074000B307F7406F0000079D
:1016100003A805009386160093854500336B0B01E4
:101620006FF05FFB1303C0FF3383670213070104EE
:101630003307D700032707FD130800023308C8400B
:1016400033170701336BEB003307D50093063000E7
:1016500093080000B386F64063CED8141307400009
:10166000B307F7409396260013070104B306D7008B
:101670000327C1013356C70023A8C6FC1306400048
:101680003306F640939727003305F500131626001E
:1016900093050000EFF08EED03270101B3376001E1
:1016A000B367F7002328F100832601018327410156
:1016B000B386DB00B387F400B3BB76012320D102ED
:1016C000B3867701B3BB76012322D1028326810141
:1016D000B3B49700B3E47401B386DC00B38796001B
:1016E000B3B69601832CC101B3B49700B3E696005C
:1016F00033049401338486002324F10223268102DB
:10170000930709000327C102B7060800B376D70084
:10171000639406006F108050B706F8FF9386F6FFBB
:101720003377D7002326E1020327010293871700AE
:101730001305C1029316F7011307010203260700E0
:101740008325470013074700135616009395F501AC
:101750003366B600232EC7FEE312E5FE0327C1025F
:10176000135717002326E1023337D00083260102E6
:1017700033E7E6002320E102378700001307F7FF75
:10178000E39EE700E3040A0613073000E31CEA06C1
:10179000E38E09049307F0FF2326F1022324F102CC
:1017A0002322F1022320F102B78700009387E7FF8D
:1017B0006F00D00483250700032E4700B30E670097
:1017C000B3D5C500331E0E01B3E5C50123A0BE008D
:1017D00093881800130747006FF01FE803244101A6
:1017E00083248101832CC10163820730B3072C411C
:1017F0006312091003264100032781000325C1005D
:10180000B365E600B3E5A500B3E57501639605048D
:10181000378700001307F7FF6392E70233679400EE
:101820003367970133676701630A070037070400CE
:1018300033F7EC0063140700130900012320610350
:101840002322810223249102232691039305000081
:101850006380072E6F0000449385F7FF63980504AB
:10186000B38B6B013306860033BB6B0123207103FE
:10187000B30B660133BB6B013336860033646601FC
:1018800033079700B307870033B4870033379700D7
:1018900033678700B30C9501B30C970123227103C2
:1018A0002324F102232691036FF0DFC53787000060
:1018B0001307F7FF6384E7006F1040483367940015
:1018C000336797013367670113090000630A070054
:1018D0003709040033F92C01133919001319490091
:1018E00023206103232281022324910223269103D2
:1018F0006FF01FC6378700001307F7FF6310EC0473
:10190000B3679400B3E79701B3E7670113090000D9
:10191000638A07003709040033F92C0113391900D1
:1019200013194900232061032322810223249102F9
:101930002326910393070C006FF09FC10327C1007A
:10194000370608003367C7002326E1001307400766
:101950006354F7006F10403F938507009307000220
:10196000B3C7F50213860600130900001307000031
:101970006346F7041386070063D4070013060000CC
:1019800013F5F50113972700631405049305300040
:1019900013060000B385F5403385E60003250500F6
:1019A000130616009386460023AEA6FEE3D6C5FEB8
:1019B00013054000B307F5406F00800703250600BC
:1019C00013071700130646003369A9006FF05FFA8A
:1019D00013050002B3E5A5021303C0FF930601043B
:1019E000131626003386C600832606FC93080000E3
:1019F000338367023305B540B396A6003369D90037
:101A0000B306E800130730003307F74063CCE80A59
:101A100093060104131727003387E6008326C100CD
:101A200013054000B307F540B3D5B6002320B7FC3B
:101A300013074000130600006346F7003307F74022
:101A400013162700939727003305F800930500002D
:101A5000EFF0CEB103270100B3372001B367F700E1
:101A60002320F1008327010003274100B307FB0077
:101A70003307E40033BB67012320F102B30767019A
:101A800033BB67012322F1028327810033348700AF
:101A900033646401B387F40033878700B3B79700DA
:101AA0008324C10033348700B3E78700B38C9C00E4
:101AB000B38C97012324E1022326910393070C00A2
:101AC0006FF05FC403A6060003AE4600B38E660047
:101AD0003356B600331EAE003366C60123A0CE00D7
:101AE00093881800938646006FF05FF237860000F7
:101AF000930719009305E6FFB3F5B70003284100EB
:101B0000832881008326C10063960540B3671801CE
:101B1000B3E7D700B3E77701631C09306394070E7E
:101B2000232061032322810223249102232691038F
:101B30008325010203264102832681020327C10275
:101B4000B3E7C500B3E7D700B3E7E7006394070046
:101B50006F100010232AC1022328B102232CD102C6
:101B6000232EE102130601039307C10303A7070015
:101B700083A6C7FF9387C7FF1317170093D6F601F5
:101B80003367D70023A2E700E312F6FE83270103A1
:101B90009397170013F77700631407006F10C009BD
:101BA000130720008326C103136919006314EA0098
:101BB0006F104008130730006314EA006F108006AE
:101BC00063040A006F10400713F7F7001306400084
:101BD0006314C7006F1040069387470093B7470010
:101BE000032741033387E7003337F7008327810357
:101BF000B307F700B3B7E700B387D700232EF1028E
